:100000000C948C1E0C94BD1E0C94BD1E0C94BD1E35
:100010000C94BD1E0C94BD1E0C94BD1E0C94BD1EF4
:100020000C94BD1E0C94BD1E0C94BD1E0C94BD1EE4
:100030000C94BD1E0C94BD1E0C94BD1E0C94BD1ED4
:100040000C94BD1E0D94CA1A0C94BD1E0C94BD1EBA
:100050000C94BD1E0C94BD1E0C9412CE0C94669193
:100060000C94BD1E0C94A3480C9499480C94BD1E8E
:100070000C94BD1E0C94BD1E0C94BD1E0C94BD1E94
:100080000C94BD1E0C94BD1E0C94BD1E0C94BD1E84
:100090000C94BD1E0C94BD1E0C94BD1E0C94BD1E74
:1000A0000C94BD1E0C94BD1E0C94BD1E0C94BD1E64
:1000B0000C94BD1E0C94BD1E0C94BD1E0C94BD1E54
:1000C0000C94BD1E0C94BD1E0C94BD1E0C94BD1E44
:1000D0000C94BD1E0C94BD1E0C94BD1E0C94BD1E34
:1000E0000C94BD1E79775C775F777C776277657754
:1000F000687774776B7787776E777177D8CC9ACD7E
:100100009FCDB2CDB7CDCACDD6CDC8CCABE2DDE266
:10011000DFE2ECE2F1E2A9E2FAE280FC83FC72FCAD
:1001200076FC7CFCBAFC87FC8BFC91FC95FC99FC72
:100130009FFCA3FCA7FCBAFCADFCB1FCB5FCDD0048
:10014000FB00F100F500DB00F900D700F300EF0041
:10015000E100D900E300E700DF00F900E900F70063
:10016000E500084AD73B3BCE016E84BCBFFDC12FE2
:100170003D6C74319ABD56833DDA3D00C77F11BE98
:10018000D9E4BB4C3E916BAAAABE000000803F059B
:10019000A84CCDB2D44EB93836A9020C50B99186CC
:1001A00088083CA6AAAA2ABE000000803F000D9441
:1001B000C6010D94EA010D94BC010D949E010D94AD
:1001C0000D020D94E0010D94F4010D942B020D9499
:1001D00003020D9417020D94C5220D94DE230D9495
:1001E000D6010D94A8010D94CE010D94B2010D9489
:1001F00021020D9435020D94A3014E414E494E4902
:100200005459494E46CDCCCC3D0AD7233C17B7D1E3
:100210003877CC2B329595E6241FB14F0A00002089
:10022000410000C84200401C4620BCBE4CCA1B0E08
:100230005AAEC59D7400407A10F35A00A0724E1851
:10024000090010A5D4E80000E87648170000E40B88
:1002500054020000CA9A3B000000E1F5050000804E
:10026000969800000040420F000000A086010000A8
:1002700000102700000000E80300000000640000F8
:100280000000000A00000000000100000000002C37
:1002900076D888DC674F0823DFC1DFAE59E1B1B7FC
:1002A00096E5E3E453C63AE651997696E8E6C284C9
:1002B00026EB898C9B62ED407C6FFCEFBC9C9F40E1
:1002C000F2BAA56FA5F490055A2AF75C936B6CF906
:1002D000676DC11BFCE0E40D47FEF520E6B500D0DC
:1002E000ED902E0300943577050080841E080000F1
:1002F000204E0A000000C80C333333330F986E12BF
:10030000831141EF8D2114893BE65516CFFEE6DBC4
:1003100018D1844B381BF77C1D901DA4BBE424200E
:100320003284725E228100C9F124ECA1E53D2743AD
:100330004F4D4D554E49434154494F4E004452593B
:1003400052554E004552524F525300494E464F00AF
:100350004543484F0047322F473320626164207085
:100360006172616D65746572730A00536C656570C6
:100370002E2E2E00436C69636B20746F20526573C0
:10038000756D652E2E2E004E6F204D6F76652E00FA
:10039000456E642066696C65206C6973740A00425E
:1003A0006567696E2066696C65206C6973740A0004
:1003B000286E6F2066696C65290043757272656EE0
:1003C000742066696C653A20005344207072696E2F
:1003D00074696E67206279746520004E6F742053D3
:1003E00044207072696E74696E670A002E0A0044B8
:1003F000656C6574696F6E206661696C65642C203C
:1004000046696C653A200046696C652064656C65D8
:100410007465643A002569730025696D2025697348
:10042000002569682025696D2025697300256964A8
:10043000202569682025696D202569730025697963
:1004400020256964202569682025696D2025697348
:10045000005072696E742074696D653A2000436FB4
:100460006F6C696E672E2E2E0048656174696E6729
:100470002E2E2E00452563202553006F6B006F66DE
:10048000660050034B0344033D032F03444542558C
:10049000473A004D3131322053687574646F776E7E
:1004A000004D313133205300436C696D6265722019
:1004B00037204F46462E004348414D4245525F5437
:1004C000454D5045524154555245004D4F54494FAA
:1004D0004E5F4D4F44455300544845524D414C5F8B
:1004E00050524F54454354494F4E004155544F527A
:1004F00045504F52545F53445F5354415455530039
:1005000050524F4D50545F535550504F5254004528
:100510004D455247454E43595F5041525345520055
:10052000434153455F4C494748545F42524947480D
:10053000544E45535300544F47474C455F4C494731
:1005400048545300534F4654574152455F504F57FC
:100550004552004255494C445F50455243454E5424
:10056000004C4556454C494E475F44415441005A62
:100570005F50524F4245004155544F4C4556454CF3
:10058000005052494E545F4A4F420050524F47521A
:10059000455353004155544F5245504F52545F54A8
:1005A000454D5000564F4C554D455452494300451A
:1005B0004550524F4D0042494E4152595F46494CB9
:1005C000455F5452414E53464552005345524941AE
:1005D0004C5F584F4E5F584F4646004649524D5764
:1005E0004152455F4E414D453A4D61726C696E20F6
:1005F00058544C5720334420284769744875622961
:1006000020534F555243455F434F44455F55524C2D
:100610003A68747470733A2F2F6769746875622E24
:10062000636F6D2F4D61726C696E4669726D776193
:1006300072652F4D61726C696E2050524F544F435A
:100640004F4C5F56455253494F4E3A312E30204D54
:10065000414348494E455F545950453A436C696D92
:1006600062657220372045585452554445525F43C5
:100670004F554E543A3220555549443A436C696DB2
:1006800062657220370A002F2F20004D313435204B
:10069000533C696E6465783E206F7574206F6620E8
:1006A00072616E67652028302D31290A00205400C0
:1006B000205200416363656C65726174696F6E3AC4
:1006C000205000486F74656E64206F6666736574B1
:1006D000733A0020466C6F773A200050726F746551
:1006E000637465642050696E0A00496E76616C69B6
:1006F000642065787472756465720A0020643A003B
:1007000020693A0020703A0020653A004C434420AA
:10071000436F6E74726173743A200064697300658C
:100720006E0043290A0061626C656420286D696E61
:100730002074656D702000436F6C6420657874725E
:10074000756465732061726520004F4646004F4E08
:100750000046696C616D656E742072756E6F75749C
:1007600020004F666673657473204170706C696514
:1007700064004572723A20546F6F206661722100E6
:10078000546F6F206661722066726F6D20726566AD
:100790006572656E636520706F696E740A00454509
:1007A00050524F4D204F4B0A00486F6D696E6720C5
:1007B00058595A004C6F61642046696C616D656ED2
:1007C00074202A004C6F6164206D6D00556E6C6F53
:1007D00061642046696C616D656E74202A00556EF7
:1007E0006C6F6164206D6D0046696C2E20446961F8
:1007F0002E202A0046696C2E204469612E00452077
:10080000696E206D6DC2B3004D33303320553120F9
:100810004525692053256900504944204175746F6E
:1008200074756E65202A005049442D44202A0050DA
:1008300049442D49202A005049442D50202A0020A7
:10084000082046616374002008204D61780020086C
:10085000204D696E004F6666004F6E004175746FE3
:1008600074656D70004572726F7220777269746979
:100870006E6720746F20454550524F4D210A003657
:10088000372603023C3D380F2E303E12282A3F1AED
:100890001C1824221E08440A414307414508094107
:1008A00042420001627573793A2070617573656424
:1008B00020666F7220696E7075740A0062757379B4
:1008C0003A2070617573656420666F722075736578
:1008D000720A00627573793A2070726F6365737380
:1008E000696E670A004D3630300053544F50504502
:1008F000442E20005072696E7465722073746F709C
:100900007065642064756520746F206572726F7203
:10091000732E2046697820746865206572726F7244
:1009200020616E6420757365204D39393920746FEC
:1009300020726573746172742E202854656D706521
:100940007261747572652069732072657365742EA7
:100950002053657420697420616674657220726525
:100960007374617274696E67290A004E6F20436860
:1009700065636B73756D2077697468206C696E654B
:10098000206E756D6265722C204C617374204C6909
:100990006E653A20004E6F20436865636B73756D1A
:1009A0002077697468206C696E65206E756D62656C
:1009B000722C204C617374204C696E653A20006380
:1009C0006865636B73756D206D69736D61746368C1
:1009D0002C204C617374204C696E653A20004C6980
:1009E0006E65204E756D626572206973206E6F743E
:1009F000204C617374204C696E65204E756D626584
:100A0000722B312C204C617374204C696E653A2036
:100A1000004D313130004D313137004D333100530D
:100A2000442072656164206572726F720A00446FBF
:100A30006E65207072696E74696E672066696C6598
:100A40000A002121204B494C4C2063617573656479
:100A5000206279204B494C4C20627574746F6E2F64
:100A600070696E0A002121204B494C4C206361754E
:100A700073656420627920746F6F206D75636820E0
:100A8000696E6163746976652074696D65202D20D7
:100A900063757272656E7420636F6D6D616E643A1A
:100AA0002000FFE0FFD140A0C8A6A22FF80023AC91
:100AB00000AF10FFFEFF05FFD0FFE0FFC1FFD1E256
:100AC00040A0C8A6A22FF800238127AC00AFFFD01A
:100AD000FF64FFD1A5FFD0FF64FF64FFD1A4FFD066
:100AE000FFFE000C0D00FE07022603BC017FFE087E
:100AF000FE08FE05080806000040F0C888889878BF
:100B000010050808060000C0F88888888888F8055D
:100B100005050600012030F8302005080806000011
:100B20002070F820202020E00509090600FF207031
:100B3000A8A8B888887020050606060001E08CEA9F
:100B40008C8A0A0509090600FFF8A8888888888821
:100B5000A8F8050A0A0600FE205050505088A8A8A0
:100B6000887003030306000340A040FFFFFFFFFF60
:100B7000FFFFFFFFFFFFFFFFFFFFFFFFFFFFFFFF85
:100B8000FF0000000605FF010707060200808080C5
:100B900080800080030303060105A0A0A0050606CF
:100BA00006000050F85050F8500509090600FF20D3
:100BB00070A8A07028A87020050707060000C8C804
:100BC000102040989805070706000040A0A040A804
:100BD000906801030306020580808003090906016D
:100BE000FF2040408080804040200309090601FF2B
:100BF000804040202020404080050707060000205C
:100C0000A8702070A8200505050600012020F82006
:100C1000200203030601FFC0408005010106000316
:100C2000F8020202060100C0C0050707060000081E
:100C3000101020404080050707060000708898A823
:100C4000C8887003070706010040C040404040E0EC
:100C5000050707060000708808102040F805070700
:100C6000060000F808103008887005070706000025
:100C700010305090F81010050707060000F880F0BB
:100C800008088870050707060000304080F0888853
:100C900070050707060000F808101020202005073F
:100CA00007060000708888708888700507070600AE
:100CB0000070888878081060020505060100C0C031
:100CC00000C0C00206060601FFC0C000C04080038D
:100CD00005050601012040804020050303060002AF
:100CE000F800F80305050601018040204080050753
:100CF0000706000070881020200020050707060066
:100D0000007088B8A8B880700507070600007088D2
:100D100088F8888888050707060000F0484870486A
:100D200048F00507070600007088808080887005FD
:100D30000707060000F04848484848F0050707063E
:100D40000000F88080F08080F8050707060000F8B2
:100D50008080F08080800507070600007088808012
:100D6000988870050707060000888888F8888888B2
:100D7000030707060100E04040404040E005070748
:100D800006000038101010109060050707060000DC
:100D90008890A0C0A090880507070600008080808A
:100DA000808080F805070706000088D8A888888812
:100DB000880507070600008888C8A898888805075E
:100DC0000706000070888888888870050707060075
:100DD00000F08888F0808080050707060000708892
:100DE0008888A89068050707060000F08888F0A0AA
:100DF00090880507070600007088807008887005D5
:100E00000707060000F820202020202005070706FD
:100E10000000888888888888700507070600008891
:100E20008888885050200507070600008888888831
:100E3000A8A8500507070600008888502050888819
:100E40000507070600008888502020202005070796
:100E5000060000F80810204080F80309090601FF89
:100E6000E080808080808080E005070706000080A9
:100E70004040201010080309090601FFE02020204F
:100E800020202020E00503030600052050880501EE
:100E9000010600FEF8030303060105804020050556
:100EA00005060000700878887805070706000080AE
:100EB00080F0888888F0050505060000708080882D
:100EC00070050707060000080878888888780505F7
:100ED000050600007088F0807005070706000030E6
:100EE0004840E04040400507070600FE70888888BB
:100EF0007808700507070600008080F088888888D9
:100F00000307070601004000C0404040E004090913
:100F10000601FE1000301010101090600507070643
:100F2000000080808890E09088030707060100C0D9
:100F30004040404040E0050505060000D0A8A8A8B4
:100F4000A8050505060000B0C888888805050506BF
:100F5000000070888888700507070600FEF0888802
:100F600088F080800507070600FE78888888780862
:100F700008050505060000B0C88080800505050647
:100F8000000078807008F00507070600002020F8B0
:100F90002020201805050506000088888898680527
:100FA0000505060000888888502005050506000014
:100FB0008888A8A85005050506000088502050889C
:100FC0000507070600FE8888885020408005050533
:100FD000060000F8102040F80309090601FF204030
:100FE000404080404040200109090602FF80808087
:100FF0008080808080800309090601FF8040404096
:10100000204040408005030306000248A890FF43AB
:10101000616E6E6F7420656E7465722073756264A4
:1010200069723A2000022E2E004D61696E004D6FEC
:1010300076652025736D6D00004D6F766520302E2E
:10104000316D6D004D6F766520316D6D004D6F76A1
:10105000652031306D6D00486F74656E6420746F6B
:101060006F20636F6C6400457874727564657220DC
:101070002A004578747275646572005431005430EA
:101080000053656C656374202A004D6F7665205AA5
:10109000004D6F76652059004D6F76652058004DE4
:1010A0006F74696F6E004D38340044697361626C0F
:1010B00065205374657070657273004C6576656C5D
:1010C000696E6700473238004175746F20486F6D54
:1010D00065004D6F76652041786973004D61696EDA
:1010E00000466C6F77207E00466C6F770046616E1D
:1010F00020537065656400426564004E6F7A7A6CB7
:1011000065207E005370656564004D61696E004D19
:1011100032313920543120582B302E3035004D32A9
:10112000313920543120582B302E3130004D32319E
:101130003920543120582B302E3135004D32313981
:1011400020543120582B302E3230004D323139208E
:10115000543120582B302E3235004D323139205445
:101160003120582B302E3330004D3231392054315C
:1011700020582B302E3335004D3231392054312058
:10118000582B302E3430004D323139205431205814
:101190002B302E3435004D32313920543120582B2C
:1011A000302E3530004D32313920543120582B301B
:1011B0002E3535004D32313920543120582B302E08
:1011C0003630004D32313920543120582B302E36F4
:1011D00035004D32313920543120582B302E3730E4
:1011E000004D32313920543120582B302E37350004
:1011F0004D32313920543120582B302E3830004DAB
:1012000032313920543120582B302E3835004D32B0
:10121000313920543120582B302E3930004D3231A5
:101220003920543120582B302E3935004D32313988
:1012300020543120582B312E30300058206C696EEC
:10124000653A2D31360058206C696E653A2D31357E
:101250000058206C696E653A2D31340058206C6955
:101260006E653A2D31330058206C696E653A2D3128
:10127000320058206C696E653A2D31310058206C6F
:10128000696E653A2D31300058206C696E653A2DD3
:1012900031380058206C696E653A2D390058206C41
:1012A000696E653A2D380058206C696E653A2D37A5
:1012B0000058206C696E653A2D360058206C696EB6
:1012C000653A2D31390058206C696E653A2D35002C
:1012D00058206C696E653A2D31370058206C696E64
:1012E000653A2D340058206C696E653A2D330058EC
:1012F000206C696E653A2D320058206C696E653A33
:101300002D310058206C696E653A2D3230005654EC
:10131000726176204D696E00566D696E00566D6182
:1013200078204500566D6178205A00566D6178200E
:101330005900566D6178205800416D617820450054
:10134000416D6178205A00416D6178205900416DEE
:101350006178205800412D54726176656C00412DF2
:101360005265747261637400416363656C00566515
:101370002D4A65726B00565A2D4A65726B0056599C
:101380002D4A65726B0056582D4A65726B00457385
:10139000746570732F6D6D005A73746570732F6D63
:1013A0006D005973746570732F6D6D00587374659B
:1013B00070732F6D6D00416476616E6365642053B8
:1013C000657474696E6773003F0043616E63656C9A
:1013D00000496E6974004D34323800496E69746991
:1013E000616C697A6520454550524F4D0046696CE5
:1013F000616D656E740054656D70657261747572AF
:10140000650053746570732F6D6D004A65726B00D3
:10141000416363656C65726174696F6E0056656CDB
:101420006F636974790053657420486F6D65204F50
:1014300066667365747300436F6E66696775726183
:1014400074696F6E005A2052616973650042656469
:10145000004E6F7A7A6C650046616E205370656548
:101460006400436F6E66696775726174696F6E00C0
:101470004C6F61642053657474696E6773005265C4
:1014800073746F7265206661696C73616665005381
:10149000746F72652053657474696E67730050725F
:1014A00065686561742041425320436F6E66005049
:1014B00072656865617420504C4120436F6E660010
:1014C0004F6666004F6E0052756E6F7574205365DF
:1014D0006E736F72004C434420436F6E747261737D
:1014E0007400546F6F6C204368616E6765004944F7
:1014F000452D582053657400416476616E636564C0
:101500002053657474696E6773004D61696E004D98
:1015100037303220542564004D36303020423020A0
:10152000542564004D373032203B2564004D373060
:101530003120542564004368616E67652046696CFC
:10154000616D656E7400556E6C6F61642046696CE8
:10155000616D656E74004C6F61642046696C616DED
:10156000656E740050726568656174204142530075
:101570005072656865617420437573746F6D0050B7
:1015800072656865617420504C41004261636B0074
:10159000554E4C4F41442046494C414D454E540018
:1015A0004C4F41442046494C414D454E540046491C
:1015B0004C414D454E54204348414E4745004D3621
:1015C000303020423020542569004D3730312054CE
:1015D0002569004D37303220542569004C6F616415
:1015E0002046696C616D656E74202A00556E6C6FC3
:1015F00061642046696C616D656E74202A004368E1
:10160000616E67652046696C616D656E74202A00A5
:101610004D61696E004F6666004F6E0052756E6FC9
:1016200075742053656E736F720050757267652014
:101630006D6F726500436F6E74696E75650052451B
:1016400053554D45204F5054494F4E533A00505238
:10165000494E54205041555345440020204E6F7A46
:101660007A6C653A20005061726B696E672E2E2E7F
:101670000000005761697420666F720066696C61D2
:101680006D656E74206368616E676500746F2073AA
:1016900074617274005761697420666F72006669C4
:1016A0006C616D656E7420756E6C6F616400004EC8
:1016B0006F7A7A6C652068656174696E6700506C3A
:1016C0006561736520776169742E2E2E000050725B
:1016D00065737320627574746F6E00746F20686533
:1016E0006174206E6F7A7A6C650000496E73657262
:1016F000742066696C616D656E7400616E64207043
:101700007265737320627574746F6E00746F2063FA
:101710006F6E74696E7565005761697420666F72CB
:101720000066696C616D656E74206C6F61640000A9
:10173000507265737320427574746F6E00746F20FD
:10174000726573756D65207072696E740000576103
:10175000697420666F72207072696E7400746F20F5
:10176000726573756D652E2E2E00005761697420A9
:10177000666F720066696C616D656E74207075725B
:10178000676500003F004261636B0053746F700037
:101790005072696E742066726F6D204D6564696168
:1017A000004D3231004368616E6765204D656469A4
:1017B00061004368616E67652046696C616D656EA6
:1017C0007400436F6E66696775726174696F6E004D
:1017D00054656D7065726174757265004D6F7469E2
:1017E0006F6E00526573756D65205072696E74007E
:1017F0004E6F204D656469610054756E65005374C9
:101800006F70205072696E7400506175736520505E
:1018100072696E7400496E666F2053637265656EFF
:10182000003F005374617274205072696E740043FB
:10183000616E63656C005072696E74001FE0201069
:101840002310249010A011202210241037B008403B
:10185000048003001FE02010211023101520112008
:101860002110211031300840048003001FE03FF0B8
:101870003CF03B701F601EE03DF03BF038700FC045
:10188000078003001FE03FF03EF03CF01AE01EE04E
:101890003EF03EF03EF00FC00780030047323800B4
:1018A00053746F72652053657474696E6773004179
:1018B000646A757374205A20486F6D65004C6576B4
:1018C000656C20436F726E657273004C6576656C53
:1018D000204E6F7A7A6C6500326E64204E6F7A7A91
:1018E0006C65205A004D6F74696F6E002568753AFB
:1018F00025303268750025303268753A25303268F7
:101900007500256875642025303268753A253032B7
:1019100068750054183C1884186C183FFFF03800A4
:101920007030FC3020FC102078102030102C00D0BB
:101930002E31D02F7BD02F7BD02E31D02C00D02039
:10194000301020781020FC1030FC303800703FFF41
:10195000F03FFFF0380070318630238710278790E2
:101960002F87D02F03D0203010207810207810201F
:1019700030102F03D02F87D02787902387103186F0
:10198000303800703FFFF01FFFF81FFFF8041040D1
:101990000208200208200410400820801041001096
:1019A00041000820800410400000001FFFF81FFFC6
:1019B000F8290A002062797465733B206372632002
:1019C0000053657474696E67732053746F72656435
:1019D000202800454550524F4D2064617461736961
:1019E0007A65206572726F722E0A00290A002062E1
:1019F000797465733B2063726320002073746F7287
:101A000065642073657474696E677320726574729F
:101A10006965766564202800202863616C63756CB5
:101A20006174656429210A0020213D20004545504C
:101A3000524F4D20435243206D69736D617463684A
:101A4000202D202873746F7265642920002053694B
:101A50007A653A2000496E6465783A2000204D612D
:101A6000726C696E3D563735290A00454550524F14
:101A70004D2076657273696F6E206D69736D617448
:101A800063682028454550524F4D3D004D32313955
:101A900020543120592D302E3035004D323139202F
:101AA000543120592D302E3130004D3231392054EF
:101AB0003120592D302E3135004D323139205431FD
:101AC00020592D302E3230004D3231392054312002
:101AD000592D302E3235004D3231392054312059B4
:101AE0002D302E3330004D32313920543120592DD4
:101AF000302E3335004D32313920543120592D30BC
:101B00002E3430004D32313920543120592D302EB1
:101B10003435004D32313920543120592D302E3595
:101B200030004D32313920543120592D302E353589
:101B3000004D32313920543120592D302E363000AD
:101B40004D32313920543120592D302E3635004D4B
:101B500032313920543120592D302E3730004D325A
:101B6000313920543120592D302E3735004D323146
:101B70003920543120592D302E3830004D32313932
:101B800020543120592D302E3835004D3231392036
:101B9000543120592D302E3930004D3231392054F6
:101BA0003120592D302E3935004D32313920543104
:101BB00020592D312E30300059206C696E653A3134
:101BC000360059206C696E653A31350059206C69D0
:101BD0006E653A31340059206C696E653A313300D4
:101BE00059206C696E653A31320059206C696E6516
:101BF0003A31380059206C696E653A31310059200C
:101C00006C696E653A31390059206C696E653A31FC
:101C1000300059206C696E653A390059206C696E44
:101C2000653A380059206C696E653A370059206C66
:101C3000696E653A360059206C696E653A3230003B
:101C400059206C696E653A350059206C696E653AA9
:101C5000340059206C696E653A31370059206C693F
:101C60006E653A330059206C696E653A320059202E
:101C70006C696E653A31004D32313920543120584B
:101C80002B312E3030004E6F204C696E6520416C38
:101C900069676E6D656E740058206C696E653A31C7
:101CA00020746F2032300058206C696E653A2D31F7
:101CB00020746F202D323000436C696D6265722094
:101CC000370058544C5720334400000000000000F7
:101CD0000000000000000000000000000000000004
:101CE00000000000000000000000000000000000F4
:101CF00000000000000000000000000000000000E4
:101D000000000000000000000000000000000000D3
:101D100000000000000000000000000000000000C3
:101D200000000000000000000000000000000000B3
:101D300000000000000000000000000000000000A3
:101D40000000000000000000000000000000000093
:101D50000000000000000000000000000000000083
:101D600000000000001F00F03FFFF81F0000787C1B
:101D70001C00000E00C03038180E0000303818006B
:101D80000007008060380C0E0000381810000003B7
:101D900081004038000E0000381C10000001C20015
:101DA0000038000E0000181C30000000E40000386D
:101DB000000E00001C3C2000000078000038000EDF
:101DC00000001C2C2000000038000038000E00002D
:101DD0000C6E600000003C000038000E00000C4E4D
:101DE000400000006E000038000E00000EC64000EB
:101DF0000000C7000038000E00000E86C000000181
:101E000087800038000E000007878000000303C0B1
:101E10000038000E000407838000000601C000386F
:101E2000000E000807038000000C00F00038000ED0
:101E3000003803030000007E01FC01FF007FFFF07B
:101E4000020300000000000000000000000000008D
:101E50000000000000000000000000000000000082
:101E60000000000000000000000000000000000072
:101E70000000000000000000000000000000000062
:101E80000000000000000000000000000000000052
:101E90000000000000000000000000000000000042
:101EA0000000000000000000000000000000000032
:101EB0000000000000000000000000000000000022
:101EC00000002020506C616E6E657242756666651A
:101ED0007242797465733A20002046726565204D20
:101EE000656D6F72793A2000436F6D70696C65643F
:101EF0003A2046656220323820323032300A0020E3
:101F00004C61737420557064617465643A2032309A
:101F100032302D30312D3237207C20417574686F7E
:101F2000723A2058544C5733440A0058544C5720A6
:101F300033440A004D61726C696E0020536F667401
:101F4000776172652052657365740A002057617469
:101F50006368646F672052657365740A002042727B
:101F60006F776E206F75742052657365740A002058
:101F700045787465726E616C2052657365740A00F1
:101F8000506F77657255700A0073746172740A003D
:101F90006175746F25632E67004739310A47312018
:101FA0005A2B302E3520452D313620592B313020FB
:101FB00046393030300A47323858590A4D383400E3
:101FC0006572726F722077726974696E6720746FC0
:101FD0002066696C650A00446F6E652073617669DE
:101FE0006E672066696C652E0A004D323900456EB9
:101FF0006473746F7073002553202563202563205C
:10200000256320256300205A3A0020593A002058C1
:102010003A00656E6473746F7073206869743A2057
:10202000004361703A00220A00656E71756575653E
:10203000696E672022006F6B00526573656E643AAB
:10204000200020573A0042656420436F6F6C696E30
:10205000672E2E2E004265642048656174696E67A4
:102060002E2E2E0023646566696E65204445464128
:10207000554C545F004B6420004B6920004B70208E
:1020800000504944204175746F74756E652066690F
:102090006E697368656421205075742074686520CA
:1020A0006C617374204B702C204B6920616E64202E
:1020B0004B6420636F6E7374616E74732066726F0D
:1020C0006D2062656C6F7720696E746F20436F6E50
:1020D00066696775726174696F6E2E680A0050498F
:1020E00044204175746F74756E65206661696C6516
:1020F00064212074696D656F75740A005468657297
:102100006D616C2052756E6177617900486561740C
:10211000696E67206661696C6564005049442041BE
:1021200075746F74756E65206661696C65642120D5
:1021300054656D706572617475726520746F6F207F
:10214000686967680A00204B643A2000204B693AAE
:102150002000204B703A20000A20436C61737369A1
:102160006320504944200A00204B643A2000204B51
:10217000693A2000204B703A20000A204E6F206FF1
:1021800076657273686F6F740A002054753A200088
:10219000204B753A2000206D61783A2000206D694F
:1021A0006E3A200020643A200020626961733A2070
:1021B00000504944204175746F74756E65207374C6
:1021C0006172740A00504944204175746F74756ED1
:1021D00065206661696C6564212054656D70657267
:1021E000617475726520746F6F20686967680A0092
:1021F000504944204175746F74756E65206661693D
:102200006C65642120426164206578747275646530
:1022100072206E756D6265720A004572723A2075A1
:1022200074663820666F6E74206E6F7420696E69F4
:102230007469616C697A65642E004572723A207522
:1022400074663820666F6E74206E6F7420696E69D4
:102250007469616C697A65642E004572723A207502
:1022600074663820666F6E74206E6F7420696E69B4
:102270007469616C697A65642E00486F74656E6478
:10228000206F6666736574733A00204D39322058AA
:102290000020204D61783A2000200020204D696EFA
:1022A0003A2000536F667420656E6473746F7073A8
:1022B0003A200073706563696679696E67204458D7
:1022C000435F4D4952524F5245445F4D4F44452E56
:1022D0000A005072696E746572206D7573742062A5
:1022E0006520696E204458435F4455504C49434132
:1022F00054494F4E5F4D4F4445207072696F7220B4
:10230000746F200A0020496E76616C6964206578DC
:10231000747275646572200024F4D43050C38E202A
:10232000C2A24017828B7011127A910D816CD90A6A
:10233000A861E108C7586607615143061E4B5D0559
:10234000C145A7041A411104093D980371393103AD
:102350004036DB0265339102D4305402802E1D02D8
:10236000632CEE01752AC501B028A0011027810158
:102370008F2564012B244B01E0223401AC211F0185
:102380008D200D01801FFC00841EED00971DDF00D5
:10239000B81CD200E61BC600201BBC00641AB200A9
:1023A000B219A8000A19A0006A189900D117910063
:1023B00040178B00B516840031167E00B3157900E6
:1023C0003A157300C7146F0058146A00EE136600C4
:1023D0008813630025135E00C7125B006C12570060
:1023E00015125400C111510070114F0021114B0002
:1023F000D61049008D1047004610440002104200DC
:10240000C00F4000800F3E00420F3C00060F3B0013
:10241000CB0E3800930E37005C0E3500270E3400CB
:10242000F30D3200C10D3100900D3000600D2E0013
:10243000320D2D00050D2C00D90C2B00AE0C2900FF
:10244000850C29005C0C2700350C27000E0C26009B
:10245000E80B2400C40B2400A00B23007D0B2300F9
:102460005A0B2100390B2100180B2000F80A1F001D
:10247000D90A1E00BB0A1E009D0A1D00800A1D000D
:10248000630A1C00470A1B002C0A1B00110A1A00D1
:10249000F7091A00DD091900C4091900AB09190070
:1024A000920917007B091800630917004C091600F0
:1024B00036091600200916000A091500F50815004E
:1024C000E0081400CC081400B8081400A408140094
:1024D000900813007D0812006B08130058081200C2
:1024E00046081200340811002308110012081100D8
:1024F00001081100F0071000E0071000D0071000DD
:10250000C0071000B0070F00A107100091070E00D0
:1025100083070F0074070F0065070E0057070E00B2
:1025200049070E003B070D002E070E0020070D0087
:1025300013070D0006070D00F9060C00ED060D004F
:10254000E0060C00D4060C00C8060C00BC060C000B
:10255000B0060C00A4060B0099060C008D060B00BB
:1025600082060B0077060B006C060B0061060A0062
:1025700057060B004C060A0042060A0038060A00FD
:102580002E060A0024060A001A060A001006090090
:1025900007060A00FD050900F4050900EB0509001E
:1025A000E2050900D9050900D0050900C7050900A1
:1025B000BE050900B5050800AD050800A505090020
:1025C0009C050800940508008C0508008405080097
:1025D0007C050800740508006C0507006505080007
:1025E0005D050700560508004E0507004705070072
:1025F0004005080038050700310507002A050700D7
:10260000230507001C050600160507000F05070037
:102610000805060002050700FB040600F504070094
:10262000EE040600E8040600E2040700DB040600EE
:10263000D5040600CF040600C9040600C304060042
:10264000BD040600B7040600B1040500AC04060092
:10265000A6040600A00405009B04060095040500DE
:10266000900406008A040500850405008004060025
:102670007A04050075040500700405006B0405006C
:1026800066040500610405005C04050057040500AC
:10269000520405004D0405004804050043040500EC
:1026A0003E0404003A04050035040500300404002B
:1026B0002C04050027040400230405001E04040064
:1026C0001A04040016040500110404000D0404009B
:1026D000090405000404040000040400FC030400D1
:1026E000F8030400F4030400F0030400EC03040006
:1026F000E8030400E4030400E0030400DC03040036
:10270000D8030400D4030400D0030400CC03040065
:10271000C8030300C503030024F404D9201BC40C20
:102720005C0E9804C4095F0265077101F405F900A5
:10273000FB04B30048048700C10369005803550037
:1027400003034500BE023A008402310053022A000E
:102750002902250004022000E4011C00C801190020
:10276000AF011700980114008401130071011000DB
:102770006101100051010E0043010D0036010B00F4
:102780002B010B0020010B00150109000C010900B1
:1027900003010800FB000800F3000800EB0007003D
:1027A000E4000600DE000600D8000600D2000600A5
:1027B000CC000500C7000500C2000500BD000400F4
:1027C000B9000400B5000400B1000400AD0004002D
:1027D000A9000400A5000300A20003009F0004005C
:1027E0009B00030098000300950002009300030083
:1027F000900003008D0002008B000300880002009F
:102800008600020084000300810002007F000200B5
:102810007D0002007B0002007900020077000100C9
:1028200076000200740002007200010071000200D4
:102830006F0002006D0001006C0002006A000100E0
:1028400069000200670001006600010065000100E8
:1028500064000200620001006100010060000100EC
:102860005F0002005D0001005C0001005B000100F0
:102870005A000100590001005800010057000100F2
:1028800056000100550001005400010053000000F3
:1028900053000100520001005100010050000100EE
:1028A0004F0001004E0000004E0001004D000100ED
:1028B0004C0001004B0000004B0001004A000100E9
:1028C00049000100480000004800010047000100E5
:1028D00046000000460001004500000045000100E0
:1028E00044000100430000004300010042000000DA
:1028F00042000100410000004100010040000100D1
:102900003F0000003F0001003E0000003E000100CB
:102910003D0000003D0001003C0000003C000000C4
:102920003C0001003B0000003B0001003A000000B9
:102930003A000100390000003900010038000000B1
:1029400038000000380001003700000037000100A7
:10295000360000003600000036000100350000009F
:102960003500000035000100340000003400000094
:102970003400010033000000330000003300010088
:10298000320000003200000032000100310000007F
:102990003100000031000100300000003000000074
:1029A000300001002F0000002F0000002F00000069
:1029B0002F0001002E0000002E0000002E0001005C
:1029C0002D0000002D0000002D0000002D00010052
:1029D0002C0000002C0000002C0000002C00010046
:1029E0002B0000002B0000002B0000002B0001003A
:1029F0002A0000002A0000002A0000002A0001002E
:102A00002900000029000000290000002900000022
:102A10002900010028000000280000002800000014
:102A20002800000028000100270000002700000007
:102A300027000000270000002700010026000000FA
:102A400026000000260000002600000026000100ED
:102A500025000000250000002500000025000000E2
:102A600025000000250001002400000024000000D3
:102A700024000000240000002400010023000000C6
:102A800023000000230000002300000023000000BA
:102A900023000000230001002200000022000000AB
:102AA000220000002200000022000000220001009D
:102AB0002100000021000000210000002100000092
:102AC0002100000021000000210001002000000082
:102AD0002000000020000000200000002000000076
:102AE0002000000020000000200001001F00000066
:102AF0001F0000001F0000001F0000001F0000005A
:102B00001F0000001F0001001E0000001E0000004A
:102B10001E0000001E000000043700001E290000F7
:102B2000511B00005810000010090000CC040000E8
:102B30007802000041010000000045320042656457
:102B400000453100626564002C2073797374656DF3
:102B50002073746F707065642120486561746572BC
:102B60005F49443A200048656174696E6720666178
:102B7000696C656400546865726D616C2052756E95
:102B8000617761790048656174696E6720466169A3
:102B90006C65640048656174696E67206661696C84
:102BA000656400546865726D616C2052756E617762
:102BB00061790059206C696E653A3120746F20325A
:102BC000300059206C696E653A2D3120746F202DCC
:102BD000323000592043616C6962726174696F6EB2
:102BE00000582043616C6962726174696F6E0047BE
:102BF00032380053746F72652053657474696E6760
:102C00007300326E64204E6F7A7A6C65205A0032FF
:102C10006E64204E6F7A7A6C65205900326E6420A3
:102C20004E6F7A7A6C652058004D3630352053301F
:102C30000A47323820580046756C6C20436F6E741A
:102C4000726F6C004D3630352053310A54300A4DC6
:102C500036303520533220583230300A473238204F
:102C6000580A47312058350A4D3630352053332025
:102C700058323030004D3630352053310A54300A46
:102C80004732380A4D3630352053322058323030F2
:102C90000A47323820580A47312058350A4D363015
:102CA000352053332058323030004D6972726F72C4
:102CB000656420436F7079004D3630352053310AFA
:102CC00054300A4D36303520533220583130300AD6
:102CD00047323820580A473120583530004D3630B9
:102CE000352053310A54300A4732380A4D363035D0
:102CF00020533220583130300A47323820580A47A2
:102D00003120583530004475706C69636174696FA7
:102D10006E004D3630352053310A47323820580A7C
:102D20004731205835004175746F2D5061726B002A
:102D30004944452D58205365740049444558204D59
:102D40006F646500546F6F6C204F666673657473B3
:102D5000004175746F2043616C6962726174696FC0
:102D60006E00436F6E66696775726174696F6E009D
:102D7000473238004D3630352053310A54300A4737
:102D80003238003F004E65787420436F726E657272
:102D9000004D3630352053310A54300A473238005E
:102DA0004D3630352053300A54300A4732380A4DF8
:102DB000363035205331003F00546F6F6C2043682C
:102DC000616E6765004E657874004D36303520536E
:102DD000310A54300A47323800473238205A004D01
:102DE0003630352053310A54300A473238003F001C
:102DF0005265736574205A204C696D69742053774D
:102E00006974636800446F6E650052657365740091
:102E10004D3630352053310A54300A4732380020BD
:102E2000746F6F206C6F6E6720657874727573694C
:102E30006F6E2070726576656E7465640A0020633B
:102E40006F6C6420657874727573696F6E20707230
:102E50006576656E7465640A0070012C0190012727
:102E600001B0012201C0011D01F00118011002137F
:102E70000130020E016002090190020401C002FF4C
:102E8000000003FA004003F5008003F000D003EBDC
:102E9000002004E6007004E100E004DC004005D7F7
:102EA00000C005D2004006CD00D006C8008007C390
:102EB000003008BE00F008B900C009B400B00AAF85
:102EC00000B00BAA00D00CA500000EA000500F9B74
:102ED00000C01096005012910000148C00C015879D
:102EE00000B0178200B0197D00D01B7800001E735F
:102EF0000040206E0090226900F024640040275FAB
:102F00000090295A00E02B5500102E500020304B25
:102F10000010324600E033410090353C0010373756
:102F20000070383200A0392D00B03A2800A03B23B1
:102F300000603C1E00103D1900903D1400103E0F33
:102F400000703E0A00C03E0500003F0000403FFB0D
:102F5000FF803FF6FFC03FF1FF544845524D414CC2
:102F60002052554E4157415900546865726D616C4D
:102F70002052756E61776179004572723A204D4139
:102F80005854454D50004D415854454D5020747291
:102F900069676765726564004572723A204D494EF3
:102FA00054454D50004D494E54454D502074726962
:102FB000676765726564004D383420582059205A7F
:102FC000204500202F002040002042403A002040B1
:102FD0003A0020573A00496E76616C696420657842
:102FE0007472756465720A00000054C200005C438C
:102FF000000000004163746976652045787472753D
:103000006465723A200020746F6F206C6F6E6720C9
:10301000657874727573696F6E2070726576656E0F
:103020007465640A0020636F6C642065787472753F
:1030300073696F6E2070726576656E7465640A00E0
:10304000486F6D696E67204661696C6564000000B9
:103050000C4200000C420000A0405761726E696E85
:10306000673A20486F6D696E672042756D70204425
:10307000697669736F72203C20310A0002020400F5
:1030800000A0400000A0400000004000008143007C
:10309000005C4300006B43FF01FF496E736572746F
:1030A0002066696C616D656E7420616E642070725B
:1030B00065737320627574746F6E0A00220A00557E
:1030C0006E6B6E6F776E20636F6D6D616E643A200C
:1030D00022002E0A006F70656E206661696C65645F
:1030E0002C2046696C653A20004D3234004D323355
:1030F0002025730046696C652073656C6563746593
:10310000640A002053697A653A200046696C65209C
:103110006F70656E65643A2000454E4420535542F9
:10312000524F5554494E450A002220706F730022B9
:1031300020706172656E743A2200535542524F55A9
:1031400054494E452043414C4C207461726765746C
:103150003A2200747279696E6720746F2063616C23
:103160006C207375622D67636F64652066696C659A
:1031700073207769746820746F6F206D616E792099
:103180006C6576656C732E204D4158206C657665B4
:103190006C2069733A310A002E0A006F70656E2048
:1031A0006661696C65642C2046696C653A2000573D
:1031B000726974696E6720746F2066696C653A2065
:1031C00000667265736800646F696E6700206669E7
:1031D0006C653A20004E6F7720004D323139205413
:1031E0003120592B302E3035004D323139205431B9
:1031F00020592B302E3130004D32313920543120BE
:10320000592B302E3135004D32313920543120596F
:103210002B302E3230004D32313920543120592B91
:10322000302E3235004D32313920543120592B3077
:103230002E3330004D32313920543120592B302E6D
:103240003335004D32313920543120592B302E3452
:1032500030004D32313920543120592B302E343545
:10326000004D32313920543120592B302E35300069
:103270004D32313920543120592B302E3535004D07
:1032800032313920543120592B302E3630004D3216
:10329000313920543120592B302E3635004D323102
:1032A0003920543120592B302E3730004D323139EE
:1032B00020543120592B302E3735004D32313920F2
:1032C000543120592B302E3830004D3231392054B2
:1032D0003120592B302E3835004D323139205431C0
:1032E00020592B302E3930004D32313920543120C5
:1032F000592B302E3935004D323139205431205977
:103300002B312E30300059206C696E653A2D3137E3
:103310000059206C696E653A2D31360059206C6970
:103320006E653A2D31350059206C696E653A2D3144
:10333000340059206C696E653A2D31330059206C88
:10334000696E653A2D31320059206C696E653A2DEF
:1033500031310059206C696E653A2D3130005920A9
:103360006C696E653A2D390059206C696E653A2D8D
:10337000380059206C696E653A2D370059206C6908
:103380006E653A2D31380059206C696E653A2D36DC
:103390000059206C696E653A2D350059206C696EB4
:1033A000653A2D340059206C696E653A2D3139002B
:1033B00059206C696E653A2D330059206C696E6531
:1033C0003A2D320059206C696E653A2D3230005921
:1033D000206C696E653A2D31004D323139205431FF
:1033E00020582D302E3035004D32313920543120C7
:1033F000582D302E3130004D323139205431205883
:103400002D302E3135004D32313920543120582D98
:10341000302E3230004D32313920543120582D3089
:103420002E3235004D32313920543120582D302E76
:103430003330004D32313920543120582D302E3365
:1034400035004D32313920543120582D302E343052
:10345000004D32313920543120582D302E34350072
:103460004D32313920543120582D302E3530004D19
:1034700032313920543120582D302E3535004D321F
:10348000313920543120582D302E3630004D323114
:103490003920543120582D302E3635004D323139F7
:1034A00020543120582D302E3730004D3231392004
:1034B000543120582D302E3735004D3231392054BB
:1034C0003120582D302E3830004D323139205431D2
:1034D00020582D302E3835004D32313920543120CE
:1034E000582D302E3930004D32313920543120588A
:1034F0002D302E3935004D32313920543120582DA0
:10350000312E30300058206C696E653A31360058E3
:10351000206C696E653A31350058206C696E653AE9
:1035200031390058206C696E653A31340058206C8E
:10353000696E653A31330058206C696E653A3230F5
:103540000058206C696E653A31320058206C696E03
:10355000653A31310058206C696E653A3137005850
:10356000206C696E653A31300058206C696E653A9E
:10357000390058206C696E653A380058206C696EC5
:10358000653A370058206C696E653A360058206CF1
:10359000696E653A350058206C696E653A3400589A
:1035A000206C696E653A330058206C696E653A325A
:1035B0000058206C696E653A31380058206C696E8D
:1035C000653A31005072656865617420504C412045
:1035D000416C6C005072656865617420504C4120EC
:1035E000456E64207E005072656865617420504CA1
:1035F0004120426564005072656865617420504CDA
:1036000041207E00507265686561742041425320FC
:10361000416C6C00507265686561742041425320B2
:1036200042656400507265686561742041425320B0
:10363000456E64207E005072656865617420414269
:1036400053207E0054656D706572617475726500FB
:10365000436F6F6C646F776E00507265686561745C
:1036600020414253005072656865617420504C419E
:103670000046616E20537065656400426564004ECB
:103680006F7A7A6C65207E004D61696E00507269B8
:103690006E7420506175736564004D6564696120C6
:1036A00052656D6F766564004D6564696120496E91
:1036B00073657274656400436C696D62657220376E
:1036C0002052656164792E005072696E74696E676C
:1036D0002E2E2E005072696E742041626F727465D6
:1036E00064004D323520500A4D32340050617573FC
:1036F00065205072696E74000000210024002700CC
:103700002A002D00300033000101000004010701F0
:103710000A0100002200250028002B002E003100A5
:10372000340002010000050108010B010000200027
:103730002300260029002C002F0032000001000089
:103740000301060109010505050507050808080824
:10375000020202020A0A0808040404040101010129
:103760000101010103030303030303030407070724
:103770000C0C0C0C0C0C0C0C0202020206060606C9
:10378000060606060B0B0B0B0B0B0B0B0102102096
:103790002008081020401020408002010201080487
:1037A000020101020408102040808040201008041B
:1037B0000201800402018040201008040201080474
:1037C00002010102040810204080010204081020B8
:1037D000408000000A0B02090C0D0E0807030401CB
:1037E00000000000000000000000000000000000D9
:1037F00000000000000000000000000000001211A6
:1038000010000000000000000000000000000000A8
:1038100000000000000000005072696E74206672A3
:103820006F6D204D6564696100486F6D652025737B
:1038300025732573204669727374007C3C3E5E2BB1
:103840003D3F2F5B5D3B2C2A225C00486172646324
:103850006F6465642044656661756C74205365749B
:1038600074696E6773204C6F616465640A000000C0
:103870004843000048430000A040000016430000F9
:10388000A0420000A0420000C8430000BE42D00792
:103890000000D00700006400000010270000202076
:1038A0004D363033200020204D3431322053004635
:1038B000696C616D656E742072756E6F75742073BE
:1038C000656E736F723A0A00546F6F6C2D63686196
:1038D0006E67696E673A0A002055005431204C002B
:1038E0002055005430204C0046696C616D656E7443
:1038F000206C6F61642F756E6C6F6164206C656EF7
:10390000677468733A0A0020204D32353020430036
:103910004C434420436F6E74726173743A0A002002
:10392000440020490020500020204D3330312045F4
:10393000005049442073657474696E67733A0A00D5
:1039400020460020420020480020204D3134352000
:1039500053004D6174657269616C206865617475AE
:103960007020706172616D65746572733A0A00202F
:10397000204D323138205400486F74656E64206FDA
:103980006666736574733A0A0020204D3230362023
:103990005800486F6D65206F66667365743A0A005B
:1039A00020580020540020530020204D3230352074
:1039B000420020453C6D61785F655F6A65726B3ED1
:1039C0000020583C6D61785F785F6A65726B3E20BD
:1039D000593C6D61785F795F6A65726B3E205A3C35
:1039E0006D61785F7A5F6A65726B3E0041647661F3
:1039F0006E6365643A20423C6D696E5F7365676D06
:103A0000656E745F74696D655F75733E20533C6DC0
:103A1000696E5F66656564726174653E20543C6DD5
:103A2000696E5F74726176656C5F6665656472610C
:103A300074653E0020540020520020204D32303466
:103A4000205000416363656C65726174696F6E201C
:103A500028756E6974732F7332293A20503C707246
:103A6000696E745F616363656C3E20523C7265747D
:103A7000726163745F616363656C3E20543C747271
:103A80006176656C5F616363656C3E0A0020204D62
:103A90003230312058004D6178696D756D20416379
:103AA00063656C65726174696F6E2028756E6974E8
:103AB000732F7332293A0A00204500205A002059FA
:103AC0000020204D3230332058004D6178696D75EB
:103AD0006D206665656472617465732028756E6912
:103AE00074732F73293A0A005374657073207065DC
:103AF0007220756E69743A0A0020204D32303020F1
:103B000044300A0020204D3230302054312044000F
:103B100020204D3230302044002044697361626CB3
:103B200065640A0046696C616D656E742073657426
:103B300074696E67733A0020204D31343920432078
:103B40003B20556E69747320696E2043656C736900
:103B500075730A0020286D6D29002020473231201E
:103B60002020203B20556E69747320696E206D6D96
:103B7000006F70656E0054524947474552454400F6
:103B80003A200066696C616D656E74007A5F6D69DC
:103B90006E00795F6D617800785F6D617800785FA5
:103BA0006D696E005265706F7274696E6720656E24
:103BB0006473746F70207374617475730A00205A93
:103BC0003A0020593A0020436F756E7420583A002D
:103BD00020453A00205A3A0020593A00583A0050FD
:103BE0006C65617365205265736574005052494E6F
:103BF0005445522048414C5445440025533A202511
:103C000053004B494C4C45442E20005072696E7451
:103C100065722068616C7465642E206B696C6C2819
:103C2000292063616C6C6564210A006563686F3AE2
:103C3000004572726F723A00486F74656E6420744A
:103C40006F6F20636F6C640A004D3630303A205439
:103C50006F6F20436F6C6400486F74656E642074EE
:103C60006F6F20636F6C640A00507265737320621B
:103C70007574746F6E20746F20726573756D650A4C
:103C800000496E736572742066696C616D656E744F
:103C900020616E6420707265737320627574746F36
:103CA0006E0A00507265737320627574746F6E20B3
:103CB000746F2068656174206E6F7A7A6C650A0093
:103CC00043616E6E6F74206F70656E2073756264F1
:103CD0006972200053442063617264206F6B0A0094
:103CE0006F70656E526F6F74206661696C65640AEF
:103CF00000766F6C756D652E696E697420666169FA
:103D00006C65640A00534420696E697420666169B9
:103D10006C0A0000EB00ED0011241FBECFEFD1E2D2
:103D2000DEBFCDBF00E00CBF13E0A0E0B2E0E4E6F0
:103D3000F8E602E00BBF02C007900D92AA36B10769
:103D4000D9F724E1AAE6B3E001C01D92A738B20773
:103D5000E1F71EE1CBE8DEE100E006C021970109B2
:103D6000802FFE010F949033CA38D10780E00807F6
:103D7000A9F70F94171C0D9421340C9400002F9276
:103D80003F924F925F926F927F928F929F92AF92EB
:103D9000BF92CF92DF92EF92FF920F931F93CF9338
:103DA000DF93CDB7DEB7C555D1090FB6F894DEBFA6
:103DB0000FBECDBF66968FAF669720911D092596E1
:103DC0002FAF259781E080931D09809180068D3467
:103DD00009F4D1C1843511F40C94902E873411F07C
:103DE0000C94A12E20907E0630907F0635E123169C
:103DF000310411F40C94A32E94F454E025163104EC
:103E000044F482E0281631040CF043C037FE35C07C
:103E1000AEC194E02916310409F4C7C0A8C1AAE5CF
:103E20002A16310409F42EC15CF4EBE12E1631049C
:103E300009F4FAC0FCE12F16310409F40FC197C14F
:103E40002BE52216310409F421C13CE52316310487
:103E500009F08DC19AE9292E92E0392E24EBE22E49
:103E600028E0F22EA2E7B2E0BDA3ACA338EAC32E4D
:103E700038E0D32E00E010E04AC18091410288234F
:103E800011F40C94A32E0E94949C0E9469D90C9466
:103E9000A32E80914102882311F40C94A32E0E943A
:103EA000949C82E50F940610882309F44CC00F946B
:103EB000860F6B017C0120E030E0A9010F94012AFC
:103EC000882311F40C946B2F8091720290917302ED
:103ED000A0917402B09175028CA39DA3AEA3BFA361
:103EE00020917602309177024091780250917902C8
:103EF00028A739A74AA75BA78090860890908708D3
:103F0000A0908808B090890840908A0850908B084B
:103F100060908C0870908D08A5019401BC01CD01C2
:103F20000F94012A81110C94B02EA301920168A56F
:103F300079A58AA59BA50F94012A882311F40C94D6
:103F40006B2F0C94B02E89E40F940610882329F06F
:103F50000F94860F6B017C0103C0C12CD12C76011C
:103F60008AE40F940610882311F40C94722F0F9496
:103F7000860F6CA77DA78EA79FA720E030E0A90140
:103F8000C701B6010F94012A81110C947F2F20E004
:103F900030E0A9016CA57DA58EA59FA50F94012AEF
:103FA00081110C947F2F0C946B2F80E50F940610D9
:103FB000882329F00E946CA46B017C0103C0C12CF2
:103FC000D12C760183E50F940610882361F00F94BD
:103FD000860F20E030E04AE754E40F94662A0F94FD
:103FE000C2316B017C010E94B1D180910D0F811112
:103FF00005C060E08BE693E00E9455F80F947602CE
:10400000C60ED71EE81EF91E0F947602DC01CB0106
:104010008C199D09AE09BF09B7FD02C00C94A32EEF
:1040200080E00E949142F0CF0E94C5FD81110C9466
:10403000A32E8CE0EEE8F2E0DE01119601900D92E5
:104040008A95E1F760E070E080E50E94A69FBE01DE
:104050006F5F7F4F0E942CF70C94A32EE0901B09FA
:10406000D0905E028091D1088770873011F00C9457
:10407000163360E08FE40E94F3A481110C94A32E08
:104080000C941633109275030C94A32E8FE080933A
:1040900075030C94A32E0F94860F2B013C01133053
:1040A00049F0D6012D913D914D915C910F9478305E
:1040B0002B013C01ECA1FDA1208131814281538182
:1040C000C301B2010F9478304B015C012DEB37E353
:1040D00046E855EB0F949F3287FD21C02DEB37E367
:1040E00046E855E3C501B4010F94012A1816BCF047
:1040F0001F5FF4E0EF0EF11C2CA13DA12C5F3F4FA0
:104100003DA32CA334E0C30ED11C143031F1F101D6
:1041100081911F010F940610882351F3BCCF1330F7
:1041200051F440927E0250927F026092800270921F
:10413000810201E0DDCFA5019401D7016D917D9150
:104140008D919C910F947930F70160837183828304
:104150009383812F0E94E7D5CBCF002321F08EE7F8
:1041600092E00E9402C60F94E00B0C94A32E0E94D2
:10417000FEE00C94A32E00917E0610917F06073777
:10418000110511F40C9410290CF0EBC00D3411053D
:1041900009F4DAC40CF062C00931110509F4E5C272
:1041A00034F50431110509F46FC28CF401311105A5
:1041B00009F456C234F40230110508F4D5C10C9448
:1041C0008D2E0231110509F493C60C948D2E063103
:1041D000110509F47EC20CF478C20731110509F407
:1041E00081C20831110509F492C20C948D2E0E3152
:1041F000110509F42EC3B4F40B31110509F4CEC234
:104200000CF4BEC20C31110509F41BC30D311105AC
:1042100011F00C948D2E8091470D8E7F8093470D69
:104220000C94A32E0A32110509F462C454F40F3120
:10423000110509F4B2C30032110509F46BC30C94E3
:104240008D2E0B34110509F47BC40C34110511F0CB
:104250000C948D2E0E94AC8B0C94A32E0B36110562
:1042600009F45FC50CF043C00535110509F46CC6AF
:104270004CF50235110509F42DC6D4F401351105AC
:1042800011F00C948D2E0E9449CE0E94C18B0E9489
:10429000B8D30E94BA4068EE73E080E090E00F94DB
:1042A000BB1060E088EA94E00E9455F80C94A32EBD
:1042B0000335110509F415C60435110509F418C6AE
:1042C0000C948D2E0836110509F442C434F40C35D3
:1042D000110509F45CC60C948D2E0936110509F4FC
:1042E000E7C40A36110509F4F9C40C948D2E003781
:1042F000110509F47DC584F40D36110509F464C473
:104300000CF471C50E36110509F416C50F361105EA
:1043100009F424C50C948D2E0337110509F4D5C674
:104320007CF40137110509F46EC50237110511F04F
:104330000C948D2E0E94B1D10F94E00B0C94A32EFF
:104340000537110509F42AC70637110511F00C9439
:104350008D2E00917C0610917D0694E0F12C40E0BA
:1043600043C70A3F110511F40C94392C0CF06DC0B1
:104370000B3C110511F40C94092A5CF50139110567
:1043800009F460C784F40937110509F454C70CF423
:104390004AC70D37110509F49AC50C38110509F4FF
:1043A00054C50C948D2E0E3B110509F467C534F4E9
:1043B0000B39110509F465C50C948D2E083C1105C7
:1043C00009F49BC7093C110511F40C94E6290C94DF
:1043D0008D2E093D110511F40C94812AB4F40D3C85
:1043E000110511F40C945C2A14F40C94282A0E3C48
:1043F000110511F40C945F2A033D110511F00C9482
:104400008D2E0E947BA00C94A32E0C3D110511F45F
:104410000C94D92A74F40A3D110511F40C94962ACF
:104420000B3D110511F00C948D2E0E945EA30C948F
:10443000A32E0D3D110511F40C94E62A023E110540
:1044400011F40C943C2B0C948D2E063F41E0140784
:1044500011F40C94032D0CF046C0003981E01807CC
:1044600011F40C94922CECF40D32A1E01A0711F423
:104470000C949D2B3CF40C32114011F40C94882BBD
:104480000C948D2E0E32F1E01F0711F40C944E2C7B
:104490000F32114011F00C948D2E0E94EB920C946F
:1044A000A32E0C3A31E0130711F40C949D2C64F404
:1044B0000A3951E0150709F4A3C40C39114011F46D
:1044C0000C94952C0C948D2E043F91E0190711F457
:1044D0000C94002D053F114011F00C948D2E0F947B
:1044E000D30B0C94A32E0B35B2E01B0711F40C94E4
:1044F000282DC4F4083FF1E01F0711F40C940F2D90
:1045000014F40C94062D0C3032E0130711F40C94C3
:10451000202D0835124011F00C948D2E0E94C3A15D
:104520000C94A32E0E3B52E0150711F40C94A62D0B
:104530007CF40D3592E0190711F40C94A32D0D3B7A
:10454000124011F00C948D2E0E94769D0C94A32E97
:10455000003AB3E01B0709F412C2073E134011F4FE
:104560000C947F2E0C948D2EA0907C06B0907D062E
:1045700080E50F940610882359F00E946CA46B010B
:104580007C0111E0672B682B692B31F410E004C02B
:1045900010E0C12CD12C760183E50F9406108823FE
:1045A00011F40C949D340F94860F20E030E04AE71C
:1045B00054E40F94662A0F94C2316B017C011111EF
:1045C0000BC0672B682B692B39F4A114B10421F0BF
:1045D000D5018C91811102C010E001C011E00E9450
:1045E000B1D1112329F061E0C5010E94CFF805C0C7
:1045F00060E084E793E00E9455F810911D0983E084
:1046000080931D0981E080931C09C114D104E10449
:10461000F104B1F00F947602C60ED71EE81EF91E03
:104620000F947602DC01CB018C199D09AE09BF09FC
:10463000B7FF0EC080911C0981110C94A23408C0F0
:1046400080911C09882321F080E00E949142F8CFDC
:104650000E94F2F810921C0910931D090C94A32ECD
:104660008091780684FF02C00C94A73480917A066A
:1046700087FF02C00C94A73480917B06837011F0F1
:104680000C94A7340C94CA348FE993E00F94DF1094
:104690008AE89BE00F9432048BE1EAE8FBE0DE015C
:1046A000119601900D928A95E1F760E070E0CE01DD
:1046B00001960F94DB19CE0101960F94370480E91F
:1046C00093E00F94DF100C94A32E0F9455150C94C7
:1046D000A32E0E9426E68091470D877F8093470D89
:1046E0000C94A32EE0917C06F0917D0680818823B6
:1046F00029F0803209F410823196F8CF60E0809181
:104700007C0690917D060E9482E60C94A32E8091F7
:104710008F0E8823F1F080E090E0A0EAB1E488A356
:1047200099A3AAA3BBA31C8E1D8E1E8E1F8E198259
:104730001A821B821C820FEF20E0AE01405E5F4FA9
:10474000BE01645E7F4FCE0101960F947E110C94E2
:10475000A32E0E94BD40882321F00E949BE70E9467
:104760008A8B0E94F2F80C94A32E8091470D82FF51
:1047700003C08B7F8093470D0E94D29E0C94A32E82
:104780008091470D83FD02C00C94A32E83E50F9406
:10479000061081110C94DE340C94A32E83E40F9444
:1047A000BD0F882319F18AEB93E00F94DF108091FD
:1047B000340B882391F0BE016F5F7F4F81E39BE054
:1047C0000F94FA028E010F5F1F4FF80181918F0144
:1047D000882339F00E947141F8CF80EB93E00F9469
:1047E000DF108AE00E9471410C94A32E8091470D46
:1047F00082FF21C089EC93E00F94DF106091430D9C
:104800007091440D8091450D9091460D4AE00E94B3
:1048100078418FE20E94714160913F0D7091400D8F
:104820008091410D9091420D4AE00E9478410E9492
:104830006E420C94A32E8BED93E00F94DF100C943A
:10484000A32E80917C0690917D060E9437E60C9401
:10485000A32E8091470D83FD02C00C94A32E0E94CD
:10486000E7E08091470D83FD02C00C94A32E409198
:104870007C0650917D06BE01645E7F4F80E00E9401
:104880003ADE8C01009711F40C94A32E6C8D7D8D73
:1048900019821C8222E0AC01CE0101960F945508CA
:1048A000811102C0F12C14C0CE0101960E94A8DD36
:1048B0008823C1F361E0CE0101960F94DE020097D8
:1048C00089F325EEDC012C931C820F94A516F82E9B
:1048D000CE0101960F943704B801FF2089F087E0DC
:1048E00094E00F9426118AE00E9471411092430DCA
:1048F0001092440D1092450D1092460D0C94A32E6B
:104900008FEE93E00F9426118CEE93E00F94DF105E
:104910000C94A32E8091470D82FD0E94B1D180910D
:10492000470D83FD02C00C94A32E60E080E50E9439
:10493000F3A4182F682F80917C0690917D060E9429
:1049400082E683E50F940610882381F00F94560FBA
:10495000AB01BC014093430D5093440D6093450D52
:104960007093460D81E39BE00F94C6180E949BE76D
:1049700011110C94A32E0E948A8B0C94A32E2091CB
:104980007C0630917D069091470D92609093470D83
:10499000C9010E9437E60C94A32E0E943B8B7B0139
:1049A0008C0120E831E541E050E00F943D30C90131
:1049B0006DE671E00F944D334B015C01C801B70106
:1049C00020E13EE040E050E00F943D30CA01B901E3
:1049D00028E130E040E050E00F943D30762E672E25
:1049E000C62ED72E8CE3282E312C412C512CC801F9
:1049F000B701A20191010F943D30F62EE72ECA01B6
:104A0000B901A20191010F943D30CB018E010F5FDE
:104A10001F4F8114910499F0EF92FF927F936F934F
:104A20006F927F92BF92AF929F928F928DE394E0AC
:104A30009F938F931F930F930F949B2913C0A114DF
:104A4000B104B1F0EF92FF927F936F936F927F92D8
:104A5000BF92AF928DE294E09F938F931F930F9339
:104A60000F949B290FB6F894DEBF0FBECDBF30C0A8
:104A7000CD2879F0EF92FF927F936F936F927F92A0
:104A800081E294E09F938F931F930F930F949B2940
:104A9000E9CF892B69F0EF92FF927F936F9389E1C1
:104AA00094E09F938F931F930F930F949B29DACFDA
:104AB000EF92FF9285E194E09F938F931F930F9362
:104AC0000F949B290F900F900F900F900F900F90C5
:104AD00060E0C8010E94CFF80F943B11B80181E556
:104AE00094E00F9426118AE00E9471410C94A32E49
:104AF00083E50F940610882311F40C94A32E0F94D1
:104B0000660FF82E6DE070E080E50E94B5A18C0183
:104B100097FF02C00C94A32E893021F4F092DA079B
:104B20000C94A32E60E089E40E94F3A481110C94FC
:104B3000EF34802F0F94E01B8111BBC50C94EF3430
:104B40000E948A8B0C94A32E0E94C18B0C94A32EDE
:104B50008091EC0783FF02C00C94A32E0E944C9D11
:104B6000B82E87FF02C00C94A32E83E50F94061085
:104B7000882331F10F94860F0F94BD316B017C01B6
:104B80008B016B2DC6010E94D19980915E0282300B
:104B900084F0B1100EC0C114D10411F40C94FD3492
:104BA00080916A0390916B038C0D9D1D61E00E94C2
:104BB000D1990C34110524F40E94C18B0E94F2F8A3
:104BC0000F9495220C94A32E8091EC0783FF02C0D2
:104BD0000C94A32E0E944C9DB82E87FF02C00C940B
:104BE000A32E83E50F940610A82E811107C082E53D
:104BF0000F940610182F882309F44EC00F94860FC7
:104C00000F94BD316B017C018B016B2DC6010E949D
:104C1000D19980915E02823024F0BB2011F40C9473
:104C200005350F94860F20E030E046E952E40F94FA
:104C3000012A181614F40C9401350E94C18B0E94AD
:104C4000F2F80B2D0B2C000C110BAB2DB7E1AB02C6
:104C5000C0011124FC01E55DF74F7F01608571857E
:104C6000072E000C880B990B0F94072A2B013C018F
:104C7000D7011496CD90DD90ED90FC901797A70189
:104C800096010F949F32181614F40C943335AA2011
:104C900011F40C94153511E00F949522112311F4A1
:104CA0000C94A32E6A2D8B2D0E94C7CA0C94A32EA0
:104CB0000E944C9D182F87FD0AC08BE794E00F944B
:104CC000DF10812F0E94FCC98AE00E947141259665
:104CD000FFAD2597F0931D090C94733660E080E5D5
:104CE0000E94A5A181110C94A32E81E40F94BD0F05
:104CF000882341F0E0911E09F0E0E652F84F608110
:104D000070E002C06FEF70E083E50E94A69F8F3FC6
:104D1000910519F010F08FEF90E08093DA070C9472
:104D2000A32E60E080E50E94A5A181110C94A32E22
:104D30001092DA070C94A32E8EE40F9406108823A9
:104D400011F40C94A32E0F94560F609305077093E3
:104D500006078093070790930807F5C783E50F942C
:104D6000BD0F882331F060E083E50E94A5A1809308
:104D7000EC070F943B118CE894E00F94DF108091C6
:104D8000EC07882369F102E8E02E04E0F02E00E051
:104D900010E020E08091EC0790E0A0E0B0E0002E71
:104DA00004C0B695A795979587950A94D2F780FF8A
:104DB0000EC0DD24D394D20E222319F08CE20E947F
:104DC0007141F701859194910F94DF102D2D0F5FA4
:104DD0001F4F32E0E30EF11C05301105D9F601CD6D
:104DE0008EE794E0FCCC10921C0910921E02ABC717
:104DF00041E060E070E083E994E00F94C914A3C738
:104E00000E943340A0C783E50F940610882371F0F9
:104E10000F94660F282F30E02D3331051CF480935A
:104E2000000291C78CE3809300028DC70F943B1161
:104E30004091000250E060E070E081EA94E00F945D
:104E4000EE108AE00E9471417EC78091EC0783FDDD
:104E50007AC783E50F940610882309F474C70F946A
:104E6000860F0F94BD316C3871050CF48B011093D3
:104E70002508009324080E945CC665C70E94F3972A
:104E800062C783E50F940610882309F45CC70F946A
:104E9000660F182F90E0CD970CF01CE31093700371
:104EA0000F9476026B017C01212F30E0A8EEB3E075
:104EB0000F946930C60ED71EE81EF91EC0926C030F
:104EC000D0926D03E0926E03F0926F033CC70E9494
:104ED000D29E39C7809175038F7D80618093750361
:104EE00032C7809175038F7E8062809375032BC7D4
:104EF00083E50F940610882399F00F94860F20E025
:104F000030E04AE754E40F94662A0F94C23160936C
:104F1000010270930202809303029093040213C76C
:104F20008091780684FF02C00C94363580917A0611
:104F300087FF02C00C94363580917B06837011F098
:104F40000C9436350C946D3583E50F94BD0F882392
:104F500009F4F9C60F947602609327087093280825
:104F60008093290890932A080F94860F20E030E060
:104F70004AE754E40F94662A0F94C2316093710398
:104F8000709372038093730390937403DCC60E9442
:104F90004C9D87FDD8C69091780694FD04C09091F1
:104FA0007A0697FF0AC0BAE9CB2EB2E0DB2E13EDEA
:104FB000E12E18E0F12E10E009C090917B0693706D
:104FC00091F7682F81E00E946AA1BDC6D6018D913C
:104FD0006D010F940610882309F46DC0133009F099
:104FE00063C00F94860F4B015C0120E030E040EA83
:104FF00051E40F94012A87FF4EC0A50194016091EE
:10500000F3087091F4088091F5089091F6080F94D8
:1050100055312B013C019B01AC016091C607709199
:10502000C7078091C8079091C9070F94662A6093BB
:10503000C6077093C7078093C8079093C907A30159
:105040009201609103097091040980910509909182
:1050500006090F94662A60930309709304098093EC
:105060000509909306096091D6077091D707809142
:10507000D8079091D9070F94052AA30192010F94A4
:10508000662A0F94C2316093D6077093D707809336
:10509000D8079093D9078092F3089092F408A092D1
:1050A000F508B092F60807C00F94860FF701648BDD
:1050B000758B868B978B1F5FF4E0EF0EF11C14301D
:1050C00009F084CF0E94DDC53EC68BED95E00F94BC
:1050D000DF1060E08BEC95E00E94479C60E086EB7F
:1050E00095E00E94479C61E08FEA95E00E94479C12
:1050F00061E084EA95E00E94479C61E084E995E0E4
:105100000E94479C60E08BE895E00E94479C61E02C
:1051100081E895E00E94479C60E087E795E00E9467
:10512000479C60E08FE695E00E94479C60E081E646
:1051300095E00E94479C60E083E595E00E94479CD3
:1051400060E084E495E00E94479C60E086E395E09F
:105150000E94479C60E080E295E00E94479C60E0EE
:105160008FE095E00E94479C60E080E095E00E941F
:10517000479C60E08BEE94E00E94479C61E088EDE4
:1051800094E00E94479C60E08BEC94E00E94479C76
:1051900060E087EB94E00E94479CD5C580917C0637
:1051A00090917D06009709F4DCCADC012C91222342
:1051B00009F4D7CA60E00E94CFF8C5C5F801808124
:1051C000282F2B7F213499F08035E9F48181805399
:1051D0008A30C8F498012E5F3F4F89012F5F3F4FFF
:1051E000F80180818032C9F3915041F70CC02181D0
:1051F000213349F4813421F0853461F741E0EACF6D
:10520000FF24F394E7CF41110F943B11FF2021F0CD
:1052100087E896E00F94DF10C8010E94724293C5A0
:105220000F94CD0990C581E08093C8048093C70492
:105230000F94190A88C51092C8041092C7040F94DD
:10524000190A81C560E070E083E50E94B5A18C0178
:105250001127023011053CF00F9438118BE896E0CD
:105260000F94DF1070C588E40F9406108823A9F00E
:105270000E94B1A1863991053CF08530F1E09F078D
:105280002CF084E091E002C086E990E0F801EE0F96
:10529000FF1FEF55F04F9183808386E40F94061033
:1052A000882381F00E94B1A197FD07C08F3F91052F
:1052B00029F024F08FEF90E001C080E0F801E5567E
:1052C000F04F808382E40F940610882309F43BC5D5
:1052D0000E94B1A18530910534F08D3891052CF0F4
:1052E0008CE890E002C085E090E0F801EE0FFF1F2F
:1052F000E356F04F9183808326C50E944C9D182F62
:1053000087FD21C584E40F94BD0F882309F45BC099
:105310000F94860F6B017C0101E020E030E0A901D1
:105320000F94012A811101C000E00093C00820E021
:1053300030E0A901C701B6010F94012A882309F4BE
:1053400042C00F94860F24E01202F0011124E753AB
:10535000F74F608371838283938320E030E0A9015B
:105360006091C9087091CA088091CB089091CC08CF
:105370000F94012A81110CC080E090E0A0EEBFE301
:105380008093C9089093CA08A093CB08B093CC0827
:1053900020E030E0A9016091CD087091CE088091A5
:1053A000CF089091D0080F94012A81110CC080E0A1
:1053B00090E0A0EEBFE38093CD089093CE08A09339
:1053C000CF08B093D0080E9493D0BDC40E944C9DDA
:1053D00087FDB9C46AE9E62E62E0F62E03ED18E017
:1053E000D7018D917D010F94BD0F882359F00F9443
:1053F000860F0F94C231F801608371838283938397
:105400000E9496C50C5F1F4FF8E0033E1F0741F74F
:105410009AC40E944C9D87FD96C45AE9E52E52E03D
:10542000F52E03ED18E0D7018D917D010F94BD0F8E
:10543000882339F00F94860FF80164A375A386A31F
:1054400097A30C5F1F4FF8E0033E1F0761F77BC473
:105450008091790687FF02C00C94703580917A069E
:105460008E7011F00C947035409107095091080925
:105470006091090970910A0983EB96E00F940A1173
:1054800040910B0950910C0960910D0970910E0922
:1054900080EB96E00F940A1140910F09509110098A
:1054A00060911109709112098DEA96E00F940A112A
:1054B0008AE00E94714147C40E947CA444C43AE936
:1054C000C32E32E0D32E4AECE42E44E0F42E10E05A
:1054D000D6018D916D010F94BD0F882351F00F946B
:1054E000860FF7016083718382839383812F0E94EB
:1054F000E7D51F5FF4E0EF0EF11C133049F70C9471
:10550000B3208AE50F940610882351F00F94860F7C
:105510006093820870938308809384089093850831
:1055200080917B0681FD0FC40C94B6350E944C9D82
:10553000182F87FD08C488E50F940610882361F0B2
:105540000F94860F2CE01202F0011124E659F74F58
:10555000608371838283938389E50F940610882387
:1055600061F00F94860F3CE01302F0011124E6591C
:10557000F74F64837583868397838AE50F940610BB
:10558000882361F00F94860F4CE01402F00111247F
:10559000E659F74F608771878287938780917A06F3
:1055A00087FDD1C380917B06837009F0CCC30C9436
:1055B000BA3583E50F940610882309F4C4C30E940A
:1055C000B1A19093650280936402BDC30E944C9D7B
:1055D000F82E87FDB8C383E50F9406100F2D0F2C0E
:1055E000000C110B882369F10E94B1A1F801EE0FA4
:1055F000FF1FEA59FD4F91838083000F111F000F99
:10560000111FF801E05DFD4F7F01BC01990F880B70
:10561000990B0F94072A2AE037ED43E25CE30F94DD
:10562000662AF801EF53F74F20813181428153817F
:105630000F94662AD7016D937D938D939C93139756
:1056400082C30F943B1185E40E94714180E38F0D6A
:105650000E947141F801EE0FFF1FEA59FD4F608172
:10566000718183ED96E00F941A1185E20E947141D9
:105670008AE00E94714167C380E50F94BD0F8823C3
:1056800009F461C360E070E080E50E94B5A1F82EE6
:105690006FEF7FEF83E50E94B5A18C010196039720
:1056A00008F051C3F7FC4FC38F2D0F94E01B8823E4
:1056B00039F00F9438118BED96E00F94DF1043C34F
:1056C0000E94B1D160E08F2D0F943B010F3FBFEFDF
:1056D0001B0731F00130110571F000E010E00DC042
:1056E0008F2D0F94E50031E020E0892B09F030E0A8
:1056F000032F122F02C001E010E08F2D0F94E50060
:105700008017910709F41FC380E00E949142F5CFF2
:1057100064E071E083E50E94A69F8C0168EE73E06F
:1057200080E50E94A69F8938E3E19E0710F088E893
:1057300093E1B8010E9429F806C360E085E40E9465
:10574000A5A1182F823008F08DC080E50F94BD0F01
:10575000E12EF12C882371F00F94860F27E12E9D06
:10576000F0012F9DF00D1124E55DF74F63877487DD
:105770008587968789E40F94BD0F8823B9F00F942D
:10578000860F27E12E9D80012F9D100D1124055DB0
:10579000174F2CEA35EC47E25EE30F94662AD801F6
:1057A0001F966D937D938D939C93529784E40F94F1
:1057B000BD0F8823A9F00F94860F27E12E9D80014D
:1057C0002F9D100D1124055D174F2CEA35EC47E293
:1057D0005EE30F945531F801638B748B858B968B48
:1057E0000F943B11B70188E097E00F941A1187E1FD
:1057F0008E9D80018F9D100D1124055D174FD801DE
:105800001B964D915D916D917C911E9784E097E080
:105810000F940A112CEA35EC47E25EE3F801678544
:105820007089818992890F945531AB01BC0180E068
:1058300097E00F940A112CEA35EC47E25EE3D801B9
:1058400053966D917D918D919C9156970F94662AF8
:10585000AB01BC018CEF96E00F940A118AE00E9424
:10586000714171C20F9438118AEE96E00F94DF10E7
:105870006AC283E40F94BD0F882321F00E94B1A176
:105880000E94855260918B0270918C028CE097E0AF
:105890000F941A118AE00E94714155C283E50F945A
:1058A000BD0F182F882371F00F94860F0F94BD3110
:1058B000709339026093380221E0672B09F020E0F1
:1058C0002093EB0780E50F94BD0F882359F02091BA
:1058D000380230913902232B11F00F94770F809307
:1058E000EB0731C211112FC20F943B1187E397E0F0
:1058F0000F94DF108091EB07882319F08FE197E078
:1059000002C08BE197E00F94DF1060913802709134
:10591000390286E297E00F941A1182E297E00F9421
:10592000DF1011C20E94B1D10EC280917A0686703A
:1059300011F00C9406360C94F1350E94C5FD8111CE
:1059400002C208EE1FE2E2E7F2E0FDA3ECA39E0133
:105950002F5F3F4F190177E9C72E70E3D72E7901EA
:10596000F8016591759185919491ACA1BDA18D903F
:105970009D90AD90BD90BDA3ACA3A50194010F94E3
:1059800078302B013C01F70160837183828393831C
:1059900020E030E040EA51EC0F949F3287FD0AC0CE
:1059A00020E030E040EA51E4C301B2010F94012A43
:1059B000181634F4F6018491181614F40C941D365C
:1059C000D7018D909D90AD90BD907D0120E030E09D
:1059D00040EA51ECC501B4010F949F3287FF02C029
:1059E0000C94293620E030E040EA51E4C501B401CE
:1059F0000F94012A181614F00C943D360C94293695
:105A00000E94B880A0C10F94230A9DC161E083E584
:105A10000E94F3A491E089270F948E0C94C181E039
:105A200080938A0F0E94688510928A0F882309F458
:105A30008AC10F943B118EE997E00F94DF1083C168
:105A40008091470D82FF7FC180648093470D7BC1A9
:105A50000E944C9D082F87FD76C185E50F94BD0FF0
:105A60008823B1F1E02E002E000CFF080F94860F62
:105A70004B015C0120E030E0A9010F949F3287FFC9
:105A800004C0B7FAB094B7F8B094C70153E0880FD8
:105A9000991F5A95E1F79C012557304F7901D9019B
:105AA0008D929D92AD92BC92139720E030E04FE230
:105AB00054E4C501B4010F949F3218164CF480E0F1
:105AC00090E0AFE2B4E4F70180839183A283B383D3
:105AD0008CE40F94BD0F882309F435C1002E000C0F
:105AE000110B0F94860F6B017C0120E030E0A901BF
:105AF0000F949F3287FF04C0F7FAF094F7F8F09400
:105B000043E0000F111F4A95E1F70557104FD801E8
:105B10001496CD92DD92ED92FC92179720E030E042
:105B20004FE254E4C701B6010F949F3218160CF0EF
:105B30000AC180E090E0AFE2B4E4F8018483958389
:105B4000A683B78300C10E94B99FFDC00E944C9DEF
:105B5000082F87FDF8C08AE50F940610882349F0C6
:105B600040E050E0BA018AE50E94D4924B015C010A
:105B700006C0812C912C30EAA32E31E4B32E402FA5
:105B800064E083E00E94487710911E09E02E002E09
:105B9000000CFF08812F90E08E159F0521F060E03A
:105BA000802F0E94E5C620E030E0A901C501B401C4
:105BB0000F949F3218167CF580E090E0A0E2B1E4EB
:105BC00089839A83AB83BC8320917A0230917B02D4
:105BD00040917C0250917D02C501B4010F9479304F
:105BE0002B013C0120E030E04BE653E40F94012A06
:105BF00087FD06C0412C512C2BE6622E23E4722E29
:105C00004C8E5D8E6E8E7F8EBE016F5F7F4FCE019C
:105C10004C960E9490D885E50F94BD0F882329F0FB
:105C20000F94860F6B017C010CC0F70193E0EE0F1F
:105C3000FF1F9A95E1F7E557F04FC080D180E280D1
:105C4000F38020E030E0A901C701B6010F949F3234
:105C500087FF04C0F7FAF094F7F8F094F7FAF0949D
:105C6000F7F8F094C982DA82EB82FC8244E061E0CA
:105C7000CE0101960F943C1320E030E0A901C5014C
:105C8000B4010F949F3218165CF580E090E0A0E21A
:105C9000B1E489839A83AB83BC83A50194016091AD
:105CA0007A0270917B0280917C0290917D020F9428
:105CB00078306B017C0120E030E0A9010F949F3225
:105CC00018161CF0C12CD12C7601CC8EDD8EEE8EF8
:105CD000FF8EBE016F5F7F4FCE014C960E9490D821
:105CE00080911E09181721F060E0812F0E94E5C6FF
:105CF00040911E0960E089E00E94487724C081E05D
:105D0000809341021092380F60E083E50E94F3A473
:105D1000811119C00E94FC9916C00E94FEE013C0B8
:105D200010917E0680911E09181729F060E083E526
:105D30000E94F3A401C081E0682F812F0E94E5C674
:105D400002C00E94FEE06696FFAD6697F11102C0A8
:105D50000E94EC9925962FAD259720931D09C3C766
:105D600011E032E02316310409F010E020E030E0C9
:105D7000A901C701B6010F94012A881F8827881F2F
:105D80001813A4C080E090E0A0E8BFE38CA79DA713
:105D9000AEA7BFA72CA13DA14EA15FA1C501B40133
:105DA0000F94783020E030E040E05FE30F94662A03
:105DB0006CA37DA38EA39FA328A539A54AA55BA5A7
:105DC000C301B2010F94783020E030E040E05FE39F
:105DD0000F94662A68A779A78AA79BA72CA13DA143
:105DE0004EA15FA1CA01B9010F94662A4B015C0163
:105DF00028A539A54AA55BA5CA01B9010F94662A51
:105E00009B01AC01C501B4010F9479300F94E532C8
:105E10004B015C019B01AC01C701B6010F947830C6
:105E20002B013C01A5019401C701B6010F94793003
:105E30009B01AC01C301B2010F94662A6B017C0186
:105E400020E030E0A9010F949F3287FD07C0C70111
:105E5000B6010F94E5322B013C0103C0412C512CBB
:105E6000320168A579A58AA59BA59058A501940142
:105E70000F9455312CA53DA54EA55FA50F94662A1C
:105E8000A30192010F94662A2CA13DA14EA15FA10E
:105E90000F9479306B017C01A50194016CA17DA167
:105EA0008EA19FA10F9455312CA53DA54EA55FA5B0
:105EB0000F94662AA30192010F94662A28A539A59A
:105EC0004AA55BA50F9479300C94B91F80E090E04F
:105ED000A0E8BFEB5BCF0F94381185E593E00F94FA
:105EE000DF1031CF20E030E0A901C701B6010F94E7
:105EF000012A882381F31CA61DA61EA61FA6A701A2
:105F0000960150582CA33DA34EA35FA38CA59DA53D
:105F1000AEA5BFA5B05888A799A7AAA7BBA7CA01D5
:105F2000B9010F94662A4B015C0128A539A54AA541
:105F30005BA5CA01B9010F94662A9B01AC01C5019A
:105F4000B4010F9479300F94E53224966CAF7DAF95
:105F50008EAF9FAF249720917202309173024091CF
:105F600074025091750228AB39AB4AAB5BABC701E9
:105F7000B6010F94793029966CAF7DAF8EAF9FAF8D
:105F800029978091760290917702A0917802B09142
:105F900079028CAB9DABAEABBFAB2CA53DA54EA59E
:105FA0005FA5BC01CD010F9479302D966CAF7DAF0C
:105FB0008EAF9FAF2D972091860830918708409132
:105FC00088085091890828AF39AF4AAF5BAF29964E
:105FD0002CAD3DAD4EAD5FAD299768AD79AD8AADC5
:105FE0009BAD0F9478306B017C0180918A08909171
:105FF0008B08A0918C08B0918D088CAF9DAFAEAF8F
:10600000BFAF2D962CAD3DAD4EAD5FAD2D97BC0114
:10601000CD010F9478304B015C01A70196016CA172
:106020007DA18EA19FA10F94662A2B013C01A501A1
:10603000940168A579A58AA59BA50F94662A9B0162
:10604000AC01C301B2010F9479302B013C01A501D1
:1060500094016CA17DA18EA19FA10F94662A4B0192
:106060005C01A701960168A579A58AA59BA50F9457
:10607000662A9B01AC01C501B4010F947830A301DD
:1060800092010F94EC306B017C0120E030E0A9011B
:106090000F94012A87FF0AC02BED3FE049EC50E442
:1060A000C701B6010F9479306B017C012BED3FE005
:1060B00049EC50E4C701B6010F94553120E030E0BF
:1060C00040EC51E40F94662A0F943F310F94C23193
:1060D0008B01672B11F401E010E092E029163104E6
:1060E00051F42BED3FE049EC50E4C701B6010F94A9
:1060F00078306B017C0120E030E0A901C701B601D6
:106100000F94012A811122C028AD39AD4AAD5BAD93
:1061100068A979A98AA99BA90F94012A811116C09F
:106120002CAD3DAD4EAD5FAD6CA97DA98EA99FA9EB
:106130000F94012A81110AC008E110E07BEDC72EFF
:106140007FE0D72E79ECE72E70E4F72E20917A02CB
:1061500030917B0240917C0250917D022CAB3DAB93
:106160004EAB5FAB60918E0870918F088091900864
:10617000909191080F9478302B013C01A701960172
:1061800024966CAD7DAD8EAD9FAD24970F94662A9D
:106190004B015C0120E030E0A901C301B2010F9482
:1061A000012A8823C9F0A5019401C501B4010F9407
:1061B000662A4B015C01A3019201C301B2010F9455
:1061C000662A9B01AC01C501B4010F9479300F948C
:1061D000E5324B015C010DC020E030E0A901C501B2
:1061E000B4010F949F3287FF04C0B7FAB094B7F898
:1061F000B0942FE632E143E85AE3C501B4010F94AD
:10620000012A87FD08C28091920890919308A0917D
:106210009408B09195088CAF9DAFAEAFBFAF209101
:106220007E0230917F02409180025091810228AF1E
:1062300039AF4AAF5BAF2AE037ED43E25CE36091F0
:106240005A0270915B0280915C0290915D020F9402
:10625000662A68AB79AB8AAB9BAB609164027091A4
:106260006502072E000C880B990B0F94072A9B01DF
:10627000AC0168A979A98AA99BA90F94662A6C8F99
:106280007D8F8E8F9F8FC501B4010F94EE310F94D7
:10629000C2311B016017710708F41801B10180E0D9
:1062A00090E00F94052A4B015C019B01AC01C701F2
:1062B000B6010F94553168AB79AB8AAB9BABA501A6
:1062C0009401C301B2010F94553161966CAF7DAF5B
:1062D0008EAF9FAF619728AD39AD4AAD5BAD6CAD68
:1062E0007DAD8EAD9FAD0F947830A50194010F94D4
:1062F000553165966CAF7DAF8EAF9FAF659728A97E
:1063000039A94AA95BA9CA01B9010F94662A20E0FC
:1063100030E040E05FE30F94662A9B01AC0160E04F
:1063200070E080E89FE30F9478306CAF7DAF8EAF64
:106330009FAF8CA99DA9AEA9BFA989879A87AB8772
:10634000BC8728AD39AD4AAD5BAD2D873E874F8701
:10635000588B0F9476029B01AC0128533F4F4F4F4F
:106360005F4F24962CAF3DAF4EAF5FAF24974CA04C
:106370005DA06EA07FA041E050E05DAB4CAB59E169
:1063800058AF8CA99DA98215930508F016C10E94EB
:10639000E4A50F947602DC01CB0124962CAD3DAD33
:1063A0004EAD5FAD2497821B930BA40BB50BB7FDCD
:1063B00011C00F9476029B01AC0128533F4F4F4F01
:1063C0005F4F24962CAF3DAF4EAF5FAF249780E078
:1063D0000E94914238AD315038AF3323E9F128A5FE
:1063E00039A54AA55BA56CAD7DAD8EAD9FAD0F9473
:1063F000662A6B017C019201A30168A979A98AA987
:106400009BA90F94662AA70196010F9479307B010E
:106410008C019201A3016CAD7DAD8EAD9FAD0F944B
:10642000662A4B015C0128A539A54AA55BA568A988
:1064300079A98AA99BA90F94662A9B01AC01C50181
:10644000B4010F9478302B013C01C701D80188A713
:1064500099A7AAA7BBA74FC04CA95DA9BA0180E024
:1064600090E00F94052A28A939A94AA95BA90F949D
:10647000662A4B015C010F9452316B017C01C5010E
:10648000B4010F94DB324B015C01A70196016CA1B2
:106490007DA18EA19FA10F94662A2B013C012CA502
:1064A0003DA54EA55FA5C501B4010F94662AA301C1
:1064B00092010F9479302B013C01A50194016CA14C
:1064C0007DA18EA19FA10F94662A4B015C012CA592
:1064D0003DA54EA55FA5C701B6010F94662A9B0195
:1064E000AC01C501B4010F94783068A779A78AA7D9
:1064F0009BA759E158AF9201A30129966CAD7DADE0
:106500008EAD9FAD29970F94793069837A838B8301
:106510009C8328A539A54AA55BA52D966CAD7DADBC
:106520008EAD9FAD2D970F9479306D837E838F83D1
:10653000988761962CAD3DAD4EAD5FAD6197698595
:106540007A858B859C850F94793069877A878B87CC
:106550009C8765962CAD3DAD4EAD5FAD65976D8565
:106560007E858F8598890F9479306D877E878F8798
:10657000988BCE0101960E9478D6A12CB12C60E8B0
:10658000C62E6FE3D62EE0901E098E01045E1F4FCB
:106590009E01235F3F4FAE01475F5F4FBE016B5FC0
:1065A0007F4FCE0101960E9414D1882331F08CA92F
:1065B0009DA901969DAB8CABE4CE80E1E6E8F8E0C6
:1065C000DE01119601900D928A95E1F7CE010196B8
:1065D0000E9478D6A12CB12C50E8C52E5FE3D52EB1
:1065E000E0901E098E01045E1F4F9E01235F3F4F06
:1065F000AE01475F5F4FBE016B5F7F4FCE010196DB
:106600000E9414D180E1FE013196A2E7B2E0019030
:106610000D928A95E1F70F947602609327087093A4
:1066200028088093290890932A088DCB0E94B1D125
:10663000C0901E0961E080E00E94E5C610921B092F
:1066400080915A0290915B02A0915C02B0915D0230
:106650008093780390937903A0937A03B0937B039C
:106660008091640290916502909377038093760302
:1066700084E690E0909365028093640281E08093C9
:10668000C8040F94190A88E50F94BD0F182F89E5E7
:106690000F94BD0F082F8AE50F94BD0F10134BC147
:1066A000181711F0012F47C101E011E0FF24F39406
:1066B00080E1E2E7F2E0A6E8B8E001900D928A9569
:1066C000E1F782E50F940610882369F00F94860F96
:1066D0004B015C0120E030E0A9010F94012A8823DE
:1066E00009F43FC006C0812C912C40EAA42E40E45E
:1066F000B42E111103C0002309F490C08091D10879
:1067000082FD09C060917A0270917B0280917C02C7
:1067100090917D0203C060E070E0CB01A50194017F
:106720000F94793060938E0870938F08809390084F
:106730009093910820917A0230917B0240917C02E3
:1067400050917D020F949F3218165CF419821A82C0
:106750001B821C82BE016F5F7F4F8EE898E00E9413
:1067600090D8112309F455C011E010931E0980E060
:106770000E94B1D88091720290917302A09174022C
:10678000B091750280933D0290933E02A0933F0228
:10679000B093400210921E0980E00E94B1D880910F
:1067A0007A0290917B02A0917C02B0917D0240918F
:1067B0007602509177026091780270917902809010
:1067C000720290907302A0907402B0907502809251
:1067D000590890925A08A0925B08B0925C084093C6
:1067E0005D0850935E0860935F0870936008809323
:1067F000610890936208A0936308B09364081092B4
:106800006508109266081092670810926808109345
:106810006908002319F081E00E94B1D8FF2019F027
:1068200082E00E94B1D80E94AED880915E02823090
:106830000CF45BC011E010931E0980E00E94B1D8F7
:106840008091720290917302A0917402B0917502CE
:1068500080933D0290933E02A0933F02B09340028A
:1068600010921E0980E00E94B1D880917A02909126
:106870007B02A0917C02B0917D0240917602509102
:106880007702609178027091790280907202909004
:106890007302A0907402B090750280925908909291
:1068A0005A08A0925B08B0925C0840935D08509330
:1068B0005E0860935F08709360088093610890930E
:1068C0006208A0936308B093640810926508109260
:1068D0006608109267081092680810936908E092A1
:1068E0001B09D0925E020F940A1B8091C70480930B
:1068F000C8048091780390917903A0917A03B091B4
:106900007B0380935A0290935B02A0935C02B09346
:106910005D02809176039091770390936502809356
:10692000640260E08C2D0E94E5C683E080938D02B6
:106930000F94E00B08CAF82EBBCE11110C94EC2278
:106940000C94E52280E00E9491420C94102388E58B
:106950000F94BD0F882331F05F98809108018270F9
:106960008093060189E50F94BD0F81118A988AE50D
:106970000F94BD0F882329F08091080181708093C6
:10698000060185E40F94BD0F882309F4DCC90E9439
:106990003040D9C960E087E893E00E9455F85F98DD
:1069A000809108018270809306018A988091080185
:1069B0008170809306010E943040C5C90F94560F24
:1069C000AB01BC014093430D5093440D6093450DC2
:1069D0007093460D81E39BE00F94C618B4C961E043
:1069E000802F0F943B016F2D802F0F940D016F2D81
:1069F00070E0802F0F947701A6C980E090E00C949E
:106A0000D6250E948A8B0C942126012B59F0809167
:106A10006A0390916B038C0D9D1D61E00E94D199DA
:106A20000C94112680E090E0F8CFA7019601C301F5
:106A3000B2010F949F321816B4F08EE594E09F9344
:106A40008F930F5C1F4F1F930F9384E794E09F93E6
:106A50008F931F920E94B6F80FB6F894DEBF0FBE58
:106A6000CDBF0C944B2689E694E0E9CF0E94B1D1CA
:106A700088E50F94BD0F882361F05F9A809108012B
:106A800080958270809306018091D1088E7F8093DB
:106A9000D10889E50F94BD0F882331F08A9A80913F
:106AA000D1088D7F8093D1088AE50F94BD0F88238C
:106AB00059F0809108018095817080930601809142
:106AC000D1088B7F8093D10885E40F94BD0F882374
:106AD00009F439C90E940F4036C90E94B8D333C99E
:106AE00083E50F940610882391F00F94860F60932E
:106AF0000709709308098093090990930A09609324
:106B00000F0970931009809311099093120980E581
:106B10000F940610882351F00F94860F6093070995
:106B2000709308098093090990930A0982E50F94EC
:106B30000610882351F00F94860F60930B09709311
:106B40000C0980930D0990930E0984E50F940610AB
:106B5000882309F4F8C80F94860F60930F09709387
:106B600010098093110990931209EDC880E00E94EA
:106B70005DA4E9C80F943B1183EC96E00F94DF10FD
:106B80000AE618E082E8E82E88E0F82E80E20E940B
:106B90007141D8016D917D918D919C9142E00E944F
:106BA000FD418CE20E947141F8016481758186810A
:106BB000978142E00E94FD418CE20E947141D80120
:106BC00018966D917D918D919C911B9743E00E9449
:106BD000FD41045F1F4FE016F10611F40C94F12300
:106BE000D5CF0F943B1181E597E00F94DF10809192
:106BF0008A02811108C08AE497E00F94DF108AE0CE
:106C00000E947141A0C88EE497E0F7CF82E50F940F
:106C1000BD0F082F83E50F94BD0F182F011103C07E
:106C2000112309F490C80F94500F112309F48BC855
:106C30000F94770F80938A0286C8B7FAB094B7F89A
:106C4000B094D7018D929D92AD92BC9213970C9403
:106C5000E02C0F94381180E897E00F94DF1061E08A
:106C600082E797E00E9455F80E94604D68E270E06C
:106C700088EC90E00E9429F866C80C5F1F4FBFEFB8
:106C8000CB1ADB0AEFE2043F1E0711F00C94B02C84
:106C90006AECE62E64E0F62E10E0F101819191910C
:106CA000A191B1911F01F70181939193A193B193A8
:106CB0007F01812F0E94E7D51F5F133071F70F947A
:106CC000E00B60E082E697E00E9455F863E972E02D
:106CD00084E690E00E9429F86AEB72E084E690E096
:106CE0000E9429F830C8CB5ADF4F0FB6F894DEBFA8
:106CF0000FBECDBFDF91CF911F910F91FF90EF900D
:106D0000DF90CF90BF90AF909F908F907F906F90CB
:106D10005F904F903F902F9008952CEA35EC47E21A
:106D20005EE360917D0370917E0380917F0390917B
:106D300080030F94553160935508709356088093E3
:106D400057089093580808952CEA35EC47E25EE323
:106D500060918103709182038091830390918403F9
:106D60000F94662A609351087093520880935308D9
:106D70009093540808952CEA35EC47E25EE3609165
:106D80007D0370917E0380917F03909180030F9427
:106D9000553160933E0870933F088093400890936C
:106DA000410808952CEA35EC47E25EE360918103E7
:106DB0007091820380918303909184030F94662ADB
:106DC00060933A0870933B0880933C0890933D0889
:106DD00008950C94684DCF93DF93EC01CB01BA0179
:106DE0000F94072A20E030E048EC51E40F94662A23
:106DF0000F94C231688379838A839B83DF91CF911B
:106E000008956BEE76E38DE097E30C94D9506EEF26
:106E100078E483E39EE40C94D9500F94072A20E091
:106E200030E048EC51E40F94662A0C947E4D0F93A9
:106E3000CF93DF93CDB7DEB700E22EE349855A85C5
:106E400068858F810E943952DF91CF910F9108950B
:106E500063E972E084E690E00E9429F86AEB72E050
:106E600084E690E00C9429F82F923F924F925F9223
:106E70006F927F928F929F92AF92BF92CF92DF924A
:106E8000EF92FF920F931F93CF93DF9300D0CDB774
:106E9000DEB748014090040F5090050F6090060F38
:106EA0007090070F411451046104710479F0E1E01E
:106EB000141415040CF0E0E0E093B7071092040FEF
:106EC0001092050F1092060F1092070F1091B7073E
:106ED000E0910A0FEB8310920A0FE11105C0E091D7
:106EE0008D02EE2309F474C029011A013B015C01F3
:106EF000C4010E943A50082FC114D10409F466C09D
:106F0000C6010E943A501A821982E114F104B1F4C8
:106F1000402F50E0282F30E0CA01820F931F469780
:106F20006CF485E190E0841B950B821B930B97FD1D
:106F30000196959587958A8381E0898301E02BE806
:106F400039E4A401BE016F5F7F4FCE0102960E941B
:106F5000A17EE114F10491F08A81882321F01A8244
:106F600089818F5F898300E02EE839E4A701BE01A3
:106F70006F5F7F4FCE0102960E94A17EC114D104A3
:106F800059F000E02BE839E4A601BE016F5F7F4FA6
:106F9000CE0102960E94A17E41E04127B30181E02B
:106FA0000E9415FFC5010E943A50412FB50194E19E
:106FB000981B892F0E9415FFFB81FF2349F01123A5
:106FC00011F0F10101C0F201199502C080E09BCFE0
:106FD0000F900F900F90DF91CF911F910F91FF9025
:106FE000EF90DF90CF90BF90AF909F908F907F9069
:106FF0006F905F904F903F902F90089580918D02F9
:10700000882331F041E069EA77E082E00C94D6FE13
:10701000089521E020930B0F0E94549A10920B0FB9
:1070200008950F931F93CF93DF93CDB7DEB76E977D
:107030000FB6F894DEBF0FBECDBFFC01EE0FFF1FF1
:10704000EB5FFD4F21812F9320812F939F938F938F
:1070500088E098E09F938F938E010F5F1F4F1F93DF
:107060000F930F949B29C801D4DF0FB6F894DEBFAD
:107070000FBECDBF6E960FB6F894DEBF0FBECDBF6C
:10708000DF91CF911F910F9108958091890F90E02A
:10709000C8CF8091890F90E0C4CFCF93DF9300D009
:1070A0001F92CDB7DEB7FC0180819181A281B381AF
:1070B00080937A0290937B02A0937C02B0937D022E
:1070C00080E090E0A0E0B1E489839A83AB83BC8345
:1070D000CE0101960E9497D70F900F900F900F90BE
:1070E000DF91CF9108958111B3CE68EB71E084E117
:1070F00090E00C9429F80F94D30BF5CF0E94B88040
:10710000F2CF282F1092580F8091040F9091050F05
:10711000A091060FB091070FB7FF08C01092040F9F
:107120001092050F1092060F1092070F8091030F17
:10713000882331F08091040F8093790410927804B1
:10714000809177041816FCF4082E000C990B821B12
:10715000910920917904022E000C330B281739076E
:1071600094F097FF02C080E090E080937904092EAC
:10717000000CAA0BBB0B8093040F9093050FA093F8
:10718000060FB093070F809179046623A9F09091C0
:107190007A04891714F480937A0420917A04022ED9
:1071A000000C330B2C5F3F4F482F082E000C550B63
:1071B000241735071CF4845080937A0408954F9265
:1071C0005F926F927F928F929F92AF92BF92CF9277
:1071D000DF92EF92FF920F931F93CF93DF9300D034
:1071E0001F92CDB7DEB761E081E08BDF60907A045B
:1071F000712C5524539423E0422E61100BC08091D2
:10720000790481112AC080910A0F10920A0F81110E
:107210001EC023C081E068120BC0909179049130A8
:10722000C1F580910A0F10920A0F811127C031C059
:1072300082E06812A1C080917904823009F0CEC04A
:1072400080910A0F10920A0F8111B7C0C7C00E9427
:10725000684D809178048111B9C380918D02882393
:1072600061F181E090917904911180E004E024E0E3
:1072700046EB53E1672D0E9439521FC080911808D8
:1072800086258093180840928D02809178048111A0
:107290009DC380918D02882381F081E0913009F0B7
:1072A00080E090911808911176C025E538E001E062
:1072B0004CE558E0672D0E94DA512CEA35EC47E2A4
:1072C0005EE360913A0870913B0880913C08909190
:1072D0003D080F945531609381037093820380932E
:1072E0008303909384032CEA35EC47E25EE36091DC
:1072F0003E0870913F0880914008909141080F949A
:10730000662A60937D0370937E0380937F0390933E
:10731000800385E068120EC01092890F8091790475
:10732000853009F007C180910A0F10920A0F811170
:10733000ECC000C186E068120EC01092890F8091E7
:107340007904863009F0DCC180910A0F10920A0F8F
:107350008111BFC1D5C187E0681232C11092890F77
:1073600080917904873009F0FCC180910A0F109256
:107370000A0F8111DFC1F5C183E068120FC080914F
:107380007904833009F055C080910A0F10920A0FDA
:1073900081113EC04EC029E538E089CF84E06812F3
:1073A0008CCF80917904843009F08DC080910A0FD0
:1073B00010920A0F81115BC086C0E12CF12C02E80B
:1073C00013E420E030E0A90168E272E08EE498E086
:1073D0000F944F00809178048111F8C280918D0242
:1073E000882309F46ACF11E080917904823009F092
:1073F00010E0609128027091290280912A029091F8
:107400002B020E943C4E00E09C014EE458E02AC052
:10741000E12CF12C02E813E420E030E0A90164E261
:1074200072E087E498E00F944F0080917804811116
:10743000CDC280918D02882309F43FCF11E0809165
:107440007904833009F010E06091240270912502E4
:1074500080912602909127020E943C4E00E09C0100
:1074600047E458E0672D812F0E94DA517DC020E06B
:1074700030E048EC52E460912C0270912D02809132
:107480002E0290912F020F94662A0F94C2311F9200
:10749000812C912CABE8AA2EA1E5BA2E6B0118EE37
:1074A000E12E13E0F12E00E010E020E030E0A90131
:1074B0006CE272E08FE398E00E944F4C0F90809155
:1074C0007804811183C280918D02882309F44CC015
:1074D00011E080917904843009F010E080912C0251
:1074E00090912D02A0912E02B0912F0289839A8350
:1074F000AB83BC83CE0101960E9409F500E09C019C
:107500004FE358E0672D812FD6CEC12CD12CE12C32
:1075100018E1F12E0CE116E420E030E040E85FE3F2
:1075200066E378E087E398E00F947624809178040E
:1075300081114CC280918D02882309F464C011E04E
:1075400080917904853009F010E0609136087091DF
:10755000370880913808909139080E94974D00E0D3
:107560009C0147E358E04BC02CEA35EC47E25EE370
:1075700060913A0870913B0880913C0890913D08D9
:107580000F9455316093810370938203809383033A
:10759000909384032CEA35EC47E25EE360913E0869
:1075A00070913F0880914008909141080F94662A9D
:1075B00060937D0370937E0380937F039093800399
:1075C00088E0681220C01092890F80917904883079
:1075D00009F478C080918D02882309F460C111E01C
:1075E00080917904883009F010E080910502909133
:1075F00006020E94C9F600E09C0148E158E0672DB0
:10760000812F0E94DA512CEA35EC47E25EE360916B
:1076100051087091520880915308909154080F942A
:107620005531609381037093820380938303909319
:1076300084032CEA35EC47E25EE3609155087091D3
:10764000560880915708909158080F94662A6093C5
:107650007D0370937E0380937F039093800389E082
:1076600068120EC05092890F80917904893009F018
:10767000C0C080910A0F10920A0F8111A5C0B9C035
:107680008AE068120EC05092890F809179048A3086
:1076900009F0E0C080910A0F10920A0F8111C3C057
:1076A000D9C08BE0681227C15092890F809179046C
:1076B0008B3009F048C180910A0F10920A0F811196
:1076C0002BC141C180910A0F10920A0F811167C02E
:1076D00081CF72EDC72E76E3D72EE12C18E1F12E83
:1076E0000CE116E42AE037ED43E25CE361E873E085
:1076F0008FE298E00F94762480917804811166C11E
:1077000080918D02882309F47ECF11E08091790465
:10771000863009F010E060918103709182038091BE
:107720008303909184030E94974D00E09C014FE2F7
:1077300058E030C05BEBC52E56E3D52EE12C18E1A6
:10774000F12E0CE116E420E030E040E85FE36DE765
:1077500073E087E298E00F94762480917804811199
:1077600035C180918D02882309F44DCF11E08091BD
:107770007904873009F010E060917D0370917E03F9
:1077800080917F03909180030E94974D00E09C01BF
:1077900047E258E0672D812F0E94DA5180C00F9494
:1077A000D900E12C09E418E324E031E046E950E097
:1077B00065E072E088E198E00E94BF4C8091780417
:1077C000882309F407CF02C1C12CD12CE12C18E188
:1077D000F12E0CE116E420E030E040E85FE36DE4D8
:1077E00078E087E398E00F94762480917804811103
:1077F000EDC080918D02882309F448C011E080918A
:107800007904893009F010E060914D0870914E08BC
:1078100080914F08909150080E94974D00E09C0184
:1078200047E358E02FC024EAC22E26E3D22EE12CF3
:1078300018E1F12E0CE116E42AE037ED43E25CE3B7
:1078400061E873E08FE298E00F94762480917804E9
:107850008111BCC080918D028823C1F011E080911C
:1078600079048A3009F010E06091810370918203FD
:1078700080918303909184030E94974D00E09C01C6
:107880004FE258E0672D812F0E94DA517394639480
:1078900085E07812B2CC8DE08093770497C02CEA13
:1078A00035EC47E25EE36091510870915208809197
:1078B0005308909154080F9455316093810370934D
:1078C000820380938303909384032CEA35EC47E290
:1078D0005EE3609155087091560880915708909129
:1078E00058080F94662A60937D0370937E038093FB
:1078F0007F03909380038CE06812C8CF5092890F69
:10790000809179048C3009F04BC080910A0F10925D
:107910000A0F811132C044C08DE8C82E86E3D82EEC
:10792000E12C18E1F12E0CE116E420E030E040E813
:107930005FE36DE773E087E298E00F94762480912F
:107940007804811143C080918D02882309F49ECF71
:1079500011E0809179048B3009F010E060917D0393
:1079600070917E0380917F03909180030E94974DD8
:1079700000E09C0147E258E085CF0F94D900E12C4C
:1079800005E418E324E031E046E950E067E072E006
:1079900088E198E00E94BF4C80917804811116C064
:1079A00080918D02882309F471CF11E080917904D0
:1079B0008C3009F010E080910702909108020E943B
:1079C000C9F600E09C0148E158E05CCF0F900F90B1
:1079D0000F900F90DF91CF911F910F91FF90EF903B
:1079E000DF90CF90BF90AF909F908F907F906F90DF
:1079F0005F904F9008952F923F924F925F926F92B7
:107A00007F928F929F92AF92BF92CF92DF92EF922E
:107A1000FF920F931F93CF93DF9300D01F92CDB7A8
:107A2000DEB761E081E06DDB70907A04612C33E0B9
:107A3000332E71100BC08091790481111CC080918C
:107A40000A0F10920A0F811110C015C021E07212A6
:107A500022C080917904813009F033C280910A0FED
:107A600010920A0F811120C22CC20E94684D809191
:107A70007804811141C280918D02882361F081E0F8
:107A800090917904911180E004E024E046EB53E109
:107A9000662D0E9439528091C008882309F4E2C003
:107AA00032E073126EC080917904823009F043C0D5
:107AB00080910A0F10920A0F8823E9F10F94D900E0
:107AC00040901E09E4E04E9EC00111249C01275302
:107AD000374F290120E030E04AE754E4F2016081A9
:107AE0007181828193810F94662A20E030E84BEB0C
:107AF00054E40F9478300F94C2311F92E3E98E2E34
:107B0000E0ED9E2EF6E8AF2EF1E5BF2E6B0116EDEF
:107B1000E12E16E0F12E00E010E02CED35E040E023
:107B200050E0B20184EF97E00E944F4C0F9080919B
:107B300078048111E1C180918D02882311F111E057
:107B400080917904823009F010E0E0911E0984E010
:107B5000E89FF0011124E753F74F80819181A281C2
:107B6000B38189839A83AB83BC83CE0101960E9443
:107B700079FF00E09C0144EF57E0662D812F0E94C1
:107B8000DA5199EC492E98E0592E23E0222E8DEF00
:107B9000820D72105DC08093890F809179048711E6
:107BA00039C080910A0F10920A0F882399F10F941F
:107BB000D90020E030E04AE754E4F20160817181AD
:107BC000828193810F94662A20E030E84BEB54E4E5
:107BD0000F9478300F94C2311F9243E9842E40ED08
:107BE000942E56E8A52E51E5B52E6B0116EDE12E2B
:107BF00016E0F12E00E010E02CED35E040E050E022
:107C0000B20188EE97E00E944F4C0F90809178046B
:107C1000811172C180918D028823D1F011E0809191
:107C20007904821110E0F20180819181A281B381F7
:107C300089839A83AB83BC83CE0101960E9479FF2E
:107C400000E09C0148EE57E0662D812F0E94DA513A
:107C50002394F4E04F0E511C25E0221298CF85E0CA
:107C6000482E02C002E0402E471042C080917904A5
:107C700084111FC080910A0F10920A0F8823C9F047
:107C80000F94D90060911E09F8E06F9FB001112494
:107C90006557704FE12CF12C0FE214E420E030E046
:107CA000A9018EED97E00F944F0080917804811127
:107CB00023C180918D028823D9F011E0809179044D
:107CC000871110E0E0911E0938E0E39FF0011124D4
:107CD000E557F04F60817181828193810E943C4E13
:107CE00000E09C014EED57E0662D812F0E94DA5195
:107CF00043941BE8C12E1FE0D12E212C741036C0F6
:107D00002092890F80917904871118C080910A0F01
:107D100010920A0F882391F00F94D900E12CF12CD6
:107D20000FE214E420E030E0A901B6018CEC97E00A
:107D30000F944F00809178048111DEC080918D02F4
:107D40008823A1F011E080917904841110E0F601FC
:107D500060817181828193810E943C4E00E09C0190
:107D60004CEC57E0662D812F0E94DA51542C4424AC
:107D70004394450C2394F8E0CF0ED11C22E022124C
:107D8000BDCF471042C08091790487111FC08091F8
:107D90000A0F10920A0F8823C9F00F94D90060913E
:107DA0001E0928E0629FB00111246157704FE12C39
:107DB000F12C0FE214E420E030E0A90184EC97E01C
:107DC0000F944F0080917804811196C080918D02AC
:107DD0008823D9F011E080917904871110E0E091B7
:107DE0001E0938E0E39FF0011124E557F04F64814C
:107DF0007581868197810E943C4E00E09C0144EC95
:107E000057E0662D812F0E94DA5153945394BFE8B6
:107E1000CB2EBFE0DB2E412C751036C04092890F6F
:107E200080917904871118C080910A0F10920A0F6F
:107E3000882391F00F94D900E12CF12C0FE214E487
:107E400020E030E0A901B60184EB97E00F944F00E9
:107E500080917804811150C080918D028823A1F017
:107E600011E080917904851110E0F6016081718143
:107E7000828193810E943C4E00E09C0144EB57E0DC
:107E8000662D812F0E94DA5153944394F8E0CF0E6F
:107E9000D11C22E04212C0CF6394739435E0631288
:107EA000C8CD5092770428C08091C0088725809360
:107EB000C00830928D020E9493D080917804811185
:107EC0001BC080918D02882309F4E5CD81E090915B
:107ED0007904913009F080E09091C008911103C0BD
:107EE00025E538E002C029E538E001E04EEF57E033
:107EF000662D0E94DA51CFCD0F900F900F900F900A
:107F0000DF91CF911F910F91FF90EF90DF90CF9075
:107F1000BF90AF909F908F907F906F905F904F90A9
:107F20003F902F9008950F931F93522F2091EA0BAB
:107F30003091EB0B2817390721F19093EB0B8093CD
:107F4000EA0B8B0120E030E00093040F1093050F43
:107F50002093060F3093070F40937A0450937704D1
:107F6000895E974721F41092020F10927C0382E001
:107F700080938D0281E0809378041092080F109214
:107F8000B7071F910F910895CF93DF9380918D02D2
:107F9000882341F06091390F70913A0F41E081E000
:107FA0000E94D6FE80910B0F81111AC081E0809350
:107FB0000B0FC091EA0BD091EB0B20E040E060E0AA
:107FC00070E084EC9FE3AFDF0E94B1D110920B0F01
:107FD00020E040E060E070E0CE01DF91CF91A3CFE0
:107FE000DF91CF9108958091A80B9091A90B891BE7
:107FF0008F7009F402C081E0089580918F0E811185
:108000000AC08091AA04813041F08091470D82FB23
:10801000882780F9089580E0089581E00895129AF4
:10802000479A08955F9AA8E0B1E08C91809582709C
:10803000E6E0F1E080838091D1088E7F8093D108C3
:108040008A9A8091D1088D7F8093D1088C918095F8
:10805000817080838091D1088B7F8093D108DFCF9E
:108060001298479808958F929F92AF92BF92CF92A5
:10807000DF92EF92FF92CF9380916F00C82FC27072
:1080800081FF05C080916F008D7F80936F0080918C
:10809000A90B8093A80B8093A70B8093A60B84E673
:1080A0008093A50B0E94CCD588EE93E090931B089B
:1080B00080931A08CC2329F080916F00826080930E
:1080C0006F0081E0809311070E94B1D181E00E948E
:1080D000B9D26B017C0180E00E94B9D24B015C01F6
:1080E0006093890370938A0380938B0390938C032E
:1080F000C0928D03D0928E03E0928F03F092900392
:1081000082E00E94B9D260939103709392038093AE
:108110009303909394038092720290927302A092C0
:108120007402B0927502C0927602D0927702E09209
:108130007802F092790260937A0270937B028093C6
:108140007C0290937D02CF91FF90EF90DF90CF90D3
:10815000BF90AF909F908F900C94AED88091880381
:10816000811107C00F94D30B882319F081E080930D
:10817000880308951092DA0708959091470D93FBB4
:10818000882780F993FF06C081E09091340B91110C
:1081900001C080E0089580918F0E81110FC0809101
:1081A000AA04823059F0E9DF882349F08091470D15
:1081B00082FB882780F991E08927089581E008955E
:1081C0008F929F92AF92BF92CF92DF92EF92FF92E7
:1081D0000F93CF93DF931F92CDB7DEB75C016B0196
:1081E0007A014901F501808191810F9418308983CA
:1081F000002311F0F6018083BE016F5F7F4FC40141
:108200000E9471DBF50180819181019691838083C9
:10821000FFEFCF1ADF0A81E0E81AF10819F780E0D2
:108220000F90DF91CF910F91FF90EF90DF90CF9063
:10823000BF90AF909F908F9008957F928F929F9262
:10824000AF92BF92CF92DF92EF92FF920F931F9364
:10825000CF93DF931F92CDB7DEB77C0159018B011D
:108260006B01C40ED51E0C151D0559F1F701808058
:108270009180F80171908F017982C4010F941830B8
:10828000781691F0672DC4010F942030C4010F942B
:1082900018309981891741F00F943B1185E698E0D9
:1082A0000F94DF1081E00EC0BE016F5F7F4FC501EC
:1082B0000E9471DBF7018081918101969183808317
:1082C000D2CF80E00F90DF91CF911F910F91FF905F
:1082D000EF90DF90CF90BF90AF909F908F907F9066
:1082E00008959091C00095FFFCCF8093C60008953B
:1082F0008F929F92AF92BF92EF92FF920F931F9334
:10830000CF93DF93CDB7DEB7A0970FB6F894DEBF5B
:108310000FBECDBF611571058105910589F100E0A2
:10832000842E912CA12CB12C102FEE24E394F12C4F
:10833000EC0EFD1EE00EF11C07FDFA94A501940160
:108340000F943D30F7016083B901CA010F5F6115D9
:1083500071058105910541F71F3F21F1E1E0F0E052
:10836000EC0FFD1FE10FF11D17FDFA9580818A309A
:1083700010F097E301C090E3890FB3DF1150ECCF09
:1083800080E3A0960FB6F894DEBF0FBECDBFDF919D
:10839000CF911F910F91FF90EF90BF90AF909F9062
:1083A0008F909FCFA0960FB6F894DEBF0FBECDBFC3
:1083B000DF91CF911F910F91FF90EF90BF90AF9001
:1083C0009F908F900895CF92DF92EF92FF926B0172
:1083D0007C0197FF0AC08DE284DFF094E094D09492
:1083E000C094C11CD11CE11CF11C4AE0C701B601BC
:1083F000FF90EF90DF90CF907BCF8F929F92AF92C4
:10840000BF92CF92DF92EF92FF92CF936B017C01EC
:10841000B42E20E030E0A9010F94012A87FF06C0A6
:108420008DE25FDFF7FAF094F7F8F094C0E060E0D7
:1084300070E080E09FE3CB1541F02DEC3CEC4CEC80
:108440005DE30F94662ACF5FF6CF9B01AC01C701B5
:10845000B6010F9479306B017C010F94C2314B014E
:108460005C014AE045DFCC2379F1C501B4010F94EA
:10847000052A9B01AC01C701B6010F9478306B014E
:108480007C018EE22EDF20E030E040E251E4C701C3
:10849000B6010F94662A4B015C010F94BD316B014C
:1084A000770FEE08FF08C701B6018DDFC701B601DF
:1084B0000F94072A9B01AC01C501B4010F947830D9
:1084C0006B017C01C150F9F6CF91FF90EF90DF90E6
:1084D000CF90BF90AF909F908F9008958DE001DF77
:1084E0008AE0FFCECF93DF93EC018991882311F0CE
:1084F000F8DEFBCFDF91CF91F1CF80918106909193
:108500008206981759F0E92FF0E0EF57F94F828172
:108510009F5F9F779093820690E008958FEF9FEF83
:1085200008952F923F924F925F926F927F928F9217
:108530009F92AF92BF92CF92DF92EF92FF920F93F2
:108540001F93CF93DF93CDB7DEB728970FB6F8947C
:10855000DEBF0FBECDBFF82E0E947CF90F947602CD
:108560004B015C0180910002882359F180911D0923
:10857000882339F1409195035091960360919703B8
:108580007091980395018401041B150B260B370B82
:1085900037FD2AC0833079F03CF4813094F00F9499
:1085A0003B1183ED98E00BC0843059F40F943B11DC
:1085B00084EA98E004C00F943B118CEB98E00F9490
:1085C000DF102091000230E0A8EEB3E00F94693094
:1085D000860E971EA81EB91E809295039092960350
:1085E000A0929703B092980380918A02882359F150
:1085F00080917304811127C000DD811104C0809136
:108600008F0E882301F18091A60F87FD03C0815052
:108610008093A60F30911E09809103018695817089
:1086200029B1922F947022FD92E0892B90915E02E5
:108630009250923008F021C5882309F42AC5809110
:10864000A60F87FD2AC580915A06843008F06CC2B7
:1086500020E6D22E80915A06843008F04DC18091D8
:10866000810690918206891B8F7709F445C145DF09
:10867000AC0197FDEFCF20910307309104078A30BA
:1086800019F08D3009F001C11092FD03211531055B
:1086900019F40E94E4A5DECFF901E356FC4F1082E5
:1086A00010920407109203070DE913E0F80181917D
:1086B000803211F48F01FACF8E3409F07AC001159F
:1086C000110509F476C061E17AE0C8010F948129AF
:1086D0005C01892B41F06EE470E0C80104960F94B0
:1086E000DE33009709F4C8014AE050E060E070E032
:1086F00001960F94FE266093990370939A038093DA
:108700009B0390939C034090050750900607609050
:108710000707709008072FEF421A520A620A720A7E
:10872000641575058605970531F0AB2821F460E0E6
:108730008EED99E0DFC06AE270E0C8010F94163454
:108740009C01009709F1982F901BE12C992339F097
:108750009150F801E90FF11D8081E826F7CF4AE03A
:1087600050E060E070E0C90101960F94FE268E2C67
:10877000912CA12CB12C681579058A059B0541F037
:1087800060E08FEB99E0B6C060E085E999E0B2C0A7
:108790008091990390919A03A0919B03B0919C03BF
:1087A0008093050790930607A0930707B0930807E7
:1087B00012C08091470D80FF0EC06AEE7FE1C801B4
:1087C0000F948129009709F492C0FC0183818053A2
:1087D0008A3008F48CC08091410281111CC067E48A
:1087E00070E0C8010F94DE330097A9F04AE050E032
:1087F00060E070E001960F94FE26643071058105FB
:10880000910548F484EF98E00F94DF1060E08AEE61
:1088100098E00E9455F86EE473E0C8010F94E933C4
:10882000892B21F410921E0210921C0963E573E05B
:10883000C8010F94E933892B39F441E060E070E01E
:1088400083E994E00F94C91468E573E0C8010F94BC
:10885000E933892B09F407DC80919D038B3309F4FC
:10886000F9CE80915A06843008F0F4CE8091D60477
:10887000D89EC00111246DE973E087529B4F0F947D
:10888000F23381E00E943F9AE5CE2F3531050CF09E
:10889000E1CE8C35B9F431DE97FDDCCE2091FD03BD
:1088A0002111D8CE2091030730910407A9014F5F11
:1088B0005F4F5093040740930307F901E356FC4FC1
:1088C0008083C8CE8B3321F481E08093FD03C2CE38
:1088D0008091FD038111BECEC901019690930407DA
:1088E00080930307F901E356FC4F4083B3CE60E069
:1088F0008BE699E00E94179A8091470D82FF14C180
:1089000080915A06811102C01092FF03DD24D39496
:108910004091430D5091440D6091450D7091460D6D
:1089200080913F0D9091400DA091410DB091420D6D
:10893000481759076A077B0708F4D12C00E010E0BC
:10894000CC24C39480E6B82E99E6A92E80915A06CD
:10895000843008F0E9C0D110E7C08091FF03811195
:10896000E3C08091390B90913A0BA0913B0BB091F1
:108970003C0B8093430D9093440DA093450DB09311
:10898000460D41E050E0BE016F5F7F4F81E39BE009
:108990000F945005019719F4898190E002C08FEF80
:1089A0009FEFE82E4090430D5090440D6090450D90
:1089B0007090460D40913F0D5091400D6091410DDA
:1089C0007091420DDD24D394441655066606770651
:1089D00008F4D12C4416550666067706B0F40196C5
:1089E00009F45EC02AE0E21609F46BC03DE0E3162C
:1089F00009F467C043E2E41619F05AE3E51279C0BE
:108A00008091FE03811175C051C00E94B1D181E3F4
:108A10009BE00F94D50280913E0D882331F1815067
:108A200080933E0DA89EC001112462E08C56914FA8
:108A30000E9482E6E0913E0D84E0E89FF00111245F
:108A4000E057F14F40815181628173814093430D22
:108A50005093440D6093450D7093460D81E39BE068
:108A60000F94C6180E949BE714C00E9426E60E943D
:108A7000B8D30E94C18B0E943B8B6D337105810579
:108A8000910518F486E19AE002C08BE19AE00E9419
:108A9000859A8091470D82FD0DC08EE29AE004C058
:108AA0000F9438118FE19AE00F94DF1093E2E912EE
:108AB00008C005C003E2E01200C300E010E0C0926D
:108AC000FF031092FE030115110519F40E94E4A59D
:108AD0000DC08091D604B89E000D111D1124F8011F
:108AE000E752FB4F108280E00E943F9A00E010E0C6
:108AF0002DCF0F35110508F029CFEBE3EE1203C09F
:108B0000C092FE0323CF8091FE0381111FCF80917D
:108B1000D604F801B89EE00DF11D1124E752FB4F79
:108B2000E0820F5F1F4F12CF0F9476024B015C0162
:108B300040917103509172036091730370917403BB
:108B4000411551056105710539F180912708909112
:108B50002808A0912908B0912A08840F951FA61F04
:108B6000B71F95018401081B190B2A0B3B0B37FD1E
:108B700013C00F943811609120097091210985E686
:108B80009AE00F9426118AE0ACDB40E060E070E0F0
:108B900080E090E00F94C9144091010250910202CC
:108BA0006091030270910402411551056105710540
:108BB00009F453C09091A80B8091A90B981759F014
:108BC0000F947602609327087093280880932908F1
:108BD00090932A0842C080918F0E81113CC0F11001
:108BE0003AC08091270890912808A0912908B09157
:108BF0002A08840F951FA61FB71FA5019401281BE3
:108C0000390B4A0B5B0B57FD26C080911304811171
:108C100024C081E0809313045F9A809108018095BD
:108C20008270809306018091D1088E7F8093D10855
:108C30008A9A8091D1088D7F8093D1088091080114
:108C400080958170809306018091D1088B7F8093FD
:108C5000D108E5D902C010921304809111049091BB
:108C60001204909902C0019604C0181619062CF43B
:108C700001979093120480931104809111049091B4
:108C800012048E3E92406CF00F94381182E49AE008
:108C90000F94DF1040E060E070E080E090E00F941F
:108CA000C9140F94760200910504109106042091D6
:108CB0000704309108046B017C01C01AD10AE20A52
:108CC000F30AF7FC4EC08B019C010C53164F2F4F3B
:108CD0003F4F00930504109306042093070430933C
:108CE00008044F9B0BC07A9B09C02091060120FF0E
:108CF00005C020912608222309F4E2C160930104F3
:108D0000709302048093030490930404009101047F
:108D100010910204209103043091040401151105FF
:108D20002105310571F0DC01CB01801B910BA20BF9
:108D3000B30B80529E44A109B109B7FF02C090E86D
:108D400001C090E0909300048091080191118095FA
:108D50008071809306016091000470E082E40F94BA
:108D600077018091650890916608A0916708B0919D
:108D700068080097A105B10591F085017401E81A12
:108D8000F90A0A0B1B0BD801C701885E9340A109A1
:108D9000B109B7FD04C08091410281119AC180914F
:108DA0000D0490910E04A0910F04B0911004950150
:108DB0008401081B190B2A0B3B0B37FD25C1909131
:108DC000A80B8091A90B981751F0E091A90B1CE416
:108DD000E19FF0011124E95FFF4E608102C06091C4
:108DE000DA07662311F070E002C060E070E089E00D
:108DF0000F94770180911808882309F4F8C0E09057
:108E00002802F090290200912A0210912B02609111
:108E10003308709134086E5F7F4F072E000C880B6B
:108E2000990B0F94072A9701A8010F94012A87FD37
:108E3000DEC03090A90B212C1A821B821C828091EB
:108E4000A80B831509F467C0832D90E02CE4289FBC
:108E5000F001299FF00D1124E054F04F4589568907
:108E60006789708D452B462B472B89F4418D528D98
:108E7000638D748D452B462B472B49F4458D568DBC
:108E8000678D70A1452B462B472B09F43FC04CE45E
:108E9000489F9001499F300D1124C9018054904F83
:108EA0006C01FC0161817281838194810F94E532B0
:108EB0002B013C01F60161A172A183A194A10F9441
:108EC000052A6D837E838F839887F60165A176A13D
:108ED00087A190A50F94052A9B01AC016D817E812D
:108EE0008F8198850F945531A30192010F94662AC2
:108EF0003B016C01222D3A814B815C810F949F32A2
:108F0000181624F4262C7A82CB82DC8281E0830D31
:108F10008F70382E94CF20912C0230912D024091E9
:108F20002E0250912F02622D7A818B819C810F94A9
:108F3000662A9701A8010F9479303B016C012090BB
:108F400024023090250240902602509027029B0177
:108F5000AC01B701C8010F949F3218166CF0910153
:108F6000A201B301C6010F949F3218161CF47101BF
:108F7000820102C0730186014090090450900A04E6
:108F800060900B0470900C049701A801C301B2011A
:108F90000F949F321816C4F420E037ED43EA5CE3E7
:108FA000B701C8010F94662A6B017C0128E431EEF9
:108FB0004AE75FE3C301B2010F94662AA701960155
:108FC0000F9479307B018C01C701D801809309048B
:108FD00090930A04A0930B04B0930C04B701C8014A
:108FE0000F94BD31DC01CB0160E00E94D199F4E621
:108FF0008F0E911CA11CB11C80920D0490920E0446
:10900000A0920F04B09210040E94E4A50E94C8F739
:1090100080917003882309F473C00F947602009145
:109020006C0310916D0320916E0330916F03DC018E
:10903000CB01801B910BA20BB30BB7FD61C00F944A
:1090400076026B017C012091700330E0A8EEB3E062
:109050000F946930C60ED71EE81EF91EC0926C032D
:10906000D0926D03E0926E03F0926F0380911E091F
:109070000E94FCC98AE035D943C090E0A0E0B0E08E
:1090800004C0B695A795979587953A95D2F780FD38
:10909000D6CA85E08093A60FD2CA81E0809373047C
:1090A00080918F0E811106C085EE98E09093D804D0
:1090B0008093D7040E94B1D1C6CA1092FE0306CD98
:1090C0002091060121FF1ACE029B18CE379B16CEA7
:1090D0001DCE8FEF9FEFDC018093650890936608AB
:1090E000A0936708B093680880E1E2E7F2E0A6E8A1
:1090F000B8E001900D928A95E1F70E9469D94FCEB0
:1091000028960FB6F894DEBF0FBECDBFDF91CF918A
:109110001F910F91FF90EF90DF90CF90BF90AF9095
:109120009F908F907F906F905F904F903F902F9087
:1091300008951F920F920FB60F9211240F900FBE39
:109140000F901F9018951F920F920FB60F92112437
:109150000BB60F922F938F939F93EF93FF932091D2
:109160008206E091810681E08E0F8F779091C60094
:10917000281729F0F0E0EF57F94F9283E82FE0939A
:109180008106FF91EF919F918F912F910F900BBED0
:109190000F900FBE0F901F9018958EBD0DB407FE57
:1091A000FDCF08958FEF8EBD0DB407FEFDCF8EB5B8
:1091B0000895909164009B7F90936400982F906A2B
:1091C00096959CBD80FD03C091E0863009F490E047
:1091D0009DBD0895CF93DF93EC01CB01BA010F94AD
:1091E000072A2AE037ED43E25CE30F94662A68839E
:1091F00079838A839B83DF91CF910895CF93DF9307
:10920000EC01CB01BA010F94072A2AE037ED43E2C3
:109210005CE30F94662A688379838A839B83DF915A
:10922000CF910895CF93DF93EC01CB01BA010F9456
:10923000072A2DEC3CEC4CEC5DE30F94662A688326
:1092400079838A839B83DF91CF910895CF93DF93B6
:10925000EC01CB01BA010F94072A20E030E048EC82
:1092600051E40F94662A688379838A839B83DF9114
:10927000CF910895CF93DF93EC01CB01BA010F9406
:10928000072A688379838A839B83DF91CF9108952E
:10929000CF93DF93EC01CB01BA010F94072A6883C7
:1092A00079838A839B83DF91CF910895CF93DF9356
:1092B000EC01CB01BA010F94072A2FE632E143E813
:1092C0005AE30F94662A688379838A839B83DF91AC
:1092D000CF910895CF93DF93EC01CB01BA010F94A6
:1092E000072A0F94BD3179836883DF91CF91089568
:1092F000CF93DF93EC01CB01BA010F94072A23E34C
:1093000033E343E250E40F94662A0F94C23168833A
:10931000DF91CF910895FC0184910895FC01808133
:109320000895089580E090E00895CF93DF9300D0F2
:109330001F92CDB7DEB70F94072A2DEC3CEC4CEC16
:109340005DE30F94662A69837A838B839C83CE01C5
:1093500001960E94D68B0F900F900F900F90DF9187
:10936000CF910895CF93DF9300D01F92CDB7DEB792
:109370000F94072A20E030E048EC51E40F94662A6D
:1093800069837A838B839C83CE0101960E940BF4C0
:109390000F900F900F900F90DF91CF910895CF9382
:1093A000DF9300D01F92CDB7DEB70F94072A6983F1
:1093B0007A838B839C83CE0101960E940BF40F90DD
:1093C0000F900F900F90DF91CF910895CF93DF937F
:1093D00000D01F92CDB7DEB70F94072A2FE632E1F7
:1093E00043E85AE30F94662A69837A838B839C83CC
:1093F000CE0101960E9479FF0F900F900F900F9071
:10940000DF91CF910895CF93DF9300D01F92CDB716
:10941000DEB70F94072A2AE037ED43E25CE30F94AE
:10942000662A69837A838B839C83CE0101960E948E
:1094300009F50F900F900F900F90DF91CF91089545
:109440000F94072A0F94BD31CB010C94C9F60F94E9
:10945000072A23E333E343E250E40F94662A0F9490
:10946000C231862F0C94FFF6DF92EF92FF920F939A
:109470001F93CF93DF93EC01D62E1CAD0BAD7C0177
:1094800084E0E80EF11CE98DFA8DC7011995412F92
:10949000480F2D2D602FC7010E94ACE59BAD890FB1
:1094A0008BAF81E090E0DF91CF911F910F91FF9002
:1094B000EF90DF9008958F929F92AF92BF92CF92DC
:1094C000DF92EF92FF920F931F93CF93DF93EC0104
:1094D0008B015A018A859B858617970731F0888111
:1094E00099810E94DDE31B870A878885998501960B
:1094F000D1F1CE80DF80D5010C91002349F1E880C5
:10950000F980602FC7010E9435E4F7011189119598
:109510004501FFEF8F1A9F0AD4018D914D018823D9
:1095200049F0F7019089190F082F682FC7010E9491
:1095300035E4F2CF003241F0D70153969C91539716
:1095400051968C91890F02C0F7018089180F01C0D4
:1095500010E0C10ED11C888599858C159D0518F4E5
:1095600081E090E024C0FC801A819E81190FC880A0
:10957000D980D6015596ED91FC915697C601199563
:10958000F80E00E0D5012D915D01222341F04F2D11
:10959000612FC6010E94ACE5180F080FF3CF8E8132
:1095A0009F81800F911D9F838E8380E090E0DF91EB
:1095B000CF911F910F91FF90EF90DF90CF90BF90D0
:1095C000AF909F908F900895AF92BF92DF92EF92ED
:1095D000FF920F931F93CF93DF938C01EB01D42E57
:1095E00079018FE0481709F463C0A5E14A1791F0AB
:1095F000BAE04B137CC0EC81FD8120E030E042E01A
:1096000061E0C801199547EB5AE0BE01C8010E940C
:109610001FE56DC0AA80BB8042EA5AE0C8010E94E3
:109620001FE5F5014481440F406BBE01C8010E9453
:1096300004E541E0BE01C8010E940DE5D501169682
:109640002D913C911797EC81FD8115964C9166E028
:10965000C801199540E0BE01C8010E9416E542EA22
:109660005AE0BE01C8010E941FE5F5014481440F84
:109670004F5F406BBE01C8010E9404E541E0BE019E
:10968000C8010E940DE5D50115964C9115971696C7
:109690002D913C911797240F311DEC81FD8166E0DF
:1096A000C801199540E0BE01C8010E9416E51FC01F
:1096B00041E0C8010E9416E540E0BE01C8010E94D9
:1096C0000DE541E8BE01C8010E9404E5F7014081B3
:1096D00050E05595479555954795BE01C8010E94A4
:1096E00004E540E0BE01C8010E9416E5A6C00A805C
:1096F000DB81C02DF2E3DF1609F46FC0FD15A0F089
:1097000085E1D81609F476C0A7E1DA1609F484C019
:10971000B4E1DB1292C02D81EE81FF81CF01820F77
:10972000911D820F911D5EC0E6E4DE1609F47EC035
:10973000F7E4DF1609F47EC08BE3D8127EC0D701B0
:1097400011968C91119713969C91913029F093303A
:1097500031F4482F885004C048E0480F01C0482F1A
:1097600051E02B81281708F450E031E02A8142179C
:1097700008F430E021E0481708F020E0822F852B24
:10978000382319F4252309F458C0F701D280913009
:1097900051F030F0923049F0933051F41FEF09C08E
:1097A00010E001E007C011E004C010E00FEF02C0BC
:1097B00010E000E0D7FE04C0B701CE010E94A7E38D
:1097C000D7018C91800F8C9311968C911197810FFA
:1097D00011968C93DD0C71F730C0B701CE010E9459
:1097E000A7E32BC011928E179F07E1F7CE010E94CD
:1097F000D2E323C0CE010E94BCE38823F9F02D817F
:10980000EE81FF81CF01820F911D820F911D119278
:109810008E179F07E1F711C0F70110828A818183BB
:109820008D81815082838B81838307C08D81D70195
:109830008C9303C08981F701808381E0DF91CF9110
:109840001F910F91FF90EF90DF90BF90AF90089520
:10985000E0917C03E63010F581E08E0F80937C036D
:109860004091040F5091050F6091060F7091070F02
:1098700090917A048091770428E0E29FF00111240E
:10988000EA5EFB4F2091EA0B3091EB0B3183208392
:1098900042835383648375839683878308952F92CD
:1098A0003F924F925F926F927F928F929F92AF9270
:1098B000BF92CF92DF92EF92FF920F931F93CF93BD
:1098C000DF9300D000D0CDB7DEB71C017A83698367
:1098D0002B833C834D835E8381E080937804B8DFE3
:1098E00083E080938D023092540420925304898146
:1098F0009A8190935204809351048B819C81AD8115
:10990000BE8180934D0490934E04A0934F04B09376
:109910005004E0924904F0924A0400934B041093DF
:109920004C04E12CF12CC092040FD092050FE09270
:10993000060FF092070FB092EB0BA092EA0B9092F9
:109940004804809247048C8D8093460426960FB677
:10995000F894DEBF0FBECDBFDF91CF911F910F9165
:10996000FF90EF90DF90CF90BF90AF909F908F903F
:109970007F906F905F904F903F902F9008952F921F
:109980003F924F925F926F927F928F929F92AF928F
:10999000BF92CF92DF92EF92FF920F931F93CF93DC
:1099A000DF93CDB7DEB729970FB6F894DEBF0FBEB1
:1099B000CDBF1C017987688769011A830983EB820F
:1099C000BA01550F880B990B0F94072A4B015C01C4
:1099D00020E030E040E05FEC0F949F3218162CF04E
:1099E000812C912CA12C2FECB22EC501B4010F9427
:1099F000BD312B013C01B601DD0C880B990B0F9496
:109A0000072A4B015C0120E030E040E05FE40F9466
:109A1000012A87FD05C0812C912CA12C9FE4B92E31
:109A2000E885F98560817181072E000C880B990B00
:109A30000F94072A6B017C01C301B2010F94072A1E
:109A40009B01AC01C701B6010F9478300F94C2316D
:109A50006C837D838E839F83C501B4010F94BD31D8
:109A60007B018C01E418F50806091709FB81FF93B7
:109A700089809A8085E9A82E81E5B82ECC80DD808A
:109A8000A301920168857985C10109DF0F902996AC
:109A90000FB6F894DEBF0FBECDBFDF91CF911F91FF
:109AA0000F91FF90EF90DF90CF90BF90AF909F907D
:109AB0008F907F906F905F904F903F902F90089580
:109AC00020E040E060E070E089EE97E70C94933F7F
:109AD000E0917C03EE2389F0E150E0937C0388E081
:109AE000E89FF0011124EA5EFB4F628173812781B8
:109AF0004681808191810C94933FE2CFCF93DF9395
:109B000000D01F92CDB7DEB70F94C2310F94052A53
:109B100069837A838B839C83CE0101960E940BF428
:109B20000F900F900F900F90DF91CF9108958F922B
:109B30009F92AF92BF92CF92DF92EF92FF92CF931C
:109B40006B017C0120E030E04AE754E40F94662A80
:109B50004B015C0120E030E0A901C701B6010F9480
:109B6000012A87FD05C020E030E040EA50E404C04F
:109B700020E030E040EA50ECC501B4010F947930A8
:109B800020E030E040E251E40F9455310F94BD31B4
:109B90006B017C0197FF0AC0F094E094D094C094CC
:109BA000C11CD11CE11CF11C8DE201C08BE2809331
:109BB000590FC701B60120E137E240E050E00F94B1
:109BC00074338AE0882E912CA12CB12CCA01B901E2
:109BD000A50194010F947433605D60935A0FC7011F
:109BE000B60128EE33E040E050E00F947433CA0130
:109BF000B901A50194010F947433605D60935B0F0C
:109C0000C701B60124E630E040E050E00F94743321
:109C1000CA01B901A50194010F947433605D60938A
:109C20005C0F8EE280935D0FC701B601A501940120
:109C30000F947433C62FCA01B901A50194010F9482
:109C40007433605D60935E0FC05DC0935F0F89E504
:109C50009FE0CF91FF90EF90DF90CF90BF90AF90BB
:109C60009F908F9008950F94072A2AE037ED43E2E2
:109C70005CE30F94662A5BCFCF92DF92EF92FF9264
:109C80006B017C0120E030E0A9010F94012A87FDDF
:109C900005C020E030E040E05FE304C020E030E0B9
:109CA00040E05FEBC701B6010F9479300F94BD31EE
:109CB000CB01FF90EF90DF90CF900C94C9F60F94FA
:109CC000072ADACFAF92BF92CF92DF92EF92FF9244
:109CD0000F931F93CF93DF93EC015B018A01FB018C
:109CE000199587FD05C090E0A0E0B0E0219628C15D
:109CF000982F907E903CC9F48F7190E0A0E0B0E086
:109D00006C017D0126E0CC0CDD1CEE1CFF1C2A95AD
:109D1000D1F7CE010196F50119958F73A701960130
:109D2000282BDA01C90122960BC1982F907F903E13
:109D300029F58F70C82ED12CE12CF12C86E0CC0CAB
:109D4000DD1CEE1CFF1C8A95D1F7CE010196F501B2
:109D500019958F73C82A96E0CC0CDD1CEE1CFF1CF5
:109D60009A95D1F7CE010296F50119958F73A70147
:109D70009601282BDA01C9012396E2C0982F987F1B
:109D8000903F91F58770C82ED12CE12CF12CF6E094
:109D9000CC0CDD1CEE1CFF1CFA95D1F7CE01019610
:109DA000F50119958F73C82AA6E0CC0CDD1CEE1CBA
:109DB000FF1CAA95D1F7CE010296F50119958F7374
:109DC000C82AB6E0CC0CDD1CEE1CFF1CBA95D1F7FE
:109DD000CE010396F50119958F73A7019601282BE3
:109DE000DA01C9012496ACC0982F9C7F983F09F0F6
:109DF0003FC08370C82ED12CE12CF12C56E0CC0C46
:109E0000DD1CEE1CFF1C5A95D1F7CE010196F50121
:109E100019958F73C82A66E0CC0CDD1CEE1CFF1C64
:109E20006A95D1F7CE010296F50119958F73C82A6C
:109E300076E0CC0CDD1CEE1CFF1C7A95D1F7CE0130
:109E40000396F50119958F73C82AE6E0CC0CDD1C4A
:109E5000EE1CFF1CEA95D1F7CE010496F501199589
:109E60008F73A7019601282BDA01C901259668C0D6
:109E7000982F9E7F9C3F09F04CC08170C82ED12C3A
:109E8000E12CF12C86E0CC0CDD1CEE1CFF1C8A952D
:109E9000D1F7CE010196F50119958F73C82A96E086
:109EA000CC0CDD1CEE1CFF1C9A95D1F7CE0102965E
:109EB000F50119958F73C82A26E0CC0CDD1CEE1C29
:109EC000FF1C2A95D1F7CE010396F50119958F73E2
:109ED000C82A36E0CC0CDD1CEE1CFF1C3A95D1F7ED
:109EE000CE010496F50119958F73C82A46E0CC0C73
:109EF000DD1CEE1CFF1C4A95D1F7CE010596F5013D
:109F000019958F73A7019601282BDA01C9012696AE
:109F100017C0982F907C903841F4807C803869F489
:109F20002196CE01F5011995F8CF8E7F8D3F28F04F
:109F30002196CE01F5011995F8CF80E090E0DC0183
:109F40000115110529F0F80180839183A283B38361
:109F5000CE01DF91CF911F910F91FF90EF90DF9095
:109F6000CF90BF90AF900895EF92FF920F931F9301
:109F7000CF93DF9300D01F92CDB7DEB7062F142FFB
:109F80007C01112309F449C0AE014F5F5F4F6BE8BC
:109F900079E4C70197DE7C0169817A818B819C819C
:109FA0006115710581059105C1F16D33710581055B
:109FB0009105A1F06E3771058105910579F0115079
:109FC0006A3271058105910519F00E94B091D9CFCF
:109FD00065E470E080E090E00E94B091602F70E056
:109FE00089819A81AB81BC81CD97A105B10519F01A
:109FF00081E390E002C080E390E0680F791F072EB4
:10A00000000C880B990B0E94B091115031F0612F18
:10A0100070E0C7010E941B92181B812F0F900F90B8
:10A020000F900F90DF91CF911F910F91FF90EF90C4
:10A0300008951F93CF93DF9300D01F92CDB7DEB763
:10A0400010E0AE014F5F5F4F6EE879E43BDE49817F
:10A050005A816B817C81452B462B472B11F01F5F6A
:10A06000F0CF812F0F900F900F900F90DF91CF9135
:10A070001F9108951F93CF93DF9300D01F92CDB708
:10A08000DEB710E0AE014F5F5F4F6BE879E41ADE98
:10A0900049815A816B817C81452B462B472B11F0DE
:10A0A0001F5FF0CF812F0F900F900F900F90DF91D7
:10A0B000CF911F910895AF92BF92CF92DF92EF920E
:10A0C000FF920F931F93CF93DF935C016B01D2DF5D
:10A0D000E82EC601AEDFF12C03E110E0081B1109E8
:10A0E0000E151F0514F0C5E201C0CFE18C2F90E0E2
:10A0F000AC014E5F5F4F2091240C30E042175307B4
:10A100003CF009972091260C30E028173907DCF540
:10A11000D0E0C114D10409F441C06AE370E080E0EA
:10A1200090E00E94B0910E151F0584F4C45F8091E9
:10A13000240CC81798F12C2F30E029503109809158
:10A14000260C90E0821793071CF428C0DD2331F120
:10A15000802F880F080F000F0093270CC093280C46
:10A1600060E270E080E090E00E94B091C601DF9173
:10A17000CF911F910F91FF90EF90DF90CF90BF9004
:10A18000AF900C94CB926091890F1092270CC093E2
:10A19000280C45E1C501E8DED1E0BBCFDF91CF91CE
:10A1A0001F910F91FF90EF90DF90CF90BF90AF90F5
:10A1B00008950F931F93CF93DF93FC01EB018091E0
:10A1C000040F9091050FA091060FB091070FB7FFF4
:10A1D00008C01092040F1092050F1092060F1092F3
:10A1E000070F8091490490914A04A0914B04B091CB
:10A1F0004C044091040F5091050F6091060F70912F
:10A20000070F84179507A607B70744F48093040F38
:10A210009093050FA093060FB093070F80918D02C6
:10A220008823F9F04091040F5091050F6091060FBB
:10A230007091070F80914D0490914E04A0914F04AE
:10A24000B09150048A019B01080F191F2A1F3B1F60
:10A25000C901B8011995BC0180915304909154042F
:10A260002ADF80910A0F811108C08091460488235B
:10A27000C9F180918D028823A9F1809151049091B8
:10A2800052040097B1F00091040F1091050F209136
:10A29000060F3091070F40914D0450914E0460918C
:10A2A0004F0470915004400F511F621F731FFE0135
:10A2B0001995E0914704F0914804309741F080915E
:10A2C0004604811103C080910A0F81111995809174
:10A2D0000A0F10920A0F882329F0DF91CF911F9166
:10A2E0000F91F6CBDF91CF911F910F91089562E10D
:10A2F00079E485E999E45DCF66E279E482EB99E45B
:10A3000058CF68E479E48FEC99E453CF66E579E4BB
:10A3100086EE99E44ECF6AEE78E483E09AE449CF82
:10A320006AE379E48FE59EE444CF6AE679E480E26B
:10A330009AE43FCF68E779E487E29AE43ACF9CE079
:10A34000899F802D112491E0980F909375042CE043
:10A35000280F2093740430E02E5F3F4F4091240C6F
:10A3600050E02417350714F480E00895292F30E0D9
:10A370004091260C50E024173507B4F7662341F0CE
:10A380008E5F0E94BEFE809174048E5F0E94BEFEAE
:10A39000809174049091240C891730F32091260C3D
:10A3A00090917504291700F31092270C8093280CC4
:10A3B00081E00895CF92DF92EF92FF920F93CF93B7
:10A3C000DF93982F862F6A017901692FB8DF8823E0
:10A3D00009F447C0C701002311F04CDE01C029DE9B
:10A3E000C82F43E1481B6091890FC601BDDDCC2316
:10A3F000C1F1D82FDD0F8D0FD82FDD0F6AE370E08C
:10A4000080E090E00E94B091D73040F060E270E0D0
:10A4100080E090E00E94B091D81BF6CF8091740448
:10A420009AEFC99FC02D1124C058C093270C809368
:10A43000280C002361F06FEF7FEFC701DF91CF9110
:10A440000F91FF90EF90DF90CF900C941B92C7017B
:10A45000DF91CF910F91FF90EF90DF90CF900C9410
:10A46000CB92DF91CF910F91FF90EF90DF90CF9043
:10A4700008950F93CF93DF93982F862FEA01692FCA
:10A480005EDF882359F143E16091890FCE016CDDD5
:10A49000C82FCC0F8C0FC82FCC0FC73040F060E214
:10A4A00070E080E090E00E94B091C81BF6CF8091F0
:10A4B00074049AE79093270C8093280C602F000F68
:10A4C000770B880B990B0E94B09160E270E080E0FE
:10A4D00090E0DF91CF910F910C94B091DF91CF91EB
:10A4E0000F910895482F50E020911504022E000C82
:10A4F000330B4217530741F08093150462EE7AE064
:10A5000080EF9BE00C94DDE308951F93CF93DF93DE
:10A510001F92CDB7DEB7883791053CF08F3F91058C
:10A5200031F02CF08FEF90E002C088E790E090933C
:10A530008C0280938B02182F8091290C811105C009
:10A5400081E08093290C0E94F3DC6091F20B709102
:10A55000F30B19839E012F5F3F4F4FE080EF9BE08D
:10A560000E94D9E30F90DF91CF911F9108958091C0
:10A570008B0290918C02C9DF81E080931404EDE29C
:10A58000FBE082EE9AE09183808313821282089529
:10A5900021E02093020F6093570470935804809336
:10A5A000590490935A0420E040E060E070E080910C
:10A5B0005F04909160040C94933F6DEC7CEC8CEC08
:10A5C0009CE3E6CF6DEC7CEC8CEC9DE3E1CF60E0AE
:10A5D00070E080E89FE3DCCF60E070E080E291E42F
:10A5E000D7CFCF92DF92EF92FF92CF93C82F8330D5
:10A5F00029F467FD60911E096093FD0E0F947602A9
:10A600006B017C0124EA30E74DE75FE3609157047A
:10A61000709158048091590490915A040F94012A22
:10A6200087FD05C08AEF90E0A0E0B0E003C080E0C5
:10A6300090E0DC01C80ED91EEA1EFB1EC092FE0E81
:10A64000D092FF0EE092000FF092010FC0938802AB
:10A65000CF91FF90EF90DF90CF9008951F93CF930D
:10A66000DF9300D01F92CDB7DEB7182F80910A0F6D
:10A6700010920A0F882319F00E94EE6F5DC060915E
:10A68000040F7091050F8091060F9091070F6115CF
:10A6900071058105910561F10F94072A20915704F6
:10A6A000309158044091590450915A040F94662AED
:10A6B00020917E0230917F02409180025091810270
:10A6C0000F94793060937E0270937F0280938002B2
:10A6D00090938102612F83E084DF81E080938D027B
:10A6E0001092040F1092050F1092060F1092070F90
:10A6F00080918D02882301F11093890F20915B04D2
:10A7000030915C0440915D0450915E0460917E0242
:10A7100070917F0280918002909181020F94783035
:10A7200069837A838B839C83CE0101960E9491F486
:10A73000BC0187E690E1BFDC0F900F900F900F9067
:10A74000DF91CF911F9108958091890F87CF8FEF6F
:10A7500085CF3F924F925F926F927F928F929F929E
:10A76000AF92BF92CF92DF92EF92FF920F931F931F
:10A77000CF93DF93CDB7DEB72A970FB6F894DEBF3D
:10A780000FBECDBF9A878987362E80910A0F10920F
:10A790000A0F882319F00E94EE6FF6C08091040F13
:10A7A0009091050FA091060FB091070F8D839E83A6
:10A7B000AF83B887892B8A2B8B2B09F4A4C094E034
:10A7C000699F80011124F801EE58FD4F40805180AF
:10A7D0006280738020E030E04AE754E4C301B201B4
:10A7E0000F9478304B015C0120E030E04AE754E4FC
:10A7F000C301B2010F9479306B017C0180915F023B
:10A800008823D1F1A1E03A1639F13A16A0F0B2E06E
:10A810003B1232C080904A0290904B02A0904C02B2
:10A82000B0904D02C0905602D0905702E09058026E
:10A83000F090590221C08090420290904302A09073
:10A840004402B0904502C0904E02D0904F02E0907A
:10A850005002F090510210C0809046029090470242
:10A86000A0904802B0904902C0905202D09053028A
:10A87000E0905402F09055026D817E818F81988521
:10A880000F94072A2091570430915804409159049D
:10A8900050915A040F94662AA30192010F947930C3
:10A8A0002B013C018D819E81AF81B885A30192016E
:10A8B000B7FF16C0C501B4010F949F32181644F0BB
:10A8C000F801EE58FD4F408251826282738215C0BA
:10A8D000F801EE58FD4F80829182A282B3820DC0B2
:10A8E000C701B6010F94012A87FFEACFF801EE589D
:10A8F000FD4FC082D182E282F3826FEF832D71DE41
:10A9000081E080938D021092040F1092050F109237
:10A91000060F1092070F80918D028823A9F1A4E001
:10A920003A9EC0011124FC01EE58FD4FDC01A855F0
:10A93000B74F2D913D914D915C91608171818281E4
:10A9400093810F94793069837A838B839C832DEC78
:10A950003CEC4CEC5DE3609157047091580480919D
:10A96000590490915A040F949F3287FD05C0CE017F
:10A9700001960E9491F404C0CE0101960E9479FFD5
:10A98000BC0189859A8597DB2A960FB6F894DEBFBD
:10A990000FBECDBFDF91CF911F910F91FF90EF9030
:10A9A000DF90CF90BF90AF909F908F907F906F90EF
:10A9B0005F904F903F90089562E08AE890E1C9CEA1
:10A9C00061E081E990E1C5CE60E088E990E1C1CE27
:10A9D000CF92DF92EF92FF920F93CF93DF9361E0DC
:10A9E00081E00E948138D0917A04C0E086EAE82EA6
:10A9F00080E1F82E94ECC92E90E1D92ED1110BC034
:10AA000080917904811128C080910A0F10920A0F59
:10AA100081111DC021C0D13059F480917904813059
:10AA200089F580910A0F10920A0F811123C02AC064
:10AA3000D23009F03FC090917904923009F05CC0A7
:10AA400080910A0F10920A0F81114EC055C040D854
:10AA50008091780481118BC080918D02882311F13F
:10AA600081E090917904911180E004E024E04CEDC4
:10AA700050E116C08FEB95E50E947D7F80917804B0
:10AA8000811175C080918D02882361F081E09091E1
:10AA90007904913009F080E003E02EE342ED50E1CB
:10AAA0006C2FE7DCCF5FDF5FC53009F0A7CFC09325
:10AAB00077045DC0D33059F480917904833089F5EF
:10AAC00080910A0F10920A0F811123C02AC0D4303E
:10AAD00049F7909179049430E1F580910A0F109232
:10AAE0000A0F81112EC035C0D092D804C092D7046D
:10AAF0008091780481113BC080918D02882391F26E
:10AB000081E0923009F080E000E22EE348EC50E171
:10AB1000C7CF8BE89FE70E947D7F809178048111E9
:10AB200026C080918D02882309F4BCCF81E09091EA
:10AB30007904933009F080E003E02EE34BEB50E121
:10AB4000AFCFF092D804E092D704809178048111BD
:10AB50000EC080918D02882309F4A4CF81E0943047
:10AB600009F080E000E22EE34AEA50E199CFDF915C
:10AB7000CF910F91FF90EF90DF90CF900895BF920B
:10AB8000CF92DF92EF92FF920F931F93CF93DF93B9
:10AB900061E081E00E948138C0917A04D0E0BB245A
:10ABA000B3948BE7E82E80E1F82E9EE7C92E90E162
:10ABB000D92EC1110BC080917904811129C08091D7
:10ABC0000A0F10920A0F81111DC022C0C13059F422
:10ABD00080917904813091F580910A0F10920A0FCB
:10ABE000811124C02BC0C23009F0B5C08091790416
:10ABF000823009F0C6C080910A0F10920A0F8111AD
:10AC0000B8C0BFC00E94684D809178048111F9C01E
:10AC100080918D02882311F181E090917904911146
:10AC200080E004E024E04FE950E116C083E799E5B5
:10AC30000E947D7F809178048111E3C080918D0214
:10AC4000882361F081E090917904913009F080E0EF
:10AC500003E02EE348E950E16D2F0BDC80911E09E3
:10AC6000882399F0C43021F51092890F90917904CE
:10AC7000943081F580910A0F10920A0F882351F1C8
:10AC8000D092D804C092D70421C0C43089F4B092C5
:10AC9000890F909179049430E9F480910A0F109211
:10ACA0000A0F8823B9F0F092D804E092D7040EC0BE
:10ACB000C530F1F480917904853009F092C080911B
:10ACC0000A0F10920A0F811184C08BC08091780402
:10ACD000811197C080918D02882351F081E09430DA
:10ACE00009F080E000E22EE341E850E16D2FC1DB86
:10ACF00016E08AEF810FC11323C08093890F8091E2
:10AD000079048C130EC080910A0F10920A0F8823C9
:10AD100041F08EE599E50E947D7F80917804811154
:10AD200070C080918D02882359F081E09091790460
:10AD3000911380E003E02EE347E650E16D2F99DBAD
:10AD40001F5F1830B1F6DF5FCF5FD53009F031CF2C
:10AD50001093770456C0C33009F080CF80917904F6
:10AD6000833039F580910A0F10920A0F811119C0B2
:10AD700020C08EE699E50E947D7F80917804811144
:10AD800040C080918D02882309F468CF81E09091C2
:10AD90007904923009F080E003E02EE341E950E1CC
:10ADA0005BCF89E699E50E947D7F809178048111CF
:10ADB00028C080918D02882309F450CF81E09091C2
:10ADC0007904933009F080E003E02EE34AE850E193
:10ADD00043CF84E699E50E947D7F809178048111BC
:10ADE00010C080918D02882309F482CF81E0909178
:10ADF0007904953009F080E003E02EE342E750E16A
:10AE000075CFDF91CF911F910F91FF90EF90DF9061
:10AE1000CF90BF9008956F927F928F929F92AF9242
:10AE2000BF92CF92DF92EF92FF920F931F93CF9337
:10AE3000DF93CDB7DEB76E970FB6F894DEBF0FBEC7
:10AE4000CDBFD82E742E7093600460935F0461E0D0
:10AE500081E00E948138E0907A048CE0C82EF12CC9
:10AE600091E02EE2822E20E1922E9E012F5F3F4F35
:10AE7000590137E1632E31E0D31691F1D31628F052
:10AE800082E0D81609F457C081C0E11001C19923AE
:10AE9000D9F0809179041816BCF04091040F5091BC
:10AEA000050F6091060F7091070F4F5F5F4F6F4F57
:10AEB0007F4F4093040F5093050F6093060F7093DC
:10AEC000070F8F5F8093790480918D02882309F4A6
:10AED0007DC143E068E970E18F2D0E94D6FE76C106
:10AEE000E110D6C09923D9F0809179041816BCF0EE
:10AEF0004091040F5091050F6091060F7091070F5C
:10AF00004F5F5F4F6F4F7F4F4093040F5093050F7C
:10AF10006093060F7093070F8F5F80937904809181
:10AF20008D02882309F463C143E061E970E18F2D4C
:10AF30000E94D6FE5CC1E110ABC09923D9F080918C
:10AF400079041816BCF04091040F5091050F6091E0
:10AF5000060F7091070F4F5F5F4F6F4F7F4F40930A
:10AF6000040F5093050F6093060F7093070F8F5FC8
:10AF70008093790480918D02882309F4B0C043E066
:10AF80006AE870E18F2D0E94D6FEA9C040917E0232
:10AF900050917F02609180027091810240935B0426
:10AFA00050935C0460935D0470935E04E11027C0CD
:10AFB0009923D9F0809179041816BCF04091040FC0
:10AFC0005091050F6091060F7091070F4F5F5F4F13
:10AFD0006F4F7F4F4093040F5093050F6093060F00
:10AFE0007093070F8F5F8093790480918D0288237F
:10AFF00031F043E062E770E18F2D0E94D6FE93E0CE
:10B00000D91246C077FC02C0E72D02C0E0911E09AC
:10B010008091EB0781113CC06E9EF0011124E55D2B
:10B02000F74F20E030E0A901648175818681978126
:10B030000F9479300F94BD3120913802309139024C
:10B04000621773072CF521E0E21220C08091790489
:10B05000813061F480910A0F10920A0F882331F039
:10B060000E94684D80917804811113C180918D02F6
:10B07000882361F081E090917904913009F080E0BB
:10B0800004E024E047E550E16F2DF3D982E030C0C1
:10B0900031E0E316C1F132E0E31609F43FC083E08A
:10B0A000E81609F446C084E0E81290C08091790463
:10B0B000843009F478C080918D02882309F486C019
:10B0C00081E090917904943009F080E003E02EE370
:10B0D00049E350E16F2DCDD992E0D91288C080911B
:10B0E0008D02882321F035E0E31609F4B1C086E033
:10B0F000F394E3949CE0C90E90E025E0F212BBCEFD
:10B1000080937704C6C080917904813021F58091C5
:10B110000A0F10920A0F811118C01DC08091790486
:10B12000823081F580910A0F10920A0F811122C09E
:10B1300029C080917904833009F044C080910A0FBE
:10B1400010920A0F811136C03DC00E94684D809157
:10B15000780481119EC080918D028823B9F181E02D
:10B1600090917904913009F080E004E024E042ED10
:10B1700050E116C08CEE92E50E947D7F80917804AC
:10B18000811187C080918D02882301F181E0909127
:10B190007904923009F080E003E02EE34DE450E1C1
:10B1A0006F2D67D913C080910A0F10920A0F811179
:10B1B0002BC081CF87EE92E50E947D7F809178043D
:10B1C000811167C080918D02811113C092E0D91264
:10B1D0000EC025E0E21283CF80917904853031F5ED
:10B1E00080910A0F10920A0F811118C01FC085E0CC
:10B1F0007FCF81E090917904933009F080E003E003
:10B200002EE344E450E1CCCF82EE92E50E947D7FB4
:10B2100080917804882309F44ECF3BC08DED92E5F0
:10B220000E947D7F80917804811133C080918D02CE
:10B23000882309F45CCF81E090917904953009F07E
:10B2400080E003E02EE348E350E16F2D12D947CFB1
:10B250001092270CC092280C8E010B5E1F4F23E02A
:10B2600041E06DEC7CEC8CEC9CE30F948B259F9380
:10B270008F939F928F92BF92AF920F949B29C5019B
:10B280000E94CB920F900F900F900F900F900F9005
:10B290002ECF6E960FB6F894DEBF0FBECDBFDF91F6
:10B2A000CF911F910F91FF90EF90DF90CF90BF90C3
:10B2B000AF909F908F907F906F9008954091890FED
:10B2C00064EA73E583E0A7CD4FEF67EA73E583E0B7
:10B2D000A2CD4FEF6CED74E582E09DCD4FEF60EEB7
:10B2E00074E581E098CD4FEF64EE74E580E093CD96
:10B2F0006F927F928F929F92AF92BF92CF92DF9286
:10B30000EF92FF920F931F93CF93DF93CDB7DEB7EA
:10B31000EB970FB6F894DEBF0FBECDBF8091030F41
:10B32000882349F18FE69BE00F9432048BE1EFE62E
:10B33000FBE0DE01919601900D928A95E1F700E025
:10B3400010E04EE65FE0BE016F5F7F4FCE01819659
:10B350000F945C1918163CF4CE0101960F946816F0
:10B36000080F111DEECFCE0181960F943704109374
:10B3700056040093550461E081E00E948138C0903A
:10B380007A04D12C82EF882E8FE6982E95E2692ED2
:10B3900090E1792EC1101FC08091790481110CC0F9
:10B3A00080910A0F10920A0F882331F00E94684D95
:10B3B00080917804811130C180918D02882359F0E9
:10B3C00081E090917904911180E004E024E049E269
:10B3D00050E16D2D4ED88091470D85FD10C083FF43
:10B3E0000EC081E0C8122CC080917904813079F4BC
:10B3F00080910A0F10920A0F811103C008C011E05A
:10B4000020C00E94F26F80917804811105C1809163
:10B410008D02882309F486C09F928F927F926F924B
:10B42000DF9281E090917904913009F080E08F9370
:10B430000E9417370F900F900F900F900F900F9062
:10B4400012E080918D02882309F46DC001E0010FA4
:10B45000A12CB12C1FEF100FE0905504F090560472
:10B46000AE14BF0408F05FC0C11257C081E0E81AF3
:10B47000F108EA18FB088FE69BE00F9432048BE199
:10B48000EFE6FBE0DE01919601900D928A95E1F7DF
:10B49000F12C4EE65FE0BE016F5F7F4FCE018196DB
:10B4A0000F945C19181694F4CE0101960F94681647
:10B4B000882379F3EF1008C0BE016F5F7F4F81E6EC
:10B4C0009FE00F948F1602C0F394E3CFCE018196D4
:10B4D0000F9437048091470D9091790484FF09C03F
:10B4E000911310C080910A0F10920A0F811123C08E
:10B4F00009C0911385C080910A0F10920A0F811123
:10B5000077C07EC080918D02882339F081E091134D
:10B5100080E041E06D2D0E944CFF8FEFA81AB80A21
:10B520000F5F98CF12E0D394C39485E0D81232CF46
:10B530001093770471C019821C828091720B811163
:10B5400003C06AE87BE002C06FE67BE021E041E6F1
:10B550005FE0CE0101960F945508882319F18BE125
:10B56000FE013196AFE6BBE001900D928A95E1F7BE
:10B570008091470D8F7D8093470DA0913D0DAA309E
:10B58000E0F481E08A0F80933D0D8BE18A9FD0012A
:10B590001124A15DB34FEFE6FBE001900D928A9577
:10B5A000E1F70BC00F943B1161E67FE08FE090E183
:10B5B0000F9426118AE00E947141CE0101960F94EA
:10B5C000370410927A0482E090E0A0E0B0E080932B
:10B5D000040F9093050FA093060FB093070F81E01F
:10B5E000809378041092080F83E080938D0214C03A
:10B5F00080E590E70E947D7F8091780481110CC0E6
:10B6000080918D02882309F488CF81E0909179049C
:10B61000911380E040E07ECFEB960FB6F894DEBF4A
:10B620000FBECDBFDF91CF911F910F91FF90EF9093
:10B63000DF90CF90BF90AF909F908F907F906F9052
:10B6400008951F93CF93DF93DC01EA01122F1616A2
:10B65000170684F4FC01EE0FFF1FE256FD4F208118
:10B660003181C9010F97681779070CF4CB016A2F54
:10B670000E94D199D7FD0EC0CC38D1051CF09CE8B2
:10B6800080E002C09C2F8D2F909324088093250882
:10B690000E945CC61093DA07DF91CF911F910C9442
:10B6A000604D0F931F93CF93DF938091890F90E0AC
:10B6B000EC01CC0FDD1FCC0FDD1F8E01005D1D4F97
:10B6C000880F991FFC01EA59FD4F60817181072E97
:10B6D000000C880B990B0F94072A2AE037ED43E200
:10B6E0005CE30F94662ACF53D74F288139814A8172
:10B6F0005B810F94662AF801608371838283938350
:10B70000DF91CF911F910F9108950F931F93CF93C6
:10B71000DF9380911E0990E0EC01CC0FDD1FCC0F70
:10B72000DD1F8E01005D1D4F880F991FFC01EA5936
:10B73000FD4F60817181072E000C880B990B0F94CF
:10B74000072A2AE037ED43E25CE30F94662ACF53E1
:10B75000D74F288139814A815B810F94662AF8018D
:10B760006083718382839383DF91CF911F910F91C7
:10B7700008958091890F811104C0809161048093A4
:10B78000DA0708952F923F924F925F926F927F92C5
:10B790008F929F92AF92BF92CF92DF92EF92FF92E1
:10B7A0000F931F93CF9361E081E00E948138C09195
:10B7B0007A0410E083E0282E83E1382E90ED492EA4
:10B7C00092E1592E2FEF622E21E1722E30EFA32E3F
:10B7D00031E1B32E46E4E42E42E1F42E51EE852E03
:10B7E00051E1952E61E5C62E62E1D62EC1110BC046
:10B7F00080917904811129C080910A0F10920A0F5B
:10B8000081111DC022C0C13059F48091790481306A
:10B81000C9F580910A0F10920A0F811127C032C01A
:10B82000C23009F04FC080917904823009F064C0C1
:10B8300080910A0F10920A0F811152C05DC00E94C0
:10B84000684D80917804811164C380918D028823B2
:10B8500081F181E090917904911180E004E024E08D
:10B8600041EE5BE2612F0E94395223C08FE091E1EB
:10B870009093D8048093D7040E94EE6F809178044F
:10B88000811147C380918D02882399F01F9289EF1F
:10B8900092E19F938F931F9381E09091790491306F
:10B8A000D1F58F930E9417370F900F900F900F9044
:10B8B0000F901F5FCF5F153009F098CF85E180931F
:10B8C000770427C3C33049F580917904833009F0A8
:10B8D0004CC080910A0F10920A0F81113AC045C0E6
:10B8E0008EE191E19093D8048093D7040E94EE6F8B
:10B8F0008091780481110DC380918D028823C9F253
:10B900001F928FEE92E19F938F931F9381E090910E
:10B910007904923031F280E0C4CFC43061F4809178
:10B920007904843009F04CC080910A0F10920A0FFC
:10B9300081113AC045C0C53049F580917904853000
:10B9400009F06AC080910A0F10920A0F811158C045
:10B9500063C08DE291E19093D8048093D7040E9454
:10B96000EE6F809178048111D4C280918D0288237A
:10B9700009F49FCF1F9285EE92E19F938F931F93BF
:10B9800081E090917904933031F68BCFC63051F538
:10B9900080917904863009F06BC080910A0F109273
:10B9A0000A0F811159C064C08CE391E19093D804CF
:10B9B0008093D7040E94EE6F809178048111A9C210
:10B9C00080918D02882309F474CF1F928BED92E150
:10B9D0009F938F931F9381E090917904943009F0A5
:10B9E0009ACF5FCFC73051F580917904873009F045
:10B9F0006BC080910A0F10920A0F811159C064C068
:10BA00008BE491E19093D8048093D7040E94EE6F69
:10BA10008091780481117DC280918D02882309F480
:10BA200048CF1F9286EC92E19F938F931F9381E002
:10BA300090917904953009F06ECF33CFC83051F52D
:10BA400080917904883009F06BC080910A0F1092C0
:10BA50000A0F811159C064C08AE591E19093D8041E
:10BA60008093D7040E94EE6F80917804811151C2B7
:10BA700080918D02882309F41CCF1F9281EB92E103
:10BA80009F938F931F9381E090917904963009F0F2
:10BA900042CF07CFC93051F580917904893009F040
:10BAA0006BC080910A0F10920A0F811159C064C0B7
:10BAB00089E691E19093D8048093D7040E94EE6FB9
:10BAC00080917804811125C280918D02882309F428
:10BAD000F0CE1F9287EA92E19F938F931F9381E0AC
:10BAE00090917904973009F016CFDBCECA3051F52A
:10BAF000809179048A3009F06BC080910A0F10920E
:10BB00000A0F811159C064C088E791E19093D8046D
:10BB10008093D7040E94EE6F809178048111F9C15F
:10BB200080918D02882309F4C4CE1F928DE992E1A1
:10BB30009F938F931F9381E090917904983009F03F
:10BB4000EACEAFCECB3051F5809179048B3009F03D
:10BB50006BC080910A0F10920A0F811159C064C006
:10BB600087E891E19093D8048093D7040E94EE6F08
:10BB7000809178048111CDC180918D02882309F4D0
:10BB800098CE1F9283E992E19F938F931F9381E058
:10BB900090917904993009F0BECE83CECC3051F526
:10BBA000809179048C3009F06BC080910A0F10925B
:10BBB0000A0F811159C064C086E991E19093D804BD
:10BBC0008093D7040E94EE6F809178048111A1C107
:10BBD00080918D02882309F46CCE1F928DE792E14B
:10BBE0009F938F931F9381E0909179049A3009F08D
:10BBF00092CE57CECD3051F5809179048D3009F039
:10BC00006BC080910A0F10920A0F811159C064C055
:10BC100085EA91E19093D8048093D7040E94EE6F57
:10BC200080917804811175C180918D02882309F477
:10BC300040CE1F9282E792E19F938F931F9381E002
:10BC4000909179049B3009F066CE2BCECE3051F521
:10BC5000809179048E3009F06BC080910A0F1092A8
:10BC60000A0F811159C064C084EB91E19093D8040C
:10BC70008093D7040E94EE6F80917804811149C1AE
:10BC800080918D02882309F414CE1F9287E692E1F9
:10BC90009F938F931F9381E0909179049C3009F0DA
:10BCA0003ACEFFCDCF3051F5809179048F3009F035
:10BCB00067C080910A0F10920A0F811157C060C0AF
:10BCC00083EC91E19093D8048093D7040E94EE6FA7
:10BCD0008091780481111DC180918D02882309F41F
:10BCE000E8CD1F928CE592E19F938F931F9381E0A3
:10BCF000909179049D3009F00ECED3CDC03141F53D
:10BD000080917904803109F063C080910A0F10920C
:10BD10000A0F811153C05CC082ED91E19093D80469
:10BD20008093D7040E94EE6F809178048111F1C056
:10BD300080918D02882309F4BCCD1F92DF92CF92AF
:10BD40001F9381E0909179049E3009F0E4CDA9CD54
:10BD5000C13131F580917904813109F063C080915E
:10BD60000A0F10920A0F811153C05CC09092D80440
:10BD70008092D7040E94EE6F809178048111C9C02F
:10BD800080918D02882309F494CD1F92FF92EF9247
:10BD90001F9381E0909179049F3009F0BCCD81CD53
:10BDA000C23141F580917904823109F066C08091F9
:10BDB0000A0F10920A0F811154C05FC0B092D804CC
:10BDC000A092D7040E94EE6F809178048111A1C0E7
:10BDD00080918D02882309F46CCD1F928BE392E150
:10BDE0009F938F931F9381E090917904903109F094
:10BDF00092CD57CDC33131F580917904833109F06B
:10BE00005AC080910A0F10920A0F811148C053C086
:10BE10007092D8046092D7040E94EE6F80917804EB
:10BE2000811177C080918D02882309F442CD1F9241
:10BE30005F924F921F9381E090917904913109F0C4
:10BE40006ACD2FCDC43109F034CD8091790484318D
:10BE500009F04FC080910A0F10920A0F81113DC066
:10BE600048C08EE092E19093D8048093D7040E945A
:10BE7000EE6F8091780481114CC080918D028823EF
:10BE800009F417CD1F9288E892E19F938F931F9337
:10BE900081E090917904923109F03DCD02CD8DE1A0
:10BEA00092E19093D8048093D7040E94EE6F809122
:10BEB000780481112EC080918D02882309F4F9CC79
:10BEC0001F928BEB92E19F938F931F9381E0909150
:10BED0007904933109F01FCDE4CC8CE292E1909388
:10BEE000D8048093D7040E94EE6F8091780481116A
:10BEF00010C080918D02882309F4DBCC1F923F9201
:10BF00002F921F9381E090917904943109F003CD31
:10BF1000C8CCCF911F910F91FF90EF90DF90CF9001
:10BF2000BF90AF909F908F907F906F905F904F9059
:10BF30003F902F9008958F929F92AF92BF92CF9291
:10BF4000DF92EF92FF920F931F93CF93DF9361E005
:10BF500081E00E948138C0917A04D0E0C1110BC009
:10BF60008091790481111BC080910A0F10920A0FF1
:10BF700081110FC014C0C13011F580917904813056
:10BF800009F07AC180910A0F10920A0F811163C1E2
:10BF900073C10E94684D80917804811187C180919E
:10BFA0008D02882361F081E090917904911180E005
:10BFB00004E024E04AE051E16D2F0E94395233E35E
:10BFC000A32E38E0B32E4EE9842E42E0942E52E0A8
:10BFD000D52E6EEFC62ECC0ECD1137C0C092890F74
:10BFE000809179048C131BC080910A0F10920A0F64
:10BFF0008823A9F00F94D900F401208131812F50BA
:10C000003109E12C03E611E640E050E0B5018BEF89
:10C0100090E10E94BF4C80917804811147C18091CA
:10C020008D02882391F011E0809179048D1110E048
:10C03000F501808191810E94C9F600E09C014BEFDF
:10C0400050E16D2F812F0E94DA51FD2CDD24D39415
:10C05000DF0CF7E1AF0EB11C82E0880E911CE4E02A
:10C06000DE12BACFC430A9F5809179048430C9F4C6
:10C0700080910A0F10920A0F882399F00F94D9002B
:10C08000E12C0CE516EC2CE830E040E050E064E2F6
:10C0900078E087EF90E10E94BF4C80917804811195
:10C0A00005C180918D028823A1F011E0809179046F
:10C0B000843009F010E080912408909125080E94B6
:10C0C000C9F600E09C0147EF50E16D2F812F0E94DF
:10C0D000DA518091DA078093610482E08F0D8C132E
:10C0E0002FC01092890F809179048C1314C0809115
:10C0F0000A0F10920A0F882371F00F94D90049EBB0
:10C100005BE561E674E08DEE90E10F940E008091A6
:10C1100078048111CBC080918D02882389F011E0D1
:10C12000809179048C1310E0809161040E94FFF6E5
:10C1300000E09C014DEE50E16D2F812F0E94DA51FD
:10C1400083E08F0D8C133CC0809179048C131CC04C
:10C1500080910A0F10920A0F8823B1F060911E0996
:10C1600070E0660F771F6A597D4FE12C05E81BE5EB
:10C1700027EE33E04AE050E088EE90E10E94BF4CA9
:10C1800080917804811192C080918D028823C1F042
:10C1900011E0809179048C1310E0E0911E09F0E029
:10C1A000EE0FFF1FEA59FD4F808191810E94C9F671
:10C1B00000E09C0148EE50E16D2F812F0E94DA5182
:10C1C000F4E0FF0E96E6C92E92E0D92EB12CCF11E5
:10C1D00032C0B092890F809179048C1316C080917F
:10C1E0000A0F10920A0F882381F0E12C01E51BE56C
:10C1F00027EE33E04AE050E0B60181EE90E10E9484
:10C20000BF4C80917804811151C080918D028823A8
:10C2100091F011E0809179048F1110E0F601808196
:10C2200091810E94C9F600E09C0141EE50E16D2F22
:10C23000812F0E94DA51F394B394F2E0CF0ED11C17
:10C2400082E0B812C4CFDF5FCF5FD53009F086CE71
:10C25000F09277042BC0E12C00E010E027EE33E0F1
:10C260004AE050E064E672E084E091E10E94BF4C55
:10C270008091780481111AC080918D02882309F47D
:10C280009ECE11E080917904813009F010E0809118
:10C290006402909165020E94C9F600E09C0144E0AE
:10C2A00051E16D2F812F0E94DA5189CEDF91CF911C
:10C2B0001F910F91FF90EF90DF90CF90BF90AF90C4
:10C2C0009F908F9008958091890F0C9471CF0C945A
:10C2D000DDC50C94DDC50C94DDC50C94DDC5EF9275
:10C2E000FF920F931F93CF93DF9300D01F92CDB790
:10C2F000DEB761E081E00E948138F0907A0410E0BE
:10C30000F1100BC08091790481112BC080910A0F2C
:10C3100010920A0F81111FC024C081E0F8120CC0D6
:10C3200080917904813009F03CC080910A0F10920D
:10C330000A0F811128C035C082E0F8125DC08091DB
:10C340007904823009F084C080910A0F10920A0F9C
:10C35000811170C07DC00E94684D80917804811168
:10C36000F5C080918D02882309F43EC081E0909150
:10C370007904911180E004E024E046EB53E1612F61
:10C380000E94395231C00F94D90047E651E667EE5A
:10C3900078E08CEA93E10F94302480917804811145
:10C3A000D5C080918D028823F9F0EE24E39480912A
:10C3B0007904813009F0E12C8091E7089091E80838
:10C3C000A091E908B091EA0889839A83AB83BC8382
:10C3D000CE0101960E94D68B00E09C014CEA53E10D
:10C3E000612F8E2D0E94DA511F5FF394153009F0F2
:10C3F00087CF10937704AAC083E0F8120CC0809115
:10C400007904833009F052C080910A0F10920A0F0C
:10C4100081113EC04BC084E0F812E6CF80917904D0
:10C42000843009F072C080910A0F10920A0F8111B6
:10C430005EC06BC00F94D9004DE651E66BEE78E01C
:10C4400082EA93E10F9430248091780481117EC0B8
:10C4500080918D02882341F2EE24E3948091790447
:10C46000823009F0E12C8091EB089091EC08A091CA
:10C47000ED08B091EE0889839A83AB83BC83CE012B
:10C4800001960E94D68B00E09C0142EA53E1A8CFBE
:10C490000F94D9004BE651E66FEE78E088E993E11E
:10C4A0000F94302480917804811150C080918D02C6
:10C4B000882309F499CFEE24E394809179048330A2
:10C4C00009F0E12C8091EF089091F008A091F1081B
:10C4D000B091F20889839A83AB83BC83CE01019625
:10C4E0000E94D68B00E09C0148E953E179CF0F947C
:10C4F000D90049E651E663EF78E08EE893E10F94C6
:10C50000302480917804811121C080918D0288238C
:10C5100009F46ACFEE24E39480917904843009F021
:10C52000E12C8091F3089091F408A091F508B09166
:10C53000F60889839A83AB83BC83CE0101960E945F
:10C54000D68B00E09C014EE853E14ACF0F900F904C
:10C550000F900F90DF91CF911F910F91FF90EF906F
:10C560000895CF92DF92EF92FF920F931F93CF9394
:10C57000DF9361E081E00E948138D0917A04C0E0CD
:10C58000D1110BC08091790481112AC080910A0FCA
:10C5900010920A0F81111EC023C0D13061F4809126
:10C5A0007904813009F043C080910A0F10920A0F7C
:10C5B000811128C03CC0D23009F05DC0809179045F
:10C5C000823009F089C080910A0F10920A0F811100
:10C5D0006EC082C00E94684D809178048111F7C0BE
:10C5E00080918D02882309F43EC081E09091790406
:10C5F000911180E004E024E046EB53E16C2F0E94AF
:10C60000395231C00F94D900E12C10E8F12E07E720
:10C6100014E420E030E040E85FE36AEB77E086E88E
:10C6200093E10F944F00809178048111D0C08091E4
:10C630008D028823C1F011E080917904813009F0E6
:10C6400010E06091BA077091BB078091BC07909190
:10C65000BD070E943C4E00E09C0146E853E16C2F70
:10C66000812F0E94DA51CF5FDF5FC53009F088CF9C
:10C67000C0937704ACC0D33061F4809179048330E7
:10C6800009F05AC080910A0F10920A0F81113DC023
:10C6900053C0D43041F780917904843009F07DC0D3
:10C6A00080910A0F10920A0F811160C076C00F941A
:10C6B000D900E12C10E8F12E07E714E420E030E087
:10C6C00040E85FE36EEB77E08EE793E10F944F0075
:10C6D0008091780481117BC080918D02882319F2AA
:10C6E00011E080917904823009F010E06091BE077A
:10C6F0007091BF078091C0079091C1070E943C4E86
:10C7000000E09C014EE753E1AACF0F94D900C12C61
:10C71000D12CE12C10E8F12E07E714E42DEC3CECD1
:10C720004CEC5DE362EC77E086E793E10F947624CE
:10C730008091780481114BC080918D02882309F487
:10C7400092CF11E080917904833009F010E060917C
:10C75000C2077091C3078091C4079091C5070E94DA
:10C76000974D00E09C0146E753E179CF0F94D90043
:10C77000C12CD12CE12C10E8F12E07E714E42DECAC
:10C780003CEC4CEC5DE366EC77E08EE693E10F94D5
:10C7900076248091780481111AC080918D028823BB
:10C7A00009F461CF11E080917904843009F010E040
:10C7B0006091C6077091C7078091C8079091C9071B
:10C7C0000E94974D00E09C014EE653E148CFDF9177
:10C7D000CF911F910F91FF90EF90DF90CF90089530
:10C7E000EF92FF920F931F93CF93DF9361E081E06D
:10C7F0000E948138D0917A04C0E0D1110BC08091A1
:10C80000790481112AC080910A0F10920A0F8111B8
:10C810001EC023C0D13061F480917904813009F0C9
:10C8200043C080910A0F10920A0F811128C03CC0AA
:10C83000D23009F05EC080917904823009F08AC05C
:10C8400080910A0F10920A0F81116FC083C00E945D
:10C85000684D8091780481116EC180918D0288238A
:10C8600009F43EC081E090917904911180E004E0E8
:10C8700024E046EB53E16C2F0E94395231C00F94F3
:10C88000D900E12C10ECF12E09E714E420E030E0AF
:10C8900040E85FE367EF78E082E393E10F944F00B5
:10C8A00080917804811147C180918D028823C1F065
:10C8B00011E080917904813009F010E06091F7086F
:10C8C0007091F8088091F9089091FA080E943C4E06
:10C8D00000E09C0142E353E16C2F812F0E94DA516A
:10C8E000CF5FDF5FC53009F088CF87E080937704A2
:10C8F00022C1D33061F480917904833009F067C09C
:10C9000080910A0F10920A0F81114CC060C0D43080
:10C91000D9F580917904843009F097C080910A0F8D
:10C9200010920A0F81117CC090C00F94D900E12CA5
:10C9300010ECF12E09E714E420E030E040E85FE37A
:10C940006BEF78E08BE293E10F944F0080917804D5
:10C950008111F1C080918D02882309F4C1CF11E0CB
:10C9600080917904823009F010E06091FB087091A9
:10C97000FC088091FD089091FE080E943C4E00E06A
:10C980009C014BE253E1A8CFD530D9F580917904D1
:10C99000853009F088C080910A0F10920A0F81112A
:10C9A0006EC081C00F94D900E12C10ECF12E09E784
:10C9B00014E420E030E040E85FE36FEF78E084E2E9
:10C9C00093E10F944F00809178048111B4C080915D
:10C9D0008D02882309F484CF11E08091790483309B
:10C9E00009F010E06091FF08709100098091010941
:10C9F000909102090E943C4E00E09C0144E253E108
:10CA00006BCFD63009F06CCF80917904863009F075
:10CA100078C080910A0F10920A0F81115EC071C018
:10CA20000F94D900E12C10ECF12E09E714E420E07A
:10CA300030E040E85FE363E079E08DE193E10F945B
:10CA40004F0080917804811176C080918D028823F7
:10CA500009F446CF11E080917904843009F010E0A8
:10CA6000609103097091040980910509909106096C
:10CA70000E943C4E00E09C014DE153E12DCF0F940C
:10CA8000D900E12C10ECF12E09E714E420E030E0AD
:10CA9000A90163E179E088E193E10F944F0080916F
:10CAA0007804811148C080918D02882309F418CF41
:10CAB00011E080917904853009F010E0609113094C
:10CAC0007091140980911509909116090E943C4EAD
:10CAD00000E09C0148E153E1FFCE0F94D900E12C26
:10CAE00010ECF12E09E714E420E030E0A90167E141
:10CAF00079E08EE093E10F944F00809178048111EA
:10CB00001AC080918D02882309F4EACE11E0809149
:10CB10007904863009F010E06091170970911809C6
:10CB20008091190990911A090E943C4E00E09C01E5
:10CB30004EE053E1D1CEDF91CF911F910F91FF9045
:10CB4000EF9008950C9496C50C9496C50C9496C5D8
:10CB50000C9496C52F923F924F925F926F927F9264
:10CB60008F929F92AF92BF92CF92DF92EF92FF92FD
:10CB70000F931F93CF93DF9300D01F92CDB7DEB7F3
:10CB800061E081E00E94813860907A04712C61102C
:10CB900020C08091790481110CC080910A0F1092FD
:10CBA0000A0F882331F00E94684D8091780481112A
:10CBB000D4C280918D02882361F081E09091790444
:10CBC000911180E004E024E046EB53E1672D0E94E0
:10CBD000395280916904811135C0C090D708D09036
:10CBE000D808E090D908F090DA088091DB0890919D
:10CBF000DC08A091DD08B091DE088C159D05AE051E
:10CC0000BF0510F4D701C601C090D308D090D40856
:10CC1000E090D508F090D608BC01CD016C157D05DB
:10CC20008E059F0510F4C701B6010F94052A609385
:10CC3000650470936604809367049093680421E010
:10CC40002093690481E068120CC0809179048130DE
:10CC500009F07EC080910A0F10920A0F81111FC047
:10CC600077C082E068120CC080917904823009F0AC
:10CC7000DCC080910A0F10920A0F811189C0D5C0C3
:10CC800083E06812FDC080917904833009F06FC1A0
:10CC900080910A0F10920A0F811110C168C10F9480
:10CCA000D9002AE037ED43E25DE3609165047091BD
:10CCB000660480916704909168040F94662A4B0182
:10CCC0005C0120E030E040E05FE40F94012A87FD42
:10CCD00005C0812C912CA12C5FE4B52E2AE037ED04
:10CCE00043E25DE3609107097091080980910909A9
:10CCF00090910A090F94662A20E030E040E85FE353
:10CD00000F9478300F94C2311B012C01C501B4017E
:10CD10000F94BD317B018C0121E0E21AF108010979
:10CD200011091F92812C912C4CE7A42E41E5B42EC1
:10CD3000610121E030E040E050E067E079E088E622
:10CD400093E10E944F4C0F9080917804811105C2AD
:10CD500080918D02882309F48AC011E080917904C2
:10CD6000813009F010E08091070990910809A091A5
:10CD70000909B0910A0989839A83AB83BC83CE01E8
:10CD800001960E940BF400E09C0148E653E16BC061
:10CD90000F94D9008090650490906604A090670479
:10CDA000B090680420E030E040E05FE4C501B401E9
:10CDB0000F94012A87FD05C0812C912CA12C3FE402
:10CDC000B32E20E030E048EC52E460910B09709102
:10CDD0000C0980910D0990910E090F9478300F94F1
:10CDE000C2311B012C01C501B4010F94BD317B017F
:10CDF0008C0124E6E21AF108010911091F92812C25
:10CE0000912C21E8A22E21E5B22E610124E630E02A
:10CE100040E050E06BE079E08EE593E10E944F4CFA
:10CE20000F9080917804811198C180918D028823A0
:10CE3000F1F011E080917904823009F010E08091E6
:10CE40000B0990910C09A0910D09B0910E098983ED
:10CE50009A83AB83BC83CE0101960E940BF400E061
:10CE60009C014EE553E1672D812F0E94DA517394A6
:10CE7000639485E078128BCE88E0809377046DC14F
:10CE800024E062120CC080917904843009F0B0C0B3
:10CE900080910A0F10920A0F811198C0A9C085E0F5
:10CEA000681285C080917904853009F0DEC08091D8
:10CEB0000A0F10920A0F8111C6C0D7C00F94D90073
:10CEC0002AE037ED43E25DE360916504709166040A
:10CED00080916704909168040F94662A4B015C016D
:10CEE00020E030E040E05FE40F94012A87FD05C0B8
:10CEF000812C912CA12C9FE4B92E2AE037ED43E23E
:10CF00005DE360910F097091100980911109909172
:10CF100012090F94662A20E030E040E85FE30F94A6
:10CF200078300F94C2311B012C01C501B4010F945C
:10CF3000BD317B018C0121E0E21AF10801091109E0
:10CF40001F92812C912C8CE7A82E81E5B82E6101CF
:10CF500021E030E040E050E06FE079E085E593E1EA
:10CF60000E944F4C0F90809178048111F6C08091FF
:10CF70008D02882309F47BCF11E0809179048330FE
:10CF800009F010E080910F0990911009A09111090A
:10CF9000B091120989839A83AB83BC83CE01019639
:10CFA0000E940BF400E09C0145E553E15CCF26E0D4
:10CFB00062123AC080917904863009F084C0809171
:10CFC0000A0F10920A0F81116CC07DC00F94D90016
:10CFD00002EA15E624E630E040E050E063ED78E058
:10CFE0008EE493E10F941825809178048111B5C0E7
:10CFF00080918D02882309F43ACF11E08091790461
:10D00000843009F010E06091D3087091D4088091C9
:10D01000D5089091D6080F94052A0E947E4D00E015
:10D020009C014EE453E11FCF87E0681220CF80912E
:10D030007904873009F075C080910A0F10920A0FA9
:10D0400081115DC06EC00F94D90008EA15E624E690
:10D0500030E040E050E067ED78E087E493E10F9442
:10D06000182580917804811178C080918D028823E1
:10D0700009F4FDCE11E080917904853009F010E0CB
:10D080006091D7087091D8088091D9089091DA08FA
:10D090000F94052A0E947E4D00E09C0147E453E175
:10D0A000E2CE0F94D90006EA15E62AE030E040E02F
:10D0B00050E06BED78E080E493E10F9418258091C7
:10D0C000780481114AC080918D02882309F4CFCE63
:10D0D00011E080917904863009F010E06091DB085E
:10D0E0007091DC088091DD089091DE080F94052A8C
:10D0F0000E947E4D00E09C0140E453E1B4CE0F94C9
:10D10000D90004EA15E624E630E040E050E06FED97
:10D1100078E089E393E10F941825809178048111D8
:10D120001CC080918D02882309F4A1CE11E080916A
:10D130007904873009F010E06091DF087091E00811
:10D140008091E1089091E2080F94052A0E947E4D9B
:10D1500000E09C0149E353E186CE0F900F900F90C1
:10D160000F90DF91CF911F910F91FF90EF90DF9083
:10D17000CF90BF90AF909F908F907F906F905F9077
:10D180004F903F902F90089580918B0290918C0248
:10D190000C948552EF92FF920F931F93CF93DF93DE
:10D1A000CDB7DEB72B970FB6F894DEBF0FBECDBF5D
:10D1B0007C0120917104422F022E000C550B8091AE
:10D1C0007204833051F0843019F088E195E10AC08F
:10D1D00027FF06C084E295E105C08DE295E102C01B
:10D1E0008FE095E15F932F939F938F938E010F5F55
:10D1F0001F4F1F930F930F949B2960917104C701D8
:10D200000E94D199C8010E9409380F900F900F9089
:10D210000F900F900F902B960FB6F894DEBF0FBEB5
:10D22000CDBFDF91CF911F910F91FF90EF900895A7
:10D23000E091710487E1E802F0011124E55DF74F08
:10D2400080859185A7CFDF92EF92FF920F931F9376
:10D25000CF93DF9361E081E00E948138D0907A041F
:10D26000C0E08D2D8C0F59F48091790481111AC082
:10D2700080910A0F10920A0F81110EC013C08130E5
:10D2800009F5809179048130A9F580910A0F1092F7
:10D290000A0F81111EC02EC00E94684D8091780433
:10D2A000811145C080918D02882361F081E09091C9
:10D2B0007904911180E004E024E042E654E16C2F0F
:10D2C0000E943952CF5FC53061F682E080937704C7
:10D2D0002EC0E12CF12C00E211E420E030E0A901A5
:10D2E00062E878E085E494E10F944F00809178043F
:10D2F00081111DC080918D02882321F3D1E080919E
:10D300007904813009F0D0E060918208709183083F
:10D3100080918408909185080E943C4E00E09C0119
:10D3200045E454E16C2F8D2F0E94DA51CBCFDF9171
:10D33000CF911F910F91FF90EF90DF9008952F9262
:10D340003F924F925F926F927F928F929F92AF9295
:10D35000BF92CF92DF92EF92FF920F931F93CF93E2
:10D36000DF9361E081E00E948138F0907A04D0E0A0
:10D37000222423948EE7482E88E3582E9FE8C92E56
:10D3800094E1D92E2EE7A22E24E1B22E3BE7832E84
:10D3900038E3932E40E7642E44E1742EF1100BC065
:10D3A0008091790481111CC080910A0F10920A0F9C
:10D3B000811110C015C081E0F81222C0809179045B
:10D3C000813009F0A1C180910A0F10920A0F8111DA
:10D3D00093C19AC10E94684D809178048111C2C1A5
:10D3E00080918D02882361F081E090917904911100
:10D3F00080E004E024E04AE055E16D2F0E943952BC
:10D400000E94F33F382E81110FC082E0F8120EC047
:10D4100080917904823009F08FC180910A0F1092B7
:10D420000A0F811181C188C1C2E001C0C3E0CF11E0
:10D4300022C0809179048C130EC080910A0F109243
:10D440000A0F882341F083E299E60E947D7F809154
:10D450007804811187C180918D02882361F081E079
:10D46000909179049F1180E003E02EE342EE54E1B5
:10D470006D2F0E94395281E08C0F8F1133C0809143
:10D4800079048F1118C080910A0F10920A0F882317
:10D4900091F0EE24E39404EC18E62FEF30E048E737
:10D4A00050E06BE872E085ED94E10E94BF4C809102
:10D4B0007804811157C180918D02882399F011E081
:10D4C000809179048F1110E080918B0290918C02F1
:10D4D0000E94C9F600E09C0145ED54E16D2F812FBB
:10D4E0000E94DA5182E08C0F8F112DC08091790457
:10D4F0008F1114C080910A0F10920A0F882371F0C7
:10D5000080918A02822580938A0283E080938D0233
:10D510000F94500F80917804811124C180918D0265
:10D52000882389F081E0909179049F1180E09091A7
:10D530008A02911114C120EC34E101E047EC54E17E
:10D540006D2F0E94DA5183E08C0F8F1122C08091E1
:10D5500079048F110EC080910A0F10920A0F882350
:10D5600041F082EF9CE60E947D7F809178048111DA
:10D57000F9C080918D02882361F081E09091790457
:10D580009F1180E003E02EE34FEA54E16D2F0E94EB
:10D59000395284E08C0F8F1122C0809179048F1151
:10D5A0000EC080910A0F10920A0F882341F084EF79
:10D5B0009CE60E947D7F809178048111D3C0809188
:10D5C0008D02882361F081E0909179049F1180E0C1
:10D5D00003E02EE34EE954E16D2F0E94395285E0BD
:10D5E0008C0F8F1127C0809179048F110CC080910E
:10D5F0000A0F10920A0F882331F00E947E38809122
:10D6000078048111AFC080918D02882399F05F92D8
:10D610004F92DF92CF92DF9381E0909179049F1136
:10D6200080E08F930E9417370F900F900F900F900C
:10D630000F900F9086E08C0F311056C08F1127C0CD
:10D64000809179048F110CC080910A0F10920A0FFB
:10D65000882331F00E947B3880917804811182C048
:10D6600080918D02882399F09F928F927F926F9282
:10D67000DF9381E0909179049F1180E08F930E9465
:10D6800017370F900F900F900F900F900F9017E09B
:10D690001C0F1F1127C080917904F8120EC08091D1
:10D6A0000A0F10920A0F882341F00F94230A0E9458
:10D6B000283780917804811155C080918D0288238C
:10D6C00089F01F92BF92AF92DF9381E0909179042D
:10D6D000911380E08F930E9417370F900F900F9057
:10D6E0000F900F9088E08C0FDF5FF394D53009F036
:10D6F00055CE8093770436C086EF9CE60E947D7FEE
:10D700008091780481112EC080918D02882309F4C4
:10D7100077CE81E090917904913009F080E003E0C8
:10D720002EE348EF54E169CE86E291EB0E947D7FC3
:10D7300080917804811116C080918D02882369F050
:10D7400081E090917904923009F080E003E02EE3CB
:10D750004EEE54E16D2F0E943952C3E08CCE24EC82
:10D7600034E1EBCEDF91CF911F910F91FF90EF90BD
:10D77000DF90CF90BF90AF909F908F907F906F90F1
:10D780005F904F903F902F9008955F926F927F929D
:10D790008F929F92AF92BF92CF92DF92EF92FF92C1
:10D7A0000F931F93CF93DF93C82F61E081E00E9416
:10D7B000813850907A04F12C8EE7A82E88E3B82E99
:10D7C0009FE8892E94E1992ED0E0CE01880F991F11
:10D7D0009C012356304F3901FC01EF55F04F6F018A
:10D7E000C556D04F51100BC08091790481112AC0C9
:10D7F00080910A0F10920A0F81111EC023C0F1E020
:10D800005F120BC0809179048130C1F580910A0FBD
:10D8100010920A0F811127C031C022E052124BC072
:10D8200080917904823009F074C080910A0F1092BF
:10D830000A0F81115EC06DC00E94684D809178040E
:10D840008111C0C080918D02882369F181E090919F
:10D850007904911180E004E024E042E654E16F2D68
:10D860000E94395220C040E050E0BE0188E594E1BA
:10D870000F940E00809178048111A4C080918D02D4
:10D88000882389F011E080917904813009F010E05B
:10D8900088810E94FFF600E09C0148E554E16F2D6D
:10D8A000812F0E94DA51F3945394F5E0FF129ACF3E
:10D8B000F092770487C023E052120CC08091790463
:10D8C000833009F04AC080910A0F10920A0F81112B
:10D8D00034C043C034E05312E6CF809179048430E1
:10D8E00009F056C080910A0F10920A0F81114AC0A8
:10D8F0004FC0E12C00E010E024E031E045E050E0D2
:10D90000B60181E594E10E94BF4C809178048111B9
:10D9100059C080918D02882331F211E08091790401
:10D92000823009F010E0F601808191810E94C9F6F1
:10D9300000E09C0141E554E1B2CFE12C00E010E0B1
:10D940002CE830E045E050E0B3018DE494E10E9422
:10D95000BF4C80917804811135C080918D0288235D
:10D9600009F4A1CF11E080917904833009F010E02F
:10D97000F301808191810E94C9F600E09C014DE491
:10D9800054E18DCF0E947E388091780481111AC0B5
:10D9900080918D02882309F486CFBF92AF929F9227
:10D9A0008F92FF9281E090917904943009F080E0A9
:10D9B0008F930E9417370F900F900F900F900F903A
:10D9C0000F9071CFDF91CF911F910F91FF90EF904A
:10D9D000DF90CF90BF90AF909F908F907F906F908F
:10D9E0005F90089580E0D1CE81E0CFCECF92DF92DC
:10D9F000EF92FF920F931F93CF93DF9361E081E04B
:10DA00000E948138C0917A04D0E086E2E82E84E159
:10DA1000F82E96EDC92E93E1D92EC1110BC080913D
:10DA20007904811129C080910A0F10920A0F811187
:10DA30001DC022C0C13061F480917904813009F0A9
:10DA4000EEC080910A0F10920A0F8111DEC0E7C06C
:10DA5000C23009F0CCC080917904823019F58091F0
:10DA60000A0F10920A0F811115C01CC00E94684D48
:10DA700080917804811144C180918D02882319F12D
:10DA800081E090917904911180E004E024E047E383
:10DA900054E116C080EF93E60E947D7F8091780468
:10DAA00081112EC180918D02882369F081E09091CF
:10DAB0007904923009F080E003E02EE34DE154E177
:10DAC0006D2F0E9439520E94F33F81110EC0C53064
:10DAD00071F480917904853009F0FFC080910A0FBC
:10DAE00010920A0F8111F1C0F8C015E001C016E0D4
:10DAF0001C1322C08091790481130EC080910A0FFB
:10DB000010920A0F882341F08FED98E30E947D7FE9
:10DB1000809178048111F4C080918D02882361F096
:10DB200081E0909179049C1380E003E02EE346EFBE
:10DB300053E16D2F0E94395281E0810F8C1322C076
:10DB4000809179048C130EC080910A0F10920A0FF5
:10DB5000882341F08BEF9CE30E947D7F80917804C5
:10DB60008111CEC080918D02882361F081E0909177
:10DB700079049C1380E003E02EE34DEE53E16D2F1A
:10DB80000E94395282E0810F8C1328C09091790451
:10DB90009C1316C080910A0F10920A0F882381F0FF
:10DBA00020E040E060E070E089E89EE6DF91CF9100
:10DBB0001F910F91FF90EF90DF90CF900C94933FC7
:10DBC00080918D02882351F081E09C1380E003E076
:10DBD0002EE34BED53E16D2F0E943952DF5FCF5F93
:10DBE000D53009F01ACF1D5F1093770489C0C33078
:10DBF00071F580917904833009F03FC080910A0F5C
:10DC000010920A0F811131C038C0D092D804C0924E
:10DC1000D7040E94604D80917804811171C0809179
:10DC20008D02882309F44FCF1F92FF92EF92DF936A
:10DC300081E090917904913009F080E08F930E9407
:10DC400017370F900F900F900F900F903CCFC4306C
:10DC500009F039CF80917904843039F580910A0F29
:10DC600010920A0F811119C020C08AEA95E60E941D
:10DC70007D7F80917804811143C080918D0288233B
:10DC800009F421CF81E090917904933009F080E08C
:10DC900003E02EE340E154E113CF81EB92E60E94D2
:10DCA0007D7F8091780481112BC080918D02882323
:10DCB00009F409CF81E090917904943009F080E073
:10DCC00003E02EE34BE054E1FBCE8FE691E60E94A9
:10DCD0007D7F80917804811113C080918D0288230B
:10DCE00069F081E090917904953009F080E003E0DB
:10DCF0002EE342E054E16D2F0E94395216E01CCF12
:10DD0000DF91CF911F910F91FF90EF90DF90CF9017
:10DD10000895CF92DF92EF92FF920F931F9388ECBA
:10DD2000C82E83E1D82EE12CF12C0BED13E129EE66
:10DD300036E348EA5EE66AEC73E181ED93E10E9426
:10DD400034371F910F91FF90EF90DF90CF9008959F
:10DD5000CF930F94230A0E94B880C82F882319F00C
:10DD600080E00F948E0C8C2FCF910C9473388F928F
:10DD70009F92AF92BF92CF92DF92EF92FF920F935A
:10DD80001F93CF93DF93F82EC62E80937204609377
:10DD9000710461E081E00E948138D0917A04C0E092
:10DDA00081E06C2D660F770B9B0122563D4F690178
:10DDB00094E6A92E95E1B92E2FE7822E25E1922E29
:10DDC000D11135C08823D9F0809179041816BCF0A0
:10DDD0004091040F5091050F6091060F7091070F4D
:10DDE0004F5F5F4F6F4F7F4F4093040F5093050F6E
:10DDF0006093060F7093070F8F5F80937904809173
:10DE00008D02882309F445C033E0F31649F044E05D
:10DE1000F41203C066E475E105C066E375E102C073
:10DE200066E575E143E08C2F0E94D6FE32C0D1300A
:10DE300059F4809179048130D9F480910A0F1092BD
:10DE40000A0F81110FC014C0D23061F5809179049E
:10DE5000823009F04BC080910A0F10920A0F811195
:10DE60003CC044C00E94684D809178048111A9C0D3
:10DE700080918D02882369F081E09091790491303E
:10DE800009F080E004E024E04BE855E16C2F0E94AB
:10DE90003952CF5FDF5F80E0C53009F091CFC0938A
:10DEA00077048FC0D33059F4809179048330A9F579
:10DEB00080910A0F10920A0F811126C02EC0D43013
:10DEC00041F780917904843009F05BC080910A0F9A
:10DED00010920A0F811139C054C08091A10F909106
:10DEE000A20F58D98091780481116BC080918D0266
:10DEF000882379F21F929F928F92CF9381E0909125
:10DF000079049230C1F418C08091A30F9091A40FAE
:10DF100041D980917804811154C080918D02882369
:10DF200009F4B7CF1F92BF92AF92CF9381E0909147
:10DF30007904933009F080E08F930E9417370F9097
:10DF40000F900F900F900F90A4CF0F94D900F6016F
:10DF5000208131812F5031096091710447E16403C0
:10DF6000B00111246D5C774FE12C08E119E646E918
:10DF700050E080E795E10E94BF4C809178048111C8
:10DF800020C080918D02882309F483CF11E0809115
:10DF90007904843009F010E02091710437E1230303
:10DFA000F0011124E55DF74F808591850E94C9F647
:10DFB00000E09C0140E755E16C2F812F0E94DA516F
:10DFC00068CFDF91CF911F910F91FF90EF90DF907D
:10DFD000CF90BF90AF909F908F9008951092020FB6
:10DFE0000C94684D80913D0D8823C9F08150809339
:10DFF0003D0D882359F090E001972BE1289FF00117
:10E00000299FF00D1124E15DF34F02C0EAE8FBE027
:10E010008BE1AFE6BBE001900D928A95E1F780912C
:10E020003D0D811109C08091470D80628093470D9D
:10E0300080E090E0DC0104C081E090E0A0E0B0E08E
:10E040008093040F9093050FA093060FB093070FD2
:10E0500010927A0481E08093780483E080938D02AB
:10E060000895CF92DF92EF92FF920F931F9384E86F
:10E07000C82E87E1D82EE12CF12C0EEF17E129EE06
:10E0800036E345EA58EF66E877E18BE897E10E94CE
:10E0900034371F910F91FF90EF90DF90CF9008954C
:10E0A000AF92BF92CF92DF92EF92FF920F931F93A6
:10E0B000CF93DF93CDB7DEB7ADB6BEB680916E0F0E
:10E0C000811103C061E67FE002C06EE67FE0FB01E4
:10E0D00001900020E9F7CF01861B970B01962DB721
:10E0E0003EB7281B390B0FB6F8943EBF0FBE2DBFAD
:10E0F0008DB79EB701967C0180E2EDB7FEB78183B4
:10E10000C70101960F94F23381E2C82E88E1D82E20
:10E1100003E218E129EE36E344EA50E76FE278E1E2
:10E1200086E398E10E9434370FB6F894BEBE0FBE66
:10E13000ADBEDF91CF911F910F91FF90EF90DF90D7
:10E14000CF90BF90AF90089581E69FE00E94A3E733
:10E150000E94604D0C94F2F89F92AF92BF92CF92C2
:10E16000DF92EF92FF920F931F93CF93DF9361E0C3
:10E1700081E00E948138C0917A0410E081E09AE247
:10E18000E92E96E1F92EBB24B39425E3C22E26E1B5
:10E19000D22E32E0A32E43E0942EC11128C0882352
:10E1A000D9F0809179041816BCF04091040F509179
:10E1B000050F6091060F7091070F4F5F5F4F6F4F14
:10E1C0007F4F4093040F5093050F6093060F709399
:10E1D000070F8F5F8093790480918D02882369F106
:10E1E00041E06EE376E1812F0E94D6FE26C0C13069
:10E1F00021F580917904813061F490910A0F109299
:10E200000A0F992331F0C093D208909178049111AC
:10E2100080C090918D02992381F01F92FF92EF921E
:10E220001F9391E0813009F090E09F930E9417378F
:10E230000F900F900F900F900F9080917304882390
:10E2400071F0C23071F480917904823009F046C0D7
:10E2500080910A0F10920A0F811133C03FC0D2E0A3
:10E2600001C0D3E0DC1323C0809179048D130CC06E
:10E2700090910A0F10920A0F992331F0A092D208C0
:10E2800090917804911145C090918D02992379F075
:10E290001F92DF92CF921F9391E08C1390E09F9397
:10E2A0000E9417370F900F900F900F900F901F5FE5
:10E2B000CF5F80E0153009F070CFDF5FD093770437
:10E2C00028C080918A028B2580938A0290928D02C9
:10E2D0000F94500F8091780481111BC080918D02A2
:10E2E0008823A9F081E090917904923009F080E0D0
:10E2F00090918A02911103C025E136E102C029E123
:10E3000036E101E04CE156E1612F0E94DA51D3E0A1
:10E31000CECFDF91CF911F910F91FF90EF90DF90C3
:10E32000CF90BF90AF909F9008952F923F924F92C1
:10E330005F926F927F928F929F92AF92BF92CF9295
:10E34000DF92EF92FF920F931F93CF93DF934C01D5
:10E350000F94512901968401080F191FC8010F94C9
:10E36000512901965801A80EB91EF8015080CC24FD
:10E37000C394511001C0C12CF5013080DD24D39429
:10E38000311001C0D12CC1E05110C0E060E085E047
:10E390000E94813820907A04EE24E394F12C612CC1
:10E3A000D0E02196CC0DD11DCD0DD11D57E1452ECC
:10E3B000D22CD60CC1F480918D02882339F1E091E2
:10E3C0000902E250E33040F4F0E0EE0FFF1FEE559B
:10E3D000FD4F6081718102C06EE476E143E0862DDD
:10E3E0000E94D6FE13C0511003C022E0C22E02C00C
:10E3F000CC24C394CD100FC080918D02882359F096
:10E4000041E0B401862D0E94D6FE05C0552009F4D6
:10E41000C2C0CC24C394772473947C0C552071F033
:10E42000D71009C080918D02882329F041E0B801FE
:10E43000862D0E94D6FE92E0792E7C0C332061F06E
:10E440007D1009C080918D02882329F041E0B5013B
:10E45000862D0E94D6FE7394C330D1050CF47394BC
:10E460007D106DC080918D02882309F465C042E063
:10E470006BE576E1862D0E94D6FEC0907604E09290
:10E4800075044BE04E0D409374048091240C90E091
:10E490009701235F3F4F281739070CF44DC0809137
:10E4A000260C90E0E816F9060CF046C0EEE3E09387
:10E4B000270C4093280C65E470E080E090E00E9417
:10E4C000B09161E36C0D062E000C770B880B990B55
:10E4D0000E94B09160E270E080E090E00E94B09114
:10E4E000D12C4C9CF0014D9CF00D1124E55DF74FB3
:10E4F00020E030E0A90164817581868197810F94C5
:10E5000079300F94BD31CB010E94C9F60E94CB92A5
:10E510006FE270E080E090E00E94B09122D581111E
:10E520002BC085E08C9DF0018D9DF00D1124E25FE4
:10E53000F74F8481882301F1E2E0E0938D02639438
:10E54000FCE0EF0EF11C85E0681232CF73947092FC
:10E550007704DF91CF911F910F91FF90EF90DF90A3
:10E56000CF90BF90AF909F908F907F906F905F9073
:10E570004F903F902F9008954C9CC0014D9C900D62
:10E580001124FC01E55DF74F808591850E94C9F655
:10E590000E94CB92D1CF82E0C82E3DCF86E696E195
:10E5A000C4CE83E796E1C1CE85E996E1BECE80E395
:10E5B00097E1BBCE8BEE96E1B8CE88E197E1B5CE80
:10E5C0008BE697E1B2CE8EE497E1AFCE8EEC96E18A
:10E5D000ACCE8FEA96E1A9CE6091890F84E0C7CBDB
:10E5E0006091890F83E0C3CB6091890F82E0BFCB3C
:10E5F0002F923F925F926F927F928F929F92AF92F3
:10E60000BF92CF92DF92EF92FF920F931F93CF931F
:10E61000DF9361E081E00E94813810917A04D0E0BC
:10E6200083E1682E89EF782E9CE8E92E98EFF92E89
:10E6300029E0C22E28E1D22E30EFA32E37E1B32EEF
:10E6400041EA842E47E1942E111120C08091790473
:10E6500081110CC080910A0F10920A0F882331F0AB
:10E660000E94684D809178048111EAC180918D02E9
:10E67000882361F081E090917904911180E004E0B9
:10E6800024E045E158E16D2F0E9439520E94FD3F80
:10E69000582E8091470D83FB222420F883FF04C06D
:10E6A0000E94BD40382E01C0312C552059F1113047
:10E6B00061F480917904813009F052C180910A0F90
:10E6C00010920A0F811146C14BC1123061F4809142
:10E6D0007904823009F08DC080910A0F10920A0FE0
:10E6E00081117FC086C0133009F047C08091790442
:10E6F000833009F057C180910A0F10920A0F8111DF
:10E7000049C150C10E94CB40882371F0113071F48F
:10E7100080917904813009F05BC180910A0F1092D9
:10E720000A0F81114FC154C1C1E001C0C2E0C11341
:10E7300022C0809179048C130EC080910A0F109230
:10E740000A0F882341F088EE94E50E947D7F809136
:10E750007804811175C180918D02882361F081E078
:10E7600090917904911380E003E02EE34CED57E1A2
:10E770006D2F0E943952CF5F01C0C4E0C11322C087
:10E78000809179048C130EC080910A0F10920A0FA9
:10E79000882341F084E692EF0E947D7F8091780487
:10E7A00081114EC180918D02882361F081E09091AA
:10E7B0007904911380E003E02EE340ED57E16D2FE3
:10E7C0000E94395281E08C0F811326C08091790418
:10E7D000811322C180910A0F10920A0F811114C176
:10E7E0001BC181E390E70E947D7F809178048111B5
:10E7F00027C180918D02882309F420C181E0909186
:10E800007904923009F080E003E02EE34EEF57E107
:10E810006D2F0E943952C4E082E08C0F811322C018
:10E820008091790481130EC080910A0F10920A0F13
:10E83000882341F082E395E70E947D7F80917804F0
:10E840008111FEC080918D02882361F081E090915A
:10E850007904911380E003E02EE342EB57E16D2F42
:10E860000E94395283E08C0F222009F44CC03110F1
:10E8700069C0811320C09091790491130EC08091DA
:10E880000A0F10920A0F882341F09092D8048092C8
:10E89000D704809178048111D3C080918D028823A0
:10E8A00051F081E0911380E000E22EE345EA57E168
:10E8B0006D2F0E94395284E08C0F811322C0809109
:10E8C000790481130EC080910A0F10920A0F8823D9
:10E8D00041F088E799E50E947D7F8091780481115D
:10E8E000AFC080918D02882361F081E0909179041E
:10E8F000911380E003E02EE340E957E16D2F0E9481
:10E90000395285E01EC081131BC0809179048113A8
:10E9100002C010920A0F90918D02992389F01F92E4
:10E920001F92BF92AF92DF9391E0811390E09F938B
:10E930000E9417370F900F900F900F900F900F902D
:10E9400084E08C0FDF5F1F5FD53009F07DCE8093B0
:10E95000770476C00E948CF880917804811170C091
:10E9600080918D02882309F469C0FF92EF92DF92B3
:10E97000CF92DF9381E090917904913009F080E0AB
:10E980008F930E9417370F900F900F900F900F905A
:10E990000F9054C08BE99FE50E947D7F80917804A1
:10E9A00081114EC080918D02882309F447C081E017
:10E9B00090917904933009F080E003E02EE349EF71
:10E9C00057E126CF0E9413F980917804811138C055
:10E9D00080918D028823B1F07F926F9283EE97E150
:10E9E0009F938F93DF9381E090917904913009F0A8
:10E9F00080E08F930E9417370F900F900F900F9029
:10EA00000F900F90C2E0B7CE8FE999E60E947D7F0C
:10EA100080917804811114C080918D02882309F4BB
:10EA2000FBCE81E090917904911380E003E02EE326
:10EA300042EC57E16D2F0E943952EECEC4E0C2CEB7
:10EA4000DF91CF911F910F91FF90EF90DF90CF90CA
:10EA5000BF90AF909F908F907F906F905F903F900E
:10EA60002F9008952F923F924F925F926F927F92D4
:10EA70008F929F92AF92BF92CF92DF92EF92FF92CE
:10EA80000F931F93CF93DF93CDB7DEB72C970FB6BD
:10EA9000F894DEBF0FBECDBF61E081E00E948138F7
:10EAA000E0907A04F12CCE0101965C0123ED422E18
:10EAB00025E1522E1E2D1F0D01F580917904811143
:10EAC0000CC080910A0F10920A0F882331F00E9427
:10EAD000684D809178048111C2C180918D02882394
:10EAE00061F081E090917904911180E004E024E0EC
:10EAF00040E156E16F2D0E9439520E94CB408111B6
:10EB000002C082E001C081E0809361049BE2892E13
:10EB100098E0992E340122242394C12CD12C2C2D41
:10EB2000C6013091EB07311119C060913802709124
:10EB30003902F30140855185461757077CF41211BD
:10EB400034C0C092890F8091790481131EC08091D6
:10EB50000A0F10920A0F811110C017C0121125C0A0
:10EB60002093890F20917904211302C120910A0F6B
:10EB700010920A0F2111E5C0FBC084EF92E70E94BA
:10EB80007D7F8091780481116AC180918D028823F4
:10EB900061F081E090917904911380E003E02EE32D
:10EBA0004EEF55E16F2D0E94395233243394320CCD
:10EBB000FFEFCF1ADF0A239427E1620E711C82E077
:10EBC000C816D10409F0ABCF0E94F33F8111B2C047
:10EBD0008BE2682E88E0782EC12CD12C2C2DC6011A
:10EBE0003091EB07311119C06091380270913902F0
:10EBF000F30140855185461757077CF4131134C043
:10EC0000C092890F8091790481131EC080910A0FF0
:10EC100010920A0F811110C017C0131125C0209344
:10EC2000890F209179042113D3C020910A0F1092EB
:10EC30000A0F2111B6C0CCC080EF92E70E947D7F01
:10EC40008091780481110BC180918D02882361F03D
:10EC500081E090917904911380E003E02EE34CED84
:10EC600055E16F2D0E94395281E0830DFFEFCF1ADD
:10EC7000DF0A339427E1620E711C92E0C916D104B9
:10EC800009F0ACCF782EC12CD12C2C2DC60130919F
:10EC9000EB07311119C0F40160857185409138028C
:10ECA00050913902641775077CF4171134C0C09273
:10ECB000890F8091790481131EC080910A0F1092F0
:10ECC0000A0F811110C017C0171125C02093890F9A
:10ECD000209179042113AAC020910A0F10920A0FE3
:10ECE00021118FC0A3C08CEE92E70E947D7F80919E
:10ECF00078048111B4C080918D02882361F081E095
:10ED000090917904911380E003E02EE34CEE55E1FD
:10ED10006F2D0E94395233243394370CFFEFCF1AF2
:10ED2000DF0A739427E1820E911C82E0C816D10499
:10ED300009F0ABCFF39495E0F912BCCE3092770492
:10ED40008EC09F938F93EEEBF5E1FF93EF93BF920D
:10ED5000AF920F949B29C5010E9409380F900F9024
:10ED60000F900F900F900F9080917804811177C0D1
:10ED700080918D02882309F418CF1F928EEF95E1C0
:10ED80009F938F93FF9281E090917904911380E09B
:10ED90008F930E9417370F900F900F900F900F9046
:10EDA00004CF9F938F938AEC95E19F938F93BF92AB
:10EDB000AF920F949B29C5010E9409380F900F90C4
:10EDC0000F900F900F900F9080917804811147C0A1
:10EDD00080918D02882309F447CF1F928CED95E135
:10EDE0009F938F93FF9281E090917904911380E03B
:10EDF0008F930E9417370F900F900F900F900F90E6
:10EE000033CF9F938F935F924F92BF92AF920F94A5
:10EE10009B29C5010E9409380F900F900F900F9009
:10EE20000F900F9080917804811119C080918D020C
:10EE3000882309F470CF1F928CEE95E19F938F93F6
:10EE4000FF9281E090917904911380E08F930E946A
:10EE500017370F900F900F900F900F905CCF2C965C
:10EE60000FB6F894DEBF0FBECDBFDF91CF911F91DB
:10EE70000F91FF90EF90DF90CF90BF90AF909F9059
:10EE80008F907F906F905F904F903F902F9008955C
:10EE900061116093090240937604082E000C990BCF
:10EEA000AA0BBB0B8C30910590F5FC018827EE581E
:10EEB000FF4F8F4F0D94903381ED92E71FC087ED88
:10EEC00092E71CC08AED92E719C08DED92E716C05B
:10EED00080EE92E713C083EE92E710C086EE92E7D1
:10EEE0000DC089EE92E70AC01092D2088CEA90E732
:10EEF00005C08EEC92E702C084ED92E721E02093FA
:10EF0000020F20E040E060E070E00C94933F0C942E
:10EF1000604DFC01A081B1811C92A281B3818C91D2
:10EF20008F5F8C930280F381E02D90818CE0899F2C
:10EF3000800D1124ECEEFBE013AE84AF08958091B8
:10EF40001E09882369F08091D1088770873041F4C9
:10EF50008CE998E19093D8048093D70410921E090D
:10EF60000895CF92DF92EF92FF920F931F930F9429
:10EF7000760200917C0410917D0420917E043091F2
:10EF80007F046B017C01C01AD10AE20AF30AF7FC84
:10EF900013C020917B04209520937B04DC01CB01DE
:10EFA0008A549C4FAF4FBF4F80937C0490937D0455
:10EFB000A0937E04B0937F0481E090917B04911133
:10EFC00001C080E01F910F91FF90EF90DF90CF90F4
:10EFD00008952F923F924F925F926F927F928F92FD
:10EFE0009F92AF92BF92CF92DF92EF92FF920F93D8
:10EFF0001F93CF93DF93CDB7DEB728970FB6F89462
:10F00000DEBF0FBECDBF1092580F80910A0F109235
:10F010000A0F882311F120E040E060E070E088EF03
:10F0200092E70E94933F28960FB6F894DEBF0FBE7A
:10F03000CDBFDF91CF911F910F91FF90EF90DF90A7
:10F04000CF90BF90AF909F908F907F906F905F9088
:10F050004F903F902F900C94B752209164023091C2
:10F0600065024091040F5091050FC901840F951F4F
:10F070002436310559F44730510514F0069723C062
:10F080004A3F5F4F0CF005C506961DC0243631057A
:10F090002CF4853691050CF0FCC405C0843691052E
:10F0A0000CF4F7C403C08A3091053CF0883EA3E01D
:10F0B0009A072CF087EE93E002C08AE090E02817D0
:10F0C000390731F411C08A30910584F78AE090E065
:10F0D00090936502809364021092040F1092050FC2
:10F0E0001092060F1092070F8091030F882309F4E6
:10F0F00092C26091330870913408072E000C880B7F
:10F10000990B0F94072AB1E0B98320912F08309111
:10F11000300840913108509132080F949F321816F0
:10F120000CF0198260914A0870914B08072E000C70
:10F13000880B990B0F94072A2091460830914708B5
:10F1400040914808509149080F949F3218161CF4BA
:10F15000E981E260E9836091240870912508072E17
:10F16000000C880B990B0F94072A209120083091EE
:10F17000210840912208509123080F949F321816BD
:10F180001CF4F981F460F98329812093A90420916A
:10F19000A8083091A9084091AA085091AB08609145
:10F1A00072027091730280917402909175020F94B3
:10F1B00079304B015C012091AC083091AD08409151
:10F1C000AE085091AF0860917602709177028091FD
:10F1D0007802909179020F94793069837A838B83D6
:10F1E0009C832091B0083091B1084091B2085091B1
:10F1F000B30860917A0270917B0280917C029091B9
:10F200007D020F9479302B013C0120E030E04AE789
:10F2100054E40F94662A6B017C0120E030E0A901E0
:10F22000C301B2010F94012A87FF05C020E030E03E
:10F2300040EA50EC04C020E030E040EA50E4C7016E
:10F24000B6010F94793020E030E040E251E40F94B1
:10F2500055310F94BD312B013C0197FF0AC07094CA
:10F26000609450944094411C511C611C711C8DE2AF
:10F2700001C080E28093590F30E1431637E2530614
:10F280006104710494F0C301B20120E137E240E06F
:10F2900050E00F947433CA01B9012AE030E040E035
:10F2A00050E00F947433605D01C060E260935A0FC8
:10F2B00048EE441643E054066104710494F0C3011F
:10F2C000B20128EE33E040E050E00F947433CA01FD
:10F2D000B9012AE030E040E050E00F947433605D03
:10F2E00001C060E260935B0FC301B20124E630E02D
:10F2F00040E050E00F9474336AE0C62ED12CE12C2C
:10F30000F12CCA01B901A70196010F947433605D15
:10F3100060935C0FC301B201A70196010F9474338F
:10F320006D83662389F08EE280935D0FCA01B90177
:10F33000A70196010F947433605D60935E0F6D8139
:10F34000605D60935F0F17C0CA01B901A701960104
:10F350000F947433662339F08EE280935D0F605D05
:10F3600060935E0F05C080E280935E0F80935D0F17
:10F3700080E280935F0F69E57FE081EA94E00F947B
:10F38000F23320E030E0A901C501B4010F94012A55
:10F3900087FF05C020E030E040E05FEB04C020E0E4
:10F3A00030E040E05FE3C501B4010F9479300F9481
:10F3B000BD31CB010E9448F6BC018CE994E00F946A
:10F3C000F23320E030E0A90169817A818B819C8150
:10F3D0000F94012A87FF05C020E030E040E05FEB9A
:10F3E00004C020E030E040E05FE369817A818B81F6
:10F3F0009C810F9479300F94BD31CB010E9448F667
:10F40000BC0187E994E00F94F2330E94BD40882349
:10F4100021F180913F0D9091400DA091410DB0914F
:10F42000420D0097A105B105C1F0BC01CD016D5998
:10F430007F4F8F4F9F4F24E630E040E050E00F9425
:10F440003D306091430D7091440D8091450D909138
:10F45000460D0F943D30298301C019820E943B8BD9
:10F460006B017C016D8380910B029981891709F4EE
:10F4700042C090930B02A8E49A9FB001112480E04F
:10F4800090E00F94052A2AE037ED43E25CE30F9405
:10F49000662A0F94C23160939604B981B11103C0FA
:10F4A0001092910428C0E981E43630F08E2F64E692
:10F4B0000F944133805D01C080E280935D0FF9813C
:10F4C000FA3048F02AE08F2F622F0F9441330F94C7
:10F4D0004133905D01C090E290935E0F89816AE0B4
:10F4E0000F944133905D90935F0F6DE57FE081E96C
:10F4F00094E00F94F23380910A022D81281709F4C9
:10F500008AC0C0920A02C701B60120E13EE040E095
:10F5100050E00F943D30122FB32E29833A835CE3E1
:10F52000452E512C612C712CC701B601A30192010B
:10F530000F943D30CA01B901A30192010F943D30EF
:10F54000A62E972E30E8C31631E5D30631E0E30648
:10F55000F10450F1C701B60120E831E541E050E087
:10F560000F943D3079019F92AF9289819A8168E131
:10F5700070E00F944D339F938F933F932F9382E0CE
:10F5800099E19F938F9381E894E09F938F930F94D9
:10F590009B290FB6F894DEBF0FBECDBF9AE0E916E7
:10F5A000F10488F189E030C0A981BA81A436B1059F
:10F5B000A8F47F936F93BF921F9386EF98E19F9378
:10F5C0008F9381E894E09F938F930F949B290FB6BC
:10F5D000F894DEBF0FBECDBF85E016C07F936F935A
:10F5E000BF921F938CEE98E19F938F9381E894E0F4
:10F5F0009F938F930F949B290FB6F894DEBF0FBE95
:10F60000CDBF86E001C088E09AEF899F802D11244C
:10F61000805880938004A5DC182F81E00E947252EC
:10F620008091A904282F247082FD03C042E102E0EA
:10F6300002C048E00CE08091240C90E044977CF4F8
:10F640008091260C841758F0211126C287E899E191
:10F650007C0123E060E580EF9BE00E941AFE809130
:10F66000240C8431B8F48091260C823098F0112358
:10F6700009F415C28091DA07882309F410C281E5E4
:10F6800099E17C0102E123E042E068E680EF9BE043
:10F690000E941AFE8091240C8C3108F074C12EE077
:10F6A000A22E28E0B22E8BE298E098878F8338EA6A
:10F6B000832E32E0932E9FE09983C12CD12C43E01E
:10F6C000242E312CEC2D3C2DAF81B88514964D9015
:10F6D0005D906D907C90179718968D919C911997DD
:10F6E0009E838D838091240C843138F58091260C83
:10F6F000883018F1CC2009F4D8C162E2D4012C91F1
:10F700008091A90490E0A0E0B0E004C0B695A79570
:10F71000979587953A95D2F70E2E000CFF0BEE0FBA
:10F72000FF1F80FFBFC1E95EF64EE590F4900CE04C
:10F7300048E080EF9BE00E941AFE8091240C883004
:10F74000B8F5111104C0F5018481811131C02D81FA
:10F750003E81B901330F880B990B0F94072A20E0E3
:10F7600030E040E05FE30F9479300F94BD31CB017E
:10F770000E94C9F6FC018081803209F09AC1818122
:10F78000803209F494C182E0A101481B51094E0F57
:10F790005F1F982F990F890F67E0F981F81B8F2F52
:10F7A0000E94CE9269E070E080E090E00E94B0910B
:10F7B0008091240C8C3198F58091260C843178F15D
:10F7C00020E030E0A901C301B2010F94793020E0BC
:10F7D00030E040E05FE30F9479300F94BD31CB010E
:10F7E0000E94C9F6FC018081803209F066C18181E6
:10F7F000803209F460C192E0A101491B51094E0F0A
:10F800005F1F892F880F980F6CE18981891B0E94E7
:10F81000CE9269E070E080E090E00E94B0912FEF1E
:10F82000C21AD20A3981365E398345E0A40EB11C72
:10F830008F819885479698878F839FEF891A990AB9
:10F84000A2E0CA16D10409F03DCFC0902008D090A4
:10F850002108E0902208F09023088091240C883041
:10F86000D0F5111104C080910D08811134C0609150
:10F87000240870912508072E000C880B990B0F9413
:10F88000072A20E030E040E05FE30F9479300F94E6
:10F89000BD31CB010E94C9F6FC018081803209F0A4
:10F8A00010C18181803209F40AC192E043E050E046
:10F8B000491B51094E0F5F1F892F880F980F892F01
:10F8C000819567E0865A0E94CE9269E070E080E000
:10F8D00090E00E94B0918091240C8C3180F5809151
:10F8E000260C843160F120E030E040E05FE3C701A6
:10F8F000B6010F9479300F94BD31CB010E94C9F647
:10F90000FC018081803209F0E0C08181803209F4FD
:10F91000DAC092E043E050E0491B51094E0F5F1FEF
:10F92000892F880F980F892F81956CE1865A0E9444
:10F93000CE9269E070E080E090E00E94B09180910A
:10F94000240C8C3100F58091260C8431E0F08091FC
:10F95000DA078823C1F0B4E68B9FC00111248158D7
:10F960009F4F6FEF70E00F946133CB010E94C9F697
:10F97000AC016CE187E60E94CE9265E270E080E027
:10F9800090E00E94B0910E94BD40882349F0809190
:10F99000240C843328F48091260C8A3208F097C016
:10F9A0008091240C853328F48091260C813308F053
:10F9B000B6C08091240C843328F48091260C8233C5
:10F9C00008F0B4C08091240C8033D8F48091260CC8
:10F9D0008832B8F080919104882361F041E954E0C5
:10F9E00060E387E30E94CE9265E270E080E090E001
:10F9F0000E94B09141E854E060E3809180040E944D
:10FA0000CE928091240C883298F48091260C8D310E
:10FA100078F02BE040E86DE180E00E946CFE809180
:10FA2000240C873228F48091260C8F3108F088C08E
:10FA30008091240C833328F48091260C8B3208F0BB
:10FA400028C18091240C813408F047C18091260C94
:10FA5000863308F442C11092270C8EE38093280C61
:10FA60008DE09FE00E941950898360E870E08DE08E
:10FA70009FE00E947392B981B53108F02EC160E217
:10FA800070E080E090E00E94B091E981EF5FE9834F
:10FA9000F2CF84E690E00ACB8DE899E1D9CD8BE1F5
:10FAA00099E1EFCDED5EF64E40CE68E027CE81E0E5
:10FAB0006BCE83E069CE91E09FCE93E09DCE91E046
:10FAC000F5CE93E0F3CE91E025CF93E023CF07E08E
:10FAD00028E04AE26AE280EF9BE00E94A2FE05E095
:10FAE00022E04CE262E380EF9BE00E94A2FE24E071
:10FAF0004AE061E38AE20E946CFE6091F20B709131
:10FB0000F30B82E380930C0C8BE280930D0C2CE0C2
:10FB10003CE042E380EF9BE00E94D9E341CF24E048
:10FB20004AE461E386E30E946CFE43CF02E0209149
:10FB3000960442E367E380EF9BE00E94A2FE42CF7F
:10FB400083E08093270C36E23093280C68E570E060
:10FB500080E090E00E94B0918BE08093270C46E219
:10FB60004093280C112329F08CE994E00E94CB9259
:10FB70001EC08091960880FDF7CFECE9F4E0FA838F
:10FB8000E983A981BA816D91BA83A983662379F04B
:10FB90006F3234F4062E000C770B880B990B04C0DF
:10FBA0006FE370E080E090E00E94B091EACF88E2DD
:10FBB0008093270CB6E2B093280C69E570E080E0F2
:10FBC00090E00E94B09180E38093270CE6E2E093FE
:10FBD000280C112329F087E994E00E94CB921FC0E2
:10FBE00080919608869580FDF6CF27E934E03A8328
:10FBF0002983A981BA816D91BA83A983662379F09B
:10FC00006F3234F4062E000C770B880B990B04C06E
:10FC10006FE370E080E090E00E94B091EACF8DE465
:10FC20008093270CB6E2B093280C6AE570E080E080
:10FC300090E00E94B09185E58093270CE6E2E09386
:10FC4000280C112329F081EA94E00E94CB92F0CE97
:10FC5000809196088695869580FDF5CF21EA34E05F
:10FC60003A832983A981BA816D91BA83A9836623D6
:10FC700009F4DECE6F3234F4062E000C770B880BBD
:10FC8000990B04C06FE370E080E090E00E94B091B7
:10FC9000E9CF83E00E94725283E08093270C83E3D4
:10FCA0008093280C66E070E080E090E00E94B091C4
:10FCB00081E00E94725280916402909165020E94DC
:10FCC000C9F6AC0163E38CE00E94CE9265E270E07D
:10FCD00080E090E00E94B091B4CE28960FB6F894E0
:10FCE000DEBF0FBECDBFDF91CF911F910F91FF906F
:10FCF000EF90DF90CF90BF90AF909F908F907F90CC
:10FD00006F905F904F903F902F9008950E94B75250
:10FD10003E98469A3C98449A3A98429AEAE0F1E032
:10FD200080818E7F808380910B018095817080938C
:10FD3000090182E08093090F0E9428F910920C0FAC
:10FD400008954F925F926F927F929F92AF92BF926F
:10FD5000CF92DF92EF92FF920F931F93CF93DF9397
:10FD6000CDB7DEB728970FB6F894DEBF0FBECDBF74
:10FD7000FC01DB019C918CE0899F800D1124908116
:10FD8000A92FAA0F9A0F990F9093270C8093280CF4
:10FD90004115510509F49BC059017F01FA83E9839C
:10FDA0007C836B83011103C0142F052F75C0C42EF3
:10FDB000952E0C2D192DD12CAE014B5F5F4FB50147
:10FDC0008C2D992D0E94624EC82E992E4D805E80FA
:10FDD0006F8078844114510461047104C9F0B0E269
:10FDE0004B1651046104710481F0D301C2018D9757
:10FDF000A109B1090297A105B10550F0EBE24E1639
:10FE0000510461047104A9F503C0DD2009F458C050
:10FE1000D7012C918D2D90E0820F911D46972CF0EB
:10FE2000253018F0CE01019674D881E041145104B8
:10FE30006104710409F480E0D80EF70180818D0D12
:10FE40008083DD2081F0DA94AE014B5F5F4FB50116
:10FE5000C8010E94624E8C016D817E818F819885E0
:10FE60000E94B091EECF45284628472809F0A1CF3F
:10FE70002EC0D3940115110509F09ECF0C2D192D1C
:10FE80009BCF0E94B091D7018C918F5F8C9385316D
:10FE900018F0CE0101963DD8AE014B5F5F4FB50122
:10FEA000812F902F0E94624E182F092F6D817E8125
:10FEB0008F819885611571058105910511F707C03E
:10FEC0000115110509F475CF0F5F1F4FD3CF289689
:10FED0000FB6F894DEBF0FBECDBFDF91CF911F915B
:10FEE0000F91FF90EF90DF90CF90BF90AF909F90D9
:10FEF0007F906F905F904F900895CF93DF93EC01C8
:10FF00000E94284C20E040E060E070E0CE01DF91EC
:10FF1000CF910C94933F7F928F929F92AF92BF921A
:10FF2000CF92DF92EF92FF920F931F93CF93DF93C5
:10FF300061E081E00E948138D0917A04C0E02EE730
:10FF4000A22E28E3B22E30EA832E38E1932ED1116F
:10FF50000BC070907904711029C080910A0F109223
:10FF60000A0F81111DC022C0D13061F47090790454
:10FF700081E078125AC080910A0F10920A0F811105
:10FF80003CC053C0D23009F071C0809179048230F6
:10FF900009F580910A0F10920A0F811114C01AC03E
:10FFA0000E94684D809178048111D4C080918D02A7
:10FFB000882309F452C081E0711080E004E024E05D
:10FFC00045EE58E116C080E091EB97DF8091780410
:10FFD0008111C0C080918D02882309F43EC081E068
:10FFE00090917904923009F080E003E02EE34BEC2D
:10FFF00058E16C2F0E94395230C00F94D9008FE91C
:020000021000EC
:10000000C82E87E7D82EE12CF12C00E010E420E088
:1000100030E040E251EC6EE778E088ED98E10F9433
:10002000762480917804811195C080918D02882377
:10003000A1F060917E0870917F0880918008909176
:1000400081080E94974D9C0181E0781280E000E0D9
:1000500048ED58E16C2F0E94DA51CF5FDF5FC53069
:1000600009F075CF86E08093770474C0D33059F4DB
:1000700080917904833041F580910A0F10920A0F24
:1000800081111BC021C0D43059F48091790484308F
:1000900089F580910A0F10920A0F811124C02AC09D
:1000A000D530D9F6809179048530D1F580910A0F49
:1000B00010920A0F81112EC033C083E191EB1DDF36
:1000C00080917804811146C080918D02882329F2A5
:1000D00081E090917904933009F080E003E02EE311
:1000E0004DEB58E186CF8DEE90EB07DF80917804E1
:1000F000811130C080918D02882309F4AECF81E058
:1001000090917904943009F080E003E02EE34FEA07
:1001100058E16FCF0E947E388091780481111AC017
:1001200080918D02882309F498CFBF92AF929F925D
:100130008F92CF9381E090917904953009F080E01F
:100140008F930E9417370F900F900F900F900F9082
:100150000F9083CFDF91CF911F910F91FF90EF9080
:10016000DF90CF90BF90AF909F908F907F90089539
:100170004F925F926F927F929F92AF92BF92CF9277
:10018000DF92EF92FF920F931F93CF93DF93CDB740
:10019000DEB7CA58D1090FB6F894DEBF0FBECDBF87
:1001A000C358DF4F188219821A821B82CD57D04064
:1001B00080915D0390915E03A0915F03B091600315
:1001C000CF57DF4F88839983AA83BB83C158D04020
:1001D000CB57DF4F19821882C558D04084E690E093
:1001E000C957DF4F99838883C758D0401092C30402
:1001F0009E012B573F4F44E050E0BE016F577F4FA9
:10020000CE0189579F4F0E941D41C957DF4F8881FA
:100210009981C758D0400296C957DF4F9983888388
:10022000C758D040CB57DF4F19821882C558D040ED
:1002300081E0C657DF4F8883CA58D0409E012B57B4
:100240003F4F41E050E0BE0166577F4FCE018957D6
:100250009F4F0E941D419E012B573F4F48E450E0A5
:1002600063ED78E0CE0189579F4F0E941D419E01AA
:100270002B573F4F40E150E06AEB77E0CE018957C2
:100280009F4F0E941D418AE097EDA3EABCE3C3584B
:10029000DF4F88839983AA83BB83CD57D0409E01CB
:1002A0002B573F4F44E050E0BE0163587F4FCE01D3
:1002B00089579F4F0E941D419E012B573F4F4CE095
:1002C00050E06AEC74E0CE0189579F4F0E941D41B7
:1002D0009E012B573F4F4CE050E066E778E0CE019F
:1002E00089579F4F0E941D4119821A821B821C82CE
:1002F0009E012B573F4F41E050E06AE872E0CE018B
:1003000089579F4F0E941D419E012B573F4F44E04C
:1003100050E08E010F5F1F4FB801CE0189579F4FEC
:100320000E941D4180E090E0A0E2B1E489839A83BD
:10033000AB83BC839E012B573F4F44E050E0B80194
:10034000CE0189579F4F0E941D41C358DF4F18822D
:1003500019821A821B82CD57D0407E018DE6E80EAD
:10036000F11C83E0F701808389839E012B573F4F67
:1003700044E050E0BE0163587F4FCE0189579F4F44
:100380000E941D419E012B573F4F41E050E0B701B5
:10039000CE0189579F4F0E941D419E012B573F4F11
:1003A00041E050E0B801CE0189579F4F0E941D41A6
:1003B0007AE0D72EDA949E012B573F4FDD2059F07B
:1003C00044E050E0BE0163587F4FCE0189579F4FF4
:1003D0000E941D41EFCF4CE050E06EE073E0CE0193
:1003E00089579F4F0E941D41C358DF4F18821982C1
:1003F0001A821B82CD57D0406AE0D62EDA94DD20D7
:1004000071F09E012B573F4F44E050E0BE0163580E
:100410007F4FCE0189579F4F0E941D41EFCF83E050
:10042000C757DF4F8883C958D040EA968FAFEA9705
:1004300088E0F701982F11929A95E9F7F801119247
:100440008A95E9F7C358DF4F188219821A821B82F6
:10045000CD57D0409E012B573F4F41E050E0BE01A9
:1004600067577F4FCE0189579F4F0E941D419E01C4
:100470002B573F4F41E050E0BE0167587F4FCE0100
:1004800089579F4F0E941D419E012B573F4F48E0C7
:1004900050E0B801CE0189579F4F0E941D419E0137
:1004A0002B573F4F48E050E0B701CE0189579F4F8F
:1004B0000E941D415AE0C52ED12CF1E0CF1AD1087F
:1004C00071F09E012B573F4F44E050E0BE0163584E
:1004D0007F4FCE0189579F4F0E941D41EECFF701FC
:1004E00010828FEF89839E012B573F4F41E050E0F0
:1004F000B701CE0189579F4F0E941D419E012B5786
:100500003F4F41E050E0B801CE0189579F4F0E9414
:100510001D4180E1F80111928A95E9F79E012B5760
:100520003F4F40E150E0B801CE0189579F4F0E94F4
:100530001D4119829E012B573F4F41E050E0B80109
:10054000CE0189579F4F0E941D419E012B573F4F5F
:1005500044E050E061EA7FE0CE0189579F4F0E945E
:100560001D419E012B573F4F44E050E06DE97FE075
:10057000CE0189579F4F0E941D419E012B573F4F2F
:1005800042E050E06BE97FE0CE0189579F4F0E9427
:100590001D419BE2C92E98E0D92E29E5A22E28E024
:1005A000B22E34E1932E412C512C40E8642E4FE3BF
:1005B000742EF801892D11928A95E9F74D865E8691
:1005C0006F86788AF60183859485A585B6858983AB
:1005D0009A83AB83BC832CEA35EC47E25EE3678504
:1005E0007089818992890F9455316D837E838F83C1
:1005F00098872CEA35EC47E25EE3F601638974895B
:10060000858996890F94662A69877A878B879C8764
:100610009E012B573F4F44E150E0B801CE0189576E
:100620009F4F0E941D41F7E1CF0ED11CAC14BD04B9
:1006300009F0BFCF84E190E09A8389839E012B5714
:100640003F4F42E050E0B801CE0189579F4F0E94D2
:100650001D418CE0EAEAF2E0D80101900D928A9502
:10066000E1F79E012B573F4F4CE050E0B801CE011F
:1006700089579F4F0E941D4180918B0290918C025F
:100680009A8389839E012B573F4F42E050E0B80187
:10069000CE0189579F4F0E941D4181E089839E01B1
:1006A0002B573F4F41E050E0B801CE0189579F4F93
:1006B0000E941D4180E2E6EBF2E0D80101900D922C
:1006C0008A95E1F79E012B573F4F40E250E0B80179
:1006D000CE0189579F4F0E941D41F70110829E0154
:1006E0002B573F4F41E050E0B701CE0189579F4F54
:1006F0000E941D419E012B573F4F41E050E060ECAE
:1007000078E0CE0189579F4F0E941D419E012B57D3
:100710003F4F48E050E069EC78E0CE0189579F4FA9
:100720000E941D418CE1F80111928A95E9F79E0122
:100730002B573F4F4CE150E0B801CE0189579F4FF6
:100740000E941D4188E3E6EDF2E0D80101900D9290
:100750008A95E1F79E012B573F4F48E350E0B801DF
:10076000CE0189579F4F0E941D4188E0F8011192E8
:100770008A95E9F79E012B573F4F48E050E0B801BA
:10078000CE0189579F4F0E941D418EE0F8011192C2
:100790008A95E9F79E012B573F4F4EE050E0B80194
:1007A000CE0189579F4F0E941D41C358DF4F1882C9
:1007B00019821A821B82CD57D0409E012B573F4F82
:1007C00044E050E0BE0163587F4FCE0189579F4FF0
:1007D0000E941D419E012B573F4F44E050E0BE0157
:1007E00063587F4FCE0189579F4F0E941D418CE077
:1007F000D82EF8018D2D11928A95E9F79E012B577D
:100800003F4F4CE050E0B801CE0189579F4F0E9406
:100810001D418CE6F80111928A95E9F79E012B574C
:100820003F4F4CE650E0B801CE0189579F4F0E94E0
:100830001D419E012B573F4F4CE050E067EB74E0A9
:10084000CE0189579F4F0E941D419E012B573F4F5C
:1008500040E150E06BE87FE0CE0189579F4F0E9456
:100860001D419E012B573F4F44E050E062E878E085
:10087000CE0189579F4F0E941D41F7011192DA94D2
:10088000E9F7C757DF4F1882C958D04080E090E0A1
:10089000A0E4B0E4ED968CAF9DAFAEAFBFAFED97E7
:1008A0009E012B573F4F4CE050E0B701CE018957D6
:1008B0009F4F0E941D419E012B573F4F41E050E04A
:1008C000BE0167577F4FCE0189579F4F0E941D4140
:1008D0009E012B573F4F44E050E0BE0167587F4FC9
:1008E000CE0189579F4F0E941D411091C3041111E1
:1008F00056C0C957DF4FC880D980C758D040F4E6EA
:10090000CF1AD108CB57DF4F88819981C558D04085
:10091000F7019183808384E690E0C957DF4F998384
:100920008883C758D0409E012B573F4F44E050E08A
:100930006AE173E0CE0189579F4F0E941D419E01DD
:100940002B573F4F42E050E0B701CE0189579F4FF0
:100950000E941D410F943B11B60181EC99E10F9467
:10096000FE10F7014081518160E070E084EB99E175
:100970000F94EE1081EB99E10F94DF10FFEACF1690
:10098000F2E0DF0639F00F94381183ED99E10F940E
:10099000DF1011E08091C304182B1093C3049091D1
:1009A000C30481E08927C657DF4F0FB6F894DEBF36
:1009B0000FBECDBFDF91CF911F910F91FF90EF90B0
:1009C000DF90CF90BF90AF909F907F906F905F909F
:1009D0004F9008954F925F926F927F928F929F9265
:1009E000AF92BF92CF92DF92EF92FF92CF9340905F
:1009F0007202509073026090740270907502809041
:100A0000760290907702A0907802B0907902C09020
:100A10007A02D0907B02E0907C02F0907D020E94EE
:100A200096C50E9493D0C0E08C2F0E94E7D540E08D
:100A300060E08C2F0E9419D7CF5FC330A9F70E94C6
:100A4000DDC5209172023091730240917402509181
:100A50007502C301B2010F94012A81111CC0A501C6
:100A60009401609176027091770280917802909162
:100A700079020F94012A81110EC020917A023091DF
:100A80007B0240917C0250917D02C701B6010F9418
:100A9000012A882379F0CF91FF90EF90DF90CF90DB
:100AA000BF90AF909F908F907F906F905F904F908E
:100AB0000D94E00BCF91FF90EF90DF90CF90BF901F
:100AC000AF909F908F907F906F905F904F90089520
:100AD0003F924F925F926F927F928F929F92AF92CE
:100AE000BF92CF92DF92EF92FF920F931F93CF931B
:100AF000DF93CDB7DEB7C558D1090FB6F894DEBF86
:100B00000FBECDBF4DB65EB6EF961FAE1EAEEF97D1
:100B100084E690E0C158DF4F99838883CF57D04057
:100B200001E09E0123583F4F44E050E0BE0167586A
:100B30007F4FCE0181589F4F0E94E0409E01235875
:100B40003F4F42E050E0BE016F577F4FCE018158CA
:100B50009F4F0E94E04043E050E0BE0167587F4F46
:100B60008AE193E00F94F933892BE9F0ED968FAD8C
:100B7000ED97882339F08FE3EA968FAFEA97EB96EB
:100B80001FAEEB970F943B11BE0167587F4F8BE66A
:100B90009AE10F9426118DE59AE10F94DF1081E020
:100BA0008093C30440C5E9961CAE1DAE1EAE1FAEB9
:100BB000E997EF961FAE1EAEEF9701E09E01235816
:100BC0003F4F41E050E0BE016B577F4FCE0181584F
:100BD0009F4F0E94E0406DB67EB6CB57DF4FE88056
:100BE000C558D040F12C23E0E20EF11CEE0CFF1CA6
:100BF000EE0CFF1C8DB79EB78E199F090FB6F894A7
:100C00009EBF0FBE8DBFEDB7FEB731964F018E1957
:100C10009F090FB6F8949EBF0FBE8DBFEDB7FEB70C
:100C200031966F018E199F090FB6F8949EBF0FBEC3
:100C30008DBFEDB7FEB731965F0100918A0F11E0CD
:100C400001279E0123583F4FA701B401CE018158CF
:100C50009F4F0E94E04000918A0F01279E01235878
:100C60003F4F44E050E063EE78E0CE0181589F4F63
:100C70000E94E04000918A0F01279E0123583F4FB8
:100C8000A701B601CE0181589F4F0E94E04000911C
:100C90008A0F01279E0123583F4FA701B501CE01BE
:100CA00081589F4F0E94E04000918A0F002309F471
:100CB000F0C011E001279E0123583F4F44E050E06F
:100CC00067E079E0CE0181589F4F0E94E04000919B
:100CD0008A0F01279E0123583F4F44E050E06BE00C
:100CE00079E0CE0181589F4F0E94E04000918A0F29
:100CF00001279E0123583F4F44E050E06FE079E028
:100D0000CE0181589F4F0E94E04000918A0F012739
:100D10009E0123583F4F44E050E063E179E0CE016B
:100D200081589F4F0E94E04000918A0F01279E0149
:100D300023583F4F44E050E067E179E0CE0181580D
:100D40009F4F0E94E04000918A0F01279E01235887
:100D50003F4F40E150E06AEB77E0CE0181589F4F72
:100D60000E94E04000918A0F01279E0123583F4FC7
:100D700044E050E0BE016B587F4FCE0181589F4F39
:100D80000E94E0400FB6F8947EBE0FBE6DBE00918B
:100D90008A0F01279E0123583F4F4CE050E06AEC38
:100DA00074E0CE0181589F4F0E94E04000918A0F6D
:100DB00001279E0123583F4F4CE050E066E778E062
:100DC000CE0181589F4F0E94E04000918A0F012779
:100DD0009E0123583F4F41E050E06AE872E0CE01A7
:100DE00081589F4F0E94E04000918A0F01279E0189
:100DF00023583F4F44E050E0BE016F5F7F4FCE016C
:100E000081589F4F0E94E04000918A0F01279E0168
:100E100023583F4F44E050E0BE016B587F4FCE0156
:100E200081589F4F0E94E04000918A0F01279E0148
:100E300023583F4F44E050E0BE016B587F4FCE0136
:100E400081589F4F0E94E04001E09E0123583F4F90
:100E500041E050E0BE0163597F4FCE0181589F4F62
:100E60000E94E0409E0123583F4F41E050E0BE0108
:100E70006F5F7F4FCE0181589F4F0E94E040AE963A
:100E80008FADAE97C9808C9D60011124E12CF12CAF
:100E90008AC0CB57DF4F2881C558D04030E02E5F45
:100EA0003F4FD60143ED58E080E090E02817390726
:100EB00034F0F401C080D180E280F38010C0FC01E6
:100EC0008430910510F0E3E0F0E0EE0FFF1FEE0F2D
:100ED000FF1FE257F74CC590D590E590F490FA01CA
:100EE000C192D192E192F192AF01281739075CF0DB
:100EF000EC9111967C91119712966C911297139622
:100F0000FC91139714C0FC018430910510F0E3E0CC
:100F1000F0E0EE0FFF1FEE0FFF1FE258F74CC590F9
:100F2000D590E590F490EC2D7D2D6E2DFF2DCE2EDD
:100F3000D72EE62EFF2EFA01C08AD18AE28AF38AE2
:100F40002817390734F0F5011081718162813380EF
:100F500014C0FC018430910510F0E3E0F0E0EE0FE6
:100F6000FF1FEE0FFF1FE259F74CC590D590E5909B
:100F7000F4901C2D7D2D6E2D3F2CC12ED72EE62EEC
:100F8000F32CFA01C0A2D1A2E2A2F3A20196F4E0EE
:100F9000AF0EB11C149664E0860E911C843091054E
:100FA00009F084CF86CE00918A0FEC14FD0491F0F5
:100FB00001279E0123583F4F44E050E0BE016B588B
:100FC0007F4FCE0181589F4F0E94E0408FEFE81A7B
:100FD000F80AE9CF81E008279E0123583F4F4CE0F3
:100FE00050E0BE016F5F7F4FCE0181589F4F0E943E
:100FF000E0401AE0FF24F394115089F000918A0F29
:101000000F259E0123583F4F44E050E0BE016B582E
:101010007F4FCE0181589F4F0E94E040EDCF01E00D
:101020009E0123583F4F41E050E0BE016C577F4F77
:10103000CE0181589F4F0E94E0409E0123583F4FB0
:1010400041E050E0BE016D577F4FCE0181589F4F68
:101050000E94E04000918A0F11E001279E01235871
:101060003F4F48E050E0BE0163597F4FCE018158A9
:101070009F4F0E94E04000918A0F01279E01235854
:101080003F4F48E050E0BE016F5F7F4FCE01815877
:101090009F4F0E94E040CC57DF4F8881C458D0401A
:1010A000CD57DF4FC880C358D0408C9D60011124BC
:1010B000E12CF12C00918A0FCE14DF0491F001276E
:1010C0009E0123583F4F44E050E0BE016B587F4FD4
:1010D000CE0181589F4F0E94E0409FEFE91AF90A24
:1010E000E9CF11E001279E0123583F4F41E050E036
:1010F000BE0163597F4FCE0181589F4F0E94E0404F
:1011000000918A0F01279E0123583F4F41E050E094
:10111000BE016F5F7F4FCE0181589F4F0E94E0401C
:1011200000918A0F01279E0123583F4F40E150E074
:10113000BE016F5F7F4FCE0181589F4F0E94E040FC
:1011400000918A0F01279E0123583F4F41E050E054
:10115000BE016F5F7F4FCE0181589F4F0E94E040DC
:1011600000918A0F01279E0123583F4F44E050E031
:1011700061EA7FE0CE0181589F4F0E94E0400091DC
:101180008A0F01279E0123583F4F44E050E06DE94C
:101190007FE0CE0181589F4F0E94E04000918A0F6E
:1011A00001279E0123583F4F42E050E06BE97FE06A
:1011B000CE0181589F4F0E94E0408BE2E82E88E0EC
:1011C000F82E12E0DD24D39400918A0F0D259E01A4
:1011D00023583F4F44E150E0BE016F5F7F4FCE0187
:1011E00081589F4F0E94E04000918A0F011131C049
:1011F00089809A80AB80BC8020E030E84BE355E4E6
:10120000C501B4010F94012A882319F1F7018386DF
:101210009486A586B6862CEA35EC47E25EE36D81BE
:101220007E818F8198850F94662AF7016787708B7E
:10123000818B928B2CEA35EC47E25EE369857A85F7
:101240008B859C850F945531F701638B748B858B4F
:10125000968B1150F7E1EF0EF11C1111B5CF11E093
:1012600001279E0123583F4F42E050E0BE016F5FCF
:101270007F4FCE0181589F4F0E94E04000918A0F1E
:1012800001279E0123583F4F4CE050E0BE016F5FA5
:101290007F4FCE0181589F4F0E94E04000918A0FFE
:1012A00001279E0123583F4F42E050E0BE016F5F8F
:1012B0007F4FCE0181589F4F0E94E04089819A81E3
:1012C0000E94855200918A0F01279E0123583F4FAB
:1012D00041E050E0BE016F5F7F4FCE0181589F4FCC
:1012E0000E94E04000918A0F01279E0123583F4F42
:1012F00040E250E0BE016F5F7F4FCE0181589F4FAB
:101300000E94E04000918A0F01279E0123583F4F21
:1013100041E050E0BE0163597F4FCE0181589F4F9D
:101320000E94E04000918A0F01279E0123583F4F01
:1013300049E050E0BE016F5F7F4FCE0181589F4F63
:101340000E94E04000918A0F01110CC089818093B6
:10135000C00888E0FE013296A9ECB8E001900D9239
:101360008A95E1F711E001279E0123583F4F4CE198
:1013700050E0BE016F5F7F4FCE0181589F4F0E94AA
:10138000E04000918A0F01279E0123583F4F48E318
:1013900050E0BE016F5F7F4FCE0181589F4F0E948A
:1013A000E04000918A0F01279E0123583F4F48E0FB
:1013B00050E0BE016F5F7F4FCE0181589F4F0E946A
:1013C000E04000918A0F01279E0123583F4F4EE0D5
:1013D00050E0BE016F5F7F4FCE0181589F4F0E944A
:1013E000E04000918A0F01279E0123583F4F48E0BB
:1013F00050E0BE016F5F7F4FCE0181589F4F0E942A
:10140000E04000918A0F01279E0123583F4F4CE096
:1014100050E0BE016F5F7F4FCE0181589F4F0E9409
:10142000E04000918A0F01279E0123583F4F4CE670
:1014300050E0BE016F5F7F4FCE0181589F4F0E94E9
:10144000E04019821A821B821C821D821E821F822A
:10145000188619861A861B861C8600918A0F01271A
:101460009E0123583F4F4CE050E0BE016F5F7F4F1D
:10147000CE0181589F4F0E94E04000918A0F0127C2
:101480009E0123583F4F40E150E06BE87FE0CE01E2
:1014900081589F4F0E94E04000918A0F01279E01D2
:1014A00023583F4F44E050E062E878E0CE01815895
:1014B0009F4F0E94E04000918A0F01279E01235810
:1014C0003F4F4CE050E0BE016F5F7F4FCE0181582F
:1014D0009F4F0E94E04000918A0F01279E012358F0
:1014E0003F4F41E050E0BE016D577F4FCE01815824
:1014F0009F4F0E94E04000918A0F01279E012358D0
:101500003F4F44E050E0BE0163597F4FCE01815808
:101510009F4F0E94E040C158DF4F88819981CF578B
:10152000D0408331934041F00F94381183ED99E11D
:101530000F94DF1081E001C080E08093C304882312
:10154000C1F00F943B11C158DF4F68817981CF57AB
:10155000D0406456710985E59AE10F941A116FEA3B
:1015600072E08DE49AE10F94FE108AE00E947141CE
:1015700051C0EF962EAD3FADEF97CF57DF4F88812B
:101580009981C158D04028173907D1F081E0809364
:10159000C3040F943811CF57DF4F68817981C15848
:1015A000D0408DE29AE10F94FE10EF966EAD7FADC4
:1015B000EF9788E29AE10F94FE1088E19AE128C043
:1015C00080918A0F811126C00F943B110AE113E02C
:1015D000F80181918F01882319F00E947141F8CFA1
:1015E000C158DF4F68817981CF57D0406456710967
:1015F0008BEF99E10F941A11EF964EAD5FADEF9717
:1016000060E070E08EEE99E10F94EE108BEE99E1C0
:101610000F94DF1080918A0F811105C08091C3045F
:10162000811101C0D7D980918A0F811102C00F9416
:101630008E0C9091C30481E089270FB6F8945EBEAA
:101640000FBE4DBECB57DF4F0FB6F894DEBF0FBEB7
:10165000CDBFDF91CF911F910F91FF90EF90DF9061
:10166000CF90BF90AF909F908F907F906F905F9042
:101670004F903F9008950F931F938091AA0481305B
:1016800019F40F94760208C06091B3047091B40409
:101690008091B5049091B6040091AF041091B0040C
:1016A0002091B1043091B204601B710B820B930B3B
:1016B00028EE33E040E050E00F943D308091AB04E1
:1016C0009091AC04A091AD04B091AE04BC01CD01E9
:1016D000620F731F841F951F1F910F910895109221
:1016E000AA041092AF041092B0041092B1041092A8
:1016F000B2041092B3041092B4041092B504109284
:10170000B6041092AB041092AC041092AD04109287
:10171000AE0408958091AA048130E1F0823051F442
:10172000AADF6093AB047093AC048093AD049093F4
:10173000AE0401C0D4DF81E08093AA040F94760246
:101740006093AF047093B0048093B1049093B2049B
:1017500081E0089580E008958091AA04813079F4B1
:1017600082E08093AA040F9476026093B30470938E
:10177000B4048093B5049093B60481E0089580E0AA
:1017800008958091AA048150823010F080E008957D
:101790001092AA040F9476026093B3047093B40479
:1017A0008093B5049093B60481E008958F929F9240
:1017B000AF92BF92CF92DF92EF92FF92CF93FC0154
:1017C000C080D180E280F38020E030E0A901C70131
:1017D000B6010F94012A87FF08C0C701B6019058CF
:1017E00020E030E048EC52E406C020E030E048EC75
:1017F00052E4C701B6010F94662A20E030E040EAC7
:1018000050E40F94793020E030E040E251E40F944E
:1018100055310F94BD316B017C0180E28093590FEB
:10182000F0E1CF16F7E2DF06E104F10494F0C7011E
:10183000B60120E137E240E050E00F947433CA0172
:10184000B9012AE030E040E050E00F947433605D6D
:1018500001C060E260935A0F88EEC81683E0D80694
:10186000E104F10494F0C701B60128EE33E040E052
:1018700050E00F947433CA01B9012AE030E040E02F
:1018800050E00F947433605D01C060E260935B0FC1
:10189000E4E6CE16D104E104F10494F0C701B601E8
:1018A00024E630E040E050E00F947433CA01B901FF
:1018B0002AE030E040E050E00F947433605D01C0F6
:1018C00060E260935C0F8AE0882E912CA12CB12CF1
:1018D000C701B601A50194010F947433C62FCA0144
:1018E000B901A50194010F947433605D60935D0F9D
:1018F0008EE280935E0FC05DC0935F0F89E59FE02D
:10190000CF91FF90EF90DF90CF90BF90AF909F90DE
:101910008F9008952F923F924F925F926F927F9295
:101920008F929F92AF92BF92CF92DF92EF92FF92EF
:101930000F931F93CF9361E081E00E948138C091A3
:101940007A0410E086E3282E8CE1382E92E5492EA9
:101950009CE1592E2CE7622E2BE1722E3DE6A32E40
:101960003BE1B32E42ECE42E4BE1F42E5EE5852EF6
:101970005BE1952E6CECC62E6BE1D62EC1110BC02F
:1019800080917904811129C080910A0F10920A0F69
:1019900081111DC022C0C13059F480917904813079
:1019A000C9F580910A0F10920A0F811127C032C029
:1019B000C23009F04FC080917904823009F064C0D0
:1019C00080910A0F10920A0F811152C05DC00E94CF
:1019D000684D80917804811164C380918D028823C1
:1019E00081F181E090917904911180E004E024E09C
:1019F00043ED5BE2612F0E94395223C08CE89AE1EB
:101A00009093D8048093D7040E94EE6F809178045D
:101A1000811147C380918D02882399F01F928EE631
:101A20009CE19F938F931F9381E090917904913073
:101A3000D1F58F930E9417370F900F900F900F9052
:101A40000F901F5FCF5F153009F098CF85E180932D
:101A5000770427C3C33049F580917904833009F0B6
:101A60004CC080910A0F10920A0F81113AC045C0F4
:101A70008BE99AE19093D8048093D7040E94EE6F8B
:101A80008091780481110DC380918D028823C9F261
:101A90001F9285E69CE19F938F931F9381E0909125
:101AA0007904923031F280E0C4CFC43061F4809187
:101AB0007904843009F04CC080910A0F10920A0F0B
:101AC00081113AC045C0C53049F58091790485300F
:101AD00009F06AC080910A0F10920A0F811158C054
:101AE00063C08AEA9AE19093D8048093D7040E9455
:101AF000EE6F809178048111D4C280918D02882389
:101B000009F49FCF1F928CE59CE19F938F931F93C5
:101B100081E090917904933031F68BCFC63051F546
:101B200080917904863009F06BC080910A0F109281
:101B30000A0F811159C064C089EB9AE19093D804CF
:101B40008093D7040E94EE6F809178048111A9C21E
:101B500080918D02882309F474CF1F9289E49CE15F
:101B60009F938F931F9381E090917904943009F0B3
:101B70009ACF5FCFC73051F580917904873009F053
:101B80006BC080910A0F10920A0F811159C064C076
:101B900088EC9AE19093D8048093D7040E94EE6F6A
:101BA0008091780481117DC280918D02882309F48F
:101BB00048CF1F9280E49CE19F938F931F9381E015
:101BC00090917904953009F06ECF33CFC83051F53C
:101BD00080917904883009F06BC080910A0F1092CF
:101BE0000A0F811159C064C087ED9AE19093D8041F
:101BF0008093D7040E94EE6F80917804811151C2C6
:101C000080918D02882309F41CCF1F928DE29CE104
